:100000000C9467080C9486080C9486080C94E20BF8
:100010000C94180C0C9486080C9486080C94860892
:100020000C9486080C9486080C9486080C94860818
:100030000C9486080C9486080C9486080C94B70FD0
:100040000C9486080C9486080C9486080C948608F8
:100050000C946D720C9479690C9486080C94860843
:100060000C9486080C944F6A0C9486080C94436A8E
:100070000C9486080C9486080C9486080C948608C8
:100080000C94307E0C9486080C9486080C94860898
:100090000C948D6A0C9486080C94816A0C948608E2
:1000A0000C9486080C9486080C9486080C94860898
:1000B0000C9486080C9486080C9486080C94860888
:1000C0000C9486080C9486080C9486080C94860878
:1000D0000C9486080C9486080C9486080C94860868
:1000E0000C9486080C9426720C9430720C941C723A
:1000F0000C94D6710C9461720C9452720C944672EA
:100100000C943A720C9486080C9486080C94860819
:100110000C9486080C9486080C9486080C94860827
:10012000084AD73B3BCE016E84BCBFFDC12F3D6C5E
:1001300074319ABD56833DDA3D00C77F11BED9E4C4
:10014000BB4C3E916BAAAABE000000803F076342F1
:1001500036B79BD8A71A39685618AEBAAB558C1D5E
:100160003CB7CC5763BD6DEDFD753EF6177231BFE0
:10017000000000803F08000000BE922449123EAB00
:10018000AAAA2ABECDCCCC4C3E00000080BEABAAB1
:10019000AAAA3E00000000BF000000803F0000004F
:1001A0000000084178D3BB4387D1133D190E3CC3EF
:1001B000BD4282AD2B3E68EC8276BED98FE1A93E6E
:1001C0004C80EFFFBE01C4FF7F3F000000000050E5
:1001D0003A20256C642050612020252D372E326670
:1001E000206D0A002563002563004932433A200050
:1001F00025630074746C3D252D64200074746C3D7F
:10020000252D6420004E65772074746C3D252D6487
:1002100020002563004D533536313120503D252DCA
:10022000372E326620252D372E32666D0A00424D5C
:100230005030383520256C642050612020252D3722
:100240002E32666D00256300545F484541545F4976
:1002500044583D252D352E32662000545F444557C5
:100260003D252D352E3266200041483D252D352E69
:1002700032662000545F53485432583D252D352EA8
:100280003266200052485F53485432583D252D3580
:100290002E32662000545F52483D252D342E3166A3
:1002A000200052483D252D342E3166200025630064
:1002B00025630025630025630043757272656E74C3
:1002C000207265706F727420696E74657276616CED
:1002D0003D252D64207365630A004E6577207265A5
:1002E000706F727420696E74657276616C3D252D35
:1002F00064207365630A002563007265706F727411
:100300005F616C6C3D007265706F72743D002563B7
:1003100000256300256300256300204F53434341BC
:100320004C3D2564200020467573653A2065653D87
:10033000253032782068663D25303278206C663D65
:1003400025303278206C623D25303278004D43559F
:100350003D2530366C7800256300252D31306C75D5
:1003600020252D31306C7520252D31306C752025E0
:100370002D31306C75200A007478206C656E202059
:100380002020207268206D697373202020207268FD
:10039000207374616C652020207268206D6973631E
:1003A0000A002563004F4B0A0025630025630025E2
:1003B000630025630025630064656275675F616C97
:1003C0006C3D0064656275673D0064656275673DFC
:1003D0000025730A0025372E33662025372E336615
:1003E0000025352E326620004572726F7220302053
:1003F000566F6C74004E6F7420737570706F7274EA
:1004000065640A004572726F72203020566F6C74FA
:10041000004572726F72203020566F6C7400257325
:100420000A0073656E743D252D75206475703D2539
:100430002D752069676E6F7265643D252D7520747A
:10044000746C5F7A65726F3D252D750A0074787043
:1004500077723D25640A006368616E3D25640A0079
:100460005465737420362025730A00546573742014
:10047000352025730A005465737420342025730ACF
:10048000005465737420332025730A005465737417
:1004900020322025730A005465737420312025739F
:1004A0000A0025730A0025730A00646565700A0056
:1004B000666F7263655F69646C650A006E6F6E6576
:1004C0000A00707772733D005854414C5F54524992
:1004D0004D3D25640025730A00696E74725F736573
:1004E000635F70313D252D372E33660A00696E74C7
:1004F000725F70313D252D6C640A00696E74725F05
:100500007365635F70303D252D372E33660A0069B1
:100510006E74725F70303D252D6C640A00765F6DDD
:1005200063753D252D352E32660A00707077723D59
:1005300025730A0064656275673D0025730A0061D2
:1005400075746F0A006C6F675F6D6F64653D007551
:1005500073625F7077723D25730A007265706F7207
:10056000743D007265706F72745F696E7465727647
:10057000616C3D252D640A0072656C61793D2573BF
:100580000A0074746C3D252D640A0052494D455F84
:10059000616464723D252D642E252D640A006E650C
:1005A000696768626F725F7461626C655F73697AB4
:1005B000653D25640A00747870773D25640A006300
:1005C00068616E3D25640A006932633D0069643DDF
:1005D000007478743D25730A0053797374656D2037
:1005E00053756D6D6172790A00745F686561745F3F
:1005F00069647800745F64657700616800705F6D9E
:1006000073353631310072685F7368743278007404
:100610005F73687432780070610070006164340048
:1006200061643300616432006164310061330061F0
:100630003200613100765F696E0072680075707417
:10064000696D650070315F740070310070305F74E7
:1006500000703000765F6D637500745F6D637500C8
:100660007431007400696400653634007478740075
:100670006175746F006E6F6E650072656C61795F95
:100680006C65647900636F6D70617373006163639F
:10069000656C007072657300705F707772006165E1
:1006A000730070315F6C6564790070305F6C6564F5
:1006B00072006576656E74006C6564006F7700701B
:1006C0006B740074785F6C6564790072785F6C6538
:1006D0006472006F706572006E6F6E650025303257
:1006E0007800765F6164343D252D382E3666002013
:1006F00000765F6164333D252D382E36660020007C
:10070000765F6164323D252D382E366600200076F6
:100710005F6164313D252D382E3666002000765FFE
:100720006C696768743D252D382E3666002000768A
:100730005F61323D252D372E3366002000765F61E4
:10074000313D252D372E3366002000765F696E3DE2
:10075000252D352E326600204E657665722D757317
:10076000656420737461636B203E20256420627988
:100770007465730A00757074696D653D252D642D6F
:10078000646179732D253032643A253032643A251C
:100790003032642D686F7572730A0074657374204B
:1007A0005B6F66667C317C327C337C347C355D20CB
:1007B000202020202020202D2074657374206D6F50
:1007C0006465730A0D00776474205B6F6E7C6F66DE
:1007D000667C746573745D202020202020202020FA
:1007E00020202D207761746368646F670A0D00759F
:1007F0007067722020202020202020202020202010
:1008000020202020202020202020202D2072656202
:100810006F6F742076696120626F6F746C6F6164B2
:1008200065720A0D00626F6F742020202020202046
:1008300020202020202020202020202020202020B8
:10084000202D207265626F6F740A0D0070777273CD
:10085000205B646565707C666F7263655F69646C5C
:10086000657C6E6F6E655D202D206D637520736CE9
:10087000656570206D6F64650A0D00726573742084
:10088000656570726F6D20202020202020202020A0
:10089000202020202020202D20726573746F726527
:1008A00020656570726F6D0A0D0070707772205B45
:1008B0006F6E7C6F66665D20202020202020202027
:1008C0002020202020202D2070726F6772616D6DB6
:1008D00061626C65207077720A0D00747874205B19
:1008E000737472696E675D202020202020202020F4
:1008F000202020202020202D205365742072657038
:100900006F7274207465787420737472696E670AEC
:100910000D0074787077205B31352D305D202020FC
:1009200020202020202020202020202020202D20BA
:100930005458205077722E20486967686573742078
:100940003020283364426D290A0D0074746C205BDA
:10095000302D31355D202020202020202020202017
:10096000202020202020202D2074696D652D746F9B
:100970002D6C69766520666F72207061636B65749B
:10098000730A0D00737320202020202020202020B7
:100990002020202020202020202020202020202057
:1009A0002D2073797374656D2073756D6D61727927
:1009B0000A0D0072732020202020202020202020DB
:1009C0002020202020202020202020202020202D1A
:1009D00020726164696F2073746174730A0D007210
:1009E00069205B696E745D2020202020202020205B
:1009F00020202020202020202020202D2072657003
:100A00006F727420696E74657276616C0A0D007283
:100A100065205B6D61736B7C6175746F2C6D6173A8
:100A20006B5D2020202020202020202D206D6F7441
:100A300065207265706F72742073657474696E6777
:100A40000A0D006F77202020202020202020202049
:100A50002020202020202020202020202020202D89
:100A6000206F6E652D776972652073656E736F7286
:100A7000730A0D006C6F67205B6175746F7C6F6E1D
:100A80007C6F66665D2020202020202020202020F2
:100A90002D206D6F7465732064617461206F6E200A
:100AA0005553420A0D006E65205B666C7573685D78
:100AB0002020202020202020202020202020202036
:100AC00020202D206E65696768626F7220746162F4
:100AD0006C650A0D006572722020202020202020E5
:100AE0002020202020202020202020202020202006
:100AF000202D206572726F7220696E666F0A0D007C
:100B00006D63752020202020202020202020202000
:100B10002020202020202020202020202D206D6338
:100B20007520696E666F0A0D006964205B726573DB
:100B300065745D20202020202020202020202020DF
:100B400020202020202D2069642068616E646C695B
:100B50006E670A0D0068756D20202020202020205F
:100B60002020202020202020202020202020202085
:100B7000202D2068756D69646974792073656E73C2
:100B80006F720A0D0072656C6179205B6F6E7C6F0D
:100B900066667C73746174735D20202020202020A1
:100BA000202D2072656C6179206E6574776F726B91
:100BB000207265706F7274730A0D006465205B6D3E
:100BC00061736B5D20202020202020202020202009
:100BD000202020202020202D2064656275670A0DCA
:100BE000006368616E205B31312D32365D2020203C
:100BF000202020202020202020202020202D2063A5
:100C000068616E2031312D32362028322E34303555
:100C10002D32343830204D687A290A0D0063616C1A
:100C200069205B5B765F696E7C61317C61325D203F
:100C3000766F6C747C72657365747C6E6F6E655DC7
:100C4000202D2063616C6962726174650A0D006118
:100C5000646320202020202020202020202020200D
:100C600020202020202020202020202D2073686F8D
:100C70007720765F696E2C2061312C2061322076DE
:100C80006F6C74616765730A0D0075202020202049
:100C90002020202020202020202020202020202054
:100CA0002020202020202D20757074696D650A0D8C
:100CB00000762020202020202020202020202020FE
:100CC000202020202020202020202020202D2076C1
:100CD000657273696F6E0A0D006820202020202045
:100CE0002020202020202020202020202020202004
:100CF00020202020202D2068656C700A0D002563BF
:100D000000756E6B6E6F776E20636D640A00484DE0
:100D100043353838330025730025730020257300D0
:100D20002025362E32662000253032780074656D1D
:100D3000705F65787465726E3D252D362E326600C3
:100D4000202573002025362E3266204F6E2D426FEF
:100D500061726400253032780074656D705F626F77
:100D60006172643D252D362E3266000A004520252D
:100D7000642E256420636C6F636B20256C75206383
:100D8000707520256C75206C706D20256C75206940
:100D9000727120256C7520676C656420256C752048
:100DA000796C656420256C7520726C656420256CF7
:100DB0007520747820256C75206C697374656E20BD
:100DC000256C752073656E736F727320256C7520AA
:100DD00073657269616C20256C750A005320256467
:100DE0002E256420636C6F636B20256C75207478EE
:100DF00020256C7520727820256C752072747820FF
:100E0000256C752072727820256C75207265786D5E
:100E1000697420256C752061636B747820256C756E
:100E2000206E6F61636B747820256C752061636B35
:100E3000727820256C752074696D65646F757420F7
:100E4000256C752062616461636B727820256C7516
:100E500020746F6F6C6F6E6720256C7520746F6FD8
:100E600073686F727420256C752062616473796E8B
:100E7000636820256C752062616463726320256C51
:100E80007520636F6E74656E74696F6E64726F70D7
:100E900020256C752073656E64696E6764726F706F
:100EA00020256C75206C6C747820256C75206C6C1A
:100EB000727820256C750A00257325730A004F6E21
:100EC0006C696E650A000A002C20636865636B20FC
:100ED0007261746520257520487A0025732025737A
:100EE0002C206368616E6E656C20257520706F77AD
:100EF0006572202575000A0025783A004D4143208F
:100F000061646472657373200052616E646F6D205A
:100F10004555493634206164647265737320676592
:100F20006E6572617465640A000A2A2A2A2A2A2ACE
:100F30002A426F6F74696E672025732A2A2A2A2A2B
:100F40002A2A0A00020000FFFE00000141544D451C
:100F5000474131323872666131006C6F63616C6891
:100F60006F737400454550524F4D20697320636F75
:100F700072727570742C20726577726974696E670D
:100F800020776974682064656661756C74732E0AD5
:100F9000006E616E00696E660000407A10F35A00C0
:100FA000A0724E18090010A5D4E80000E876481792
:100FB0000000E40B54020000CA9A3B000000E1F577
:100FC00005000080969800000040420F000000A03D
:100FD0008601000000102700000000E80300000068
:100FE000006400000000000A000000000001000092
:100FF0000000002C76D888DC674F0823DFC1DFAE05
:1010000059E1B1B796E5E3E453C63AE651997696CD
:10101000E8E6C28426EB898C9B62ED407C6FFCEF96
:10102000BC9C9F40F2BAA56FA5F490055A2AF75CC4
:10103000936B6CF9676DC11BFCE0E40D47FEF52076
:10104000E6B500D0ED902E0300943577050080843E
:101050001E080000204E0A000000C80C3333333352
:101060000F986E12831141EF8D2114893BE65516BE
:10107000CFFEE6DB18D1844B381BF77C1D901DA4F6
:10108000BBE424203284725E228100C9F124ECA1E9
:10109000E53D27494E46494E4954594E414ECDCC27
:1010A000CC3D0AD7233C17B7D13877CC2B32959556
:1010B000E6241FB14F0A000020410000C842004052
:1010C0001C4620BCBE4CCA1B0E5AAEC59D741124D2
:1010D0001FBECFEFD1E4DEBFCDBF1AE0A0E0B2E08B
:1010E000E6E3F9E401E00BBF02C007900D92A830DF
:1010F000B107D9F711E3A8E0BAE001C01D92A73704
:10110000B107E1F70E9433680C9499A40C94000095
:1011100029E0FC0120935700C895802D089500D048
:1011200082EC94E0EDB7FEB7928381830E948AA19E
:101130008091EF069091F0060F900F9093FF04C0FE
:1011400000D08CEB94E009C092FF04C000D080EB8B
:1011500094E003C000D08AEA94E0EDB7FEB7928332
:1011600081830E948AA10F900F900895E091951BB2
:10117000F0E0EF71F070E651F44E80838091951BA2
:101180008F5F8093951B8091B12888608093B128F0
:1011900047E157E0CA0161E10E948B5880E090E08E
:1011A0000895EF92FF92CF93DF93E82EE7017E013F
:1011B000F92EE7018091080A9091090A86FF2DC057
:1011C0008DB79EB70C970FB6F8949EBF0FBE8DBF1C
:1011D000EDB7FEB7319680E092E0ADB7BEB712969C
:1011E0009C938E9311978A81828313828B8184834F
:1011F00015828C81868317828D81808711868E81EE
:10120000828713860E9478A12DB73EB7245F3F4F97
:101210000FB6F8943EBF0FBE2DBF8DE29AE0BE011F
:101220000E94D05980E897E0BE010E943C59DF91AE
:10123000CF91FF90EF9008953F924F925F926F92FF
:101240007F928F929F92AF92BF92CF92DF92EF9256
:10125000FF920F931F93DF93CF93CDB7DEB76097C5
:101260000FB6F894DEBF0FBECDBF3B010E94586E93
:10127000E82FF0E0EE0FFF1FE15AF44E80819181DC
:101280000196918380838091080A9091090A81FDDB
:1012900074988091EF069091F0064424439496FF51
:1012A00044240E94535F7C01DC018C91982F92951D
:1012B0009F709130B1F490E08F709070009751F46E
:1012C0008091731B9091741B01969093741B809373
:1012D000731BFBC186EB98E2B3010E94585600973E
:1012E00051F08091711B9091721B01969093721B2B
:1012F0008093711BEAC18DE29AE00E9482594FC02F
:10130000C8010296B3010E945856009709F444C0E0
:10131000C8010F9660E074E641ED58E098010E9424
:10132000475CF7019181D80114968C911497981716
:1013300031F51A968C911A978F5F1A968C9380913B
:101340006F1B9091701B01969093701B80936F1B85
:1013500084E00E948760F801208530E02817390773
:1013600028F584E00E948760D80118968C9318971E
:10137000F70180818F7019968C931997A6C1D801B7
:101380001A961C9284E00E948760F8018087D7013A
:101390008C918F7081870BC0C8010E94485A082F1A
:1013A000192F0115110509F0ABCF97C1442433243F
:1013B00031C0C8010296B3010E944F56F7018181E6
:1013C0008150D80114968C9380E091E0A0E0B0E0C9
:1013D000F80183879487A587B687128684E00E94E8
:1013E0008760D80118968C931897F70180818F70C9
:1013F00019968C938DE29AE0B8010E94095AC801AF
:101400000F9660E074E641ED58E098010E94475C59
:1014100033243394D70111968C911197F80184836A
:101420008C918F70878384E00E948760D801159625
:101430008C9383E00E948760582EF8018683878111
:101440008F3009F03324D70111968C90F8018481F4
:10145000881A9924AA24BB2486E0880C991CAA1C0B
:10146000BB1C8A95D1F7638574858585968520ECAC
:1014700030E040E050E00E947C9C672F782F892F5D
:101480009927860E971EA81EB91ED8011B968D920D
:101490009D92AD92BC921E978091080A9091090A84
:1014A00081FD08C08091EF0680FD04C081FFF1C07E
:1014B0001D9BEFC0EDB7FEB774970FB6F894FEBF53
:1014C0000FBEEDBFCDB6DEB60894C11CD11C8FE2B5
:1014D00092E092838183C7010296D60113969C9372
:1014E0008E931297F301808114968C93149715961E
:1014F0001C921597818116968C93169717961C92BD
:10150000D70111968C911197F601808711868C91E5
:1015100090E08F70907093878287D80115968C9198
:101520008487158656861786BB27AB2D9A2D892D65
:10153000918B808BC501B40124E630E040E050E09F
:101540000E947C9C672F782F892F99270E94C29C2C
:10155000F601738B628B0E9478A12091D1068DB722
:101560009EB744960FB6F8949EBF0FBE8DBF222340
:10157000A9F000D000D0EDB7FEB7319687EE91E02C
:10158000ADB7BEB712969C938E93119722831382A8
:101590000E948AA10F900F900F900F908091EF06FC
:1015A0009091F00696FF2FC0442069F1F701208149
:1015B000822F90E08F70907082309105DCF0822F46
:1015C0008F708150207F822B808389E19AE00E9476
:1015D000EF5680916D1B90916E1B019690936E1B40
:1015E00080936D1B8091080A9091090A96FF0BC0A9
:1015F000739809C08091731B9091741B019690930E
:10160000741B8093731B8091332086FF42C00E941D
:101610003965C70105960E94F8648DB79EB70C978F
:101620000FB6F8949EBF0FBE8DBFEDB7FEB73196D3
:101630006E010894C11CD11CADB7BEB71296DC92E6
:10164000CE92119780E190E09383828383E792E0CA
:1016500095838483D80115968C911597868317827C
:1016600016968C9180871186D70111968C9182876E
:1016700013860E94E1A1EDB7FEB73C960FB6F89431
:10168000FEBF0FBEEDBF82E00E941565C6010E943D
:10169000F8643320D1F082E080934A2481E090E026
:1016A000A0E0B0E280934B2490934C24A0934D246F
:1016B000B0934E241093502400934F2483E397E07B
:1016C00062E14AE454E20E948B588091080A9091AA
:1016D000090A81FF0DC0749A0BC080E897E00E9450
:1016E0001659082F192F0115110509F062CEEDCFFB
:1016F00060960FB6F894DEBF0FBECDBFCF91DF91DD
:101700001F910F91FF90EF90DF90CF90BF90AF901F
:101710009F908F907F906F905F904F903F90089533
:10172000CF93DF93EB01009791F000D000D089E1D7
:101730009DE0EDB7FEB79283818386E892E09483C3
:1017400083830E948AA10F900F900F900F9000D07A
:1017500000D086E19DE0EDB7FEB792838183D4830C
:10176000C3830E948AA10F900F900F900F90DF917A
:10177000CF91089587EE93E08115910511F00197BF
:10178000F1F708958823B9F052985A981DBA8091BC
:101790006900806280936900EA9A53985B98EB9A9B
:1017A0008091690080688093690080916800816001
:1017B000809368000895109269005A9AEA985B9A9B
:1017C000EB9808951F920F920FB60F9211248F93EA
:1017D0009F93AF93BF938091680080FF20C080915A
:1017E000912890919228A0919328B09194280196E5
:1017F000A11DB11D8093912890939228A0939328C6
:10180000B09394288091080A9091090A87FF07C035
:10181000749882E090E09093C4068093C306BF91D1
:10182000AF919F918F910F900FBE0F901F901895C1
:101830001F920F920FB60F9211248F939F93AF9325
:10184000BF938091680080FF20C08091952890917F
:101850009628A0919728B09198280196A11DB11DB6
:101860008093952890939628A0939728B0939828D2
:101870008091080A9091090A90FF07C0739882E04E
:1018800090E09093C4068093C306BF91AF919F915F
:101890008F910F900FBE0F901F90189580937C0032
:1018A00080917B00877F80937B0080917C00806C9F
:1018B00080937C0085E080937A0080917A00806834
:1018C00080937A0080917B0087FFFCCF80917B0022
:1018D00085FFFCCF80917A00806480937A008091AC
:1018E0007A0086FDFCCF109279001092780084E097
:1018F00090E060E070E020917A00206420937A000C
:1019000020917A0026FDFCCF20917800309179005B
:10191000620F731F019779F710927C0080917A0013
:101920008F7780937A00769567957695679580E0B6
:1019300090E00E94DC99089580E00E944E0C209176
:10194000C5063091C6064091C7065091C8060E9450
:10195000BC9B21EE3AE744E95EE30E944498089577
:1019600080E180935101809351019091510195FF45
:1019700003C08F5F8F31B9F76BE4869FB0011124EC
:10198000882777FD8095982F0E94DE9920E030E629
:101990004FE954E40E94449820E030E04AE754E4E0
:1019A0000E940E99089565FF4BC080917B0088606E
:1019B00080937B0089EC80937C0085E080937A00A3
:1019C00080917A00806880937A0080917B0087FF05
:1019D000FCCF80917B0085FFFCCF80917A008064F2
:1019E00080937A0080917A0086FDFCCF80917A0006
:1019F000806480937A0080917A0086FDFCCF6091AC
:101A000078007091790080E090E00E94DC9927EDE9
:101A100033EA40E95FE30E94BC9B26E636E648E8ED
:101A200053E40E9443986093621B7093631B8093FE
:101A3000641B9093651B80917A008F7780937A0066
:101A400008956F927F928F929F92AF92BF92CF92A2
:101A5000DF92EF92FF920F931F93DF93CF93CDB757
:101A6000DEB72A970FB6F894DEBF0FBECDBF3C019C
:101A70001092100A8FEF898366EAC62E6BE1D62E8C
:101A800000E010E052E0E52EF12CEC0EFD1E4E01C0
:101A90000894811C911C4AE0A42EB12CAC0EBD1EF2
:101AA0003FC00830110509F441C0C401B7012A87BD
:101AB0000E94456289812A858F3F11F08E3F19F47B
:101AC0008093100A34C06114710479F4C7010E9434
:101AD0005F628093AE28F701A6EAB8E281918D9308
:101AE000EA15FB05D9F721E022C0C7010E945F6219
:101AF000F6018083D701F80133E0EE0FFF1F3A951E
:101B0000E1F7E00FF11FE256F44E8D918193AA1593
:101B1000BB05D9F70F5F1F4F89E090E0C80ED91EB3
:101B2000202F8981882309F0BCCF01C028E0822FB3
:101B30002A960FB6F894DEBF0FBECDBFCF91DF91CE
:101B40001F910F91FF90EF90DF90CF90BF90AF90DB
:101B50009F908F907F906F90089500D08BE69DE0CE
:101B6000EDB7FEB7928381830E948AA10F900F90F8
:101B700008952F923F924F925F926F927F928F9231
:101B80009F92AF92BF92CF92DF92EF92FF920F930C
:101B90001F93DF93CF9300D000D0CDB7DEB78C0179
:101BA0004B01009741F489E290E06BE270E04AE279
:101BB00050E027E00AC08130910549F489E290E0C5
:101BC0006BE270E04AE250E026E00E942161C80129
:101BD0000E94210DF801E25FF54F80830115110588
:101BE00081F0B6EACB2EBBE1DB2E00E010E03F0136
:101BF000A8E24A2EADE05A2EF0E22F2EFDE03F2E55
:101C000044C186EA98E20E9491639C01B901882749
:101C100077FD8095982F0E94DE99C82EE92E8114B9
:101C20009104A1F000D000D000D00DB71EB70F5F17
:101C30001F4F89E59DE0ADB7BEB712969C938E937A
:101C40001197562F472F3C2D2E2D97C0E6EAAE2E2A
:101C5000E8E2BE2E04E51DE0D5018D915D0100D0C6
:101C600000D0EDB7FEB73196ADB7BEB712961C9354
:101C70000E931197828313826B837C830E948AA1C7
:101C80000F900F900F900F906B817C81BEEAAB1686
:101C9000B8E2BB0609F700D000D000D00DB71EB7E0
:101CA0000F5F1F4F84E49DE0EDB7FEB79283818301
:101CB0008C2D9E2D20E030E048EC52E40E940E99DD
:101CC000D80112966D937D938D939C9315970E94E6
:101CD0008AA1EDB7FEB736960FB6F894FEBF0FBED9
:101CE000EDBF8091AE28882319F088E892E002C009
:101CF00081E992E000D000D020E43DE0ADB7BEB76E
:101D000012963C932E93119714969C938E9313974F
:101D10000E948AA10F900F900F900F9048C07801F9
:101D200073E0EE0CFF1C7A95E1F7E00EF11EEEE990
:101D3000FBE1EE0EFF1EC7010E9491639C01B901F9
:101D4000882777FD8095982F0E94DE995C01811489
:101D5000910481F100D000D000D00DB71EB70F5F05
:101D60001F4F8DE29DE0ADB7BEB712969C938E9348
:101D70001197562F472F3A2D2B2D652F742F832F18
:101D8000922F20E030E048EC52E40E940E99F801D6
:101D900062837383848395830E948AA12DB73EB7A3
:101DA0002A5F3F4F0FB6F8943EBF0FBE2DBF0E9473
:101DB000AD0D72C020E030E0D7018D917D0100D0E3
:101DC00000D0EDB7FEB73196ADB7BEB712965C92B4
:101DD0004E9211978283138229833A836B837C838B
:101DE0000E948AA129813A812F5F3F4F0F900F9067
:101DF0000F900F906B817C8128303105E9F600D07F
:101E000000D000D0EDB6FEB60894E11CF11CEDB791
:101E1000FEB7328221828A2D9B2D20E030E048ECF3
:101E200052E40E940E99D70112966D937D938D9383
:101E30009C9315970E948AA1EDB7FEB736960FB610
:101E4000F894FEBF0FBEEDBFD6018C91882319F028
:101E500088E892E002C081E992E000D000D02CE155
:101E60003DE0EDB7FEB732832183948383830E94E4
:101E70008AA10F900F900F900F900E94AD0D0F5FF1
:101E80001F4F89E090E0C80ED91ED3018C9190E0DD
:101E9000081719070CF443CF0F900F900F900F9075
:101EA000CF91DF911F910F91FF90EF90DF90CF9036
:101EB000BF90AF909F908F907F906F905F904F906A
:101EC0003F902F900895DF93CF9300D0CDB7DEB72A
:101ED0008091A72889838091AD288A83CE010196BD
:101EE0000E946A560F900F90CF91DF910895CF9383
:101EF000DF93EC018091A6288F3FB1F58091A72850
:101F00008F3F91F58091A8288F3F71F58091A92886
:101F10008F3F51F58091AA288F3F31F58091AB28F2
:101F20008F3F11F58091AC288F3FF1F48091AD285F
:101F30008F3FD1F489E290E06BE270E04AE250E03A
:101F400027E00E94216180E090E00E94210DC25FA5
:101F5000D54F888386EA98E269E170E049E050E075
:101F60000E94D3A20E94630FDF91CF9108951F9228
:101F70000F920FB60F920BB60F9211241F932F934F
:101F80003F934F935F936F937F938F939F93AF9301
:101F9000BF93EF93FF938091B12882608093B12823
:101FA0008091EF0686FD2B9A8091EF0687FD2B9A94
:101FB0008091C3069091C4061816190614F4749AF9
:101FC000739A8091080A9091090A85FF02C074985B
:101FD000739880918A0790918B07019790938B0754
:101FE00080938A07009709F095C08091480A9091E4
:101FF000490A01969093490A8093480A2091352412
:102000003091362440913724509138242F5F3F4F30
:102010004F4F5F4F2093352430933624409337241D
:102020005093382420E130E030938B0720938A07C7
:102030002091EF0620FD02C01D9B05C010920C0AE6
:1020400010920B0A06C021E030E030930C0A209376
:102050000B0A6091ED067091EE066115710599F01D
:1020600001960E949B9C009771F477988091080AD2
:102070009091090A92FF07C0749884E090E09093D1
:10208000C4068093C3066091ED067091EE0661155B
:10209000710531F18091480A9091490A0E949B9CF8
:1020A0000097F1F481E080934A248091E9069091B1
:1020B000EA06A091EB06B091EC0680934B24909336
:1020C0004C24A0934D24B0934E241092502410928F
:1020D0004F2483E397E062E14AE454E20E948B5884
:1020E0008091EF0686FD2B988091EF069091F00687
:1020F00091FF10C00E94586E8A3119F0182F1F5F8F
:1021000001C01BE00E949C6C812F90E00E94706EC9
:102110000E943A6D84EA97E060E040E050E00E945F
:102120008B58FF91EF91BF91AF919F918F917F91CC
:102130006F915F914F913F912F911F910F900BBE27
:102140000F900FBE0F901F9018958091951B909146
:102150004924891B08950E94A510882379F0E091F5
:102160004924F0E0EF71F070E651F44E208130E048
:10217000809149248F5F8093492402C02FEF3FEF65
:10218000C9010895CF93DF93EC011092300A1092A9
:102190002F0A88819981009731F023E08F329207CE
:1021A00009F0B9C009C00E94A510882341F48FE24C
:1021B00093E099838883B3C0613109F0B0C0F8948B
:1021C00078940E94AB1090E09093340A8093330A85
:1021D0008D3009F47CC08F3F31F38231910569F174
:1021E0008F37910521F08830910509F053C0809117
:1021F000370A9091380A181619060CF060C06091E1
:1022000071317091723188E090E00E944CA1609130
:1022100071317091723180E290E00E944CA1609126
:1022200071317091723188E090E00E944CA18091F0
:10223000370A9091380A01973EC0609171317091D0
:1022400072318DE090E00E944CA11092360A1092FB
:10225000350A14C08F5A9B4DFC0180816091713109
:102260007091723190E00E944CA18091350A90915A
:10227000360A01969093360A8093350A8091350A82
:102280009091360A2091370A3091380A82179307C5
:102290000CF315C060917131709172310E944CA1A4
:1022A0008091370A9091380A2091330AFC01EF5A45
:1022B000FB4D208301969093380A8093370A8091D2
:1022C000370A9091380A8F33910509F06CCF10923C
:1022D0004924809149248093951B8091370A9091DD
:1022E000380AFC01EF5AFB4D10829093300A80931C
:1022F0002F0A1092380A1092370A8091AF289091D5
:10230000B028009709F44FCF6091310A40E050E0C7
:102310000E948B5848CF1982188283E001C081E067
:10232000DF91CF910895789480910B0A90910C0AD7
:102330000097C9F08091EF069091F00693FD13C0CD
:1023400092FF03C083B7817F03C083B7817F86601C
:1023500083BFF89483B7816083BF7894889583B7EF
:102360008E7F83BF78940895CF93DF93EC018881AB
:102370009981009721F02EE08137920799F40E940D
:102380008A6B0E94931180914E1290914F1265E8D2
:1023900040E050E00E948B5881E79EE0998388835B
:1023A00081E003C01982188283E0DF91CF91089504
:1023B000CF93DF93EB01009781F000D000D089E14B
:1023C0009DE0EDB7FEB792838183548343830E94DF
:1023D0008AA10F900F900F900F9000D000D086E14F
:1023E0009DE0EDB7FEB792838183D483C3830E94BF
:1023F0008AA10F900F900F900F90DF91CF910895C9
:10240000EF92FF920F931F93CF93DF930E948A6BFB
:1024100080EB0E9411648823A1F40E94776480916C
:102420003320909134208160909334208093332026
:1024300080E090E062E972E00E94900B01E010E021
:1024400002C000E010E0EEB0FF2484E0E822FF24A8
:10245000729A0E948A6B8EE40E941164882399F418
:102460000E94776480913320909134208260909311
:10247000342080933320E8012196C8016AE972E094
:102480000E94900B8E01E114F10409F472980E94ED
:102490008A6B8EEE0E941164882399F40E947764FF
:1024A00080913320909134208460909334208093E5
:1024B0003320E8012196C80162EA72E00E94900B85
:1024C0008E010E948A6B86EA0E941164882399F427
:1024D0000E9477648091332090913420886090939B
:1024E000342080933320E8012196C80169EA72E024
:1024F0000E94900B8E010E948A6B8CE30E941164F3
:102500008823F1F40E9477648091332090913420E5
:1025100080619093342080933320E8012196C80194
:1025200061EB72E00E94900B00D08EE09DE0EDB771
:10253000FEB7928381830E948AA10F900F908E0133
:102540000E948A6B82ED0E941164882399F40E9494
:10255000776480913320909134208062909334206E
:1025600080933320E8012196C80169EB72E00E9454
:10257000900B8E010E948A6B80E80E941164882370
:1025800099F40E9477648091332090913420916077
:102590009093342080933320E8012196C80162ECA7
:1025A00072E00E94900B8E010E948A6B80ED0E9467
:1025B0001164882399F40E9477648091332090916C
:1025C000342080689093342080933320E801219652
:1025D000C80168EC72E00E94900B8E010E948A6B29
:1025E0008CEE0E941164882399F40E947764809194
:1025F0003320909134209260909334208093332044
:10260000E8012196C80160ED72E00E94900B8E01F6
:10261000C7E0D0E00E948A6B8CE70E941164882397
:1026200089F40E94776480913320909134208064F3
:102630009093342080933320C80167ED72E00E94AC
:10264000900B02C0219731F70E9477640E94AD0D74
:10265000DF91CF911F910F91FF90EF900895DF933D
:10266000CF9300D0CDB7DEB74A8369830E944D6413
:102670006981862F0E947F644A81842F0E947F6433
:102680000E9477640F900F90CF91DF910895AF92E1
:10269000BF92DF92EF92FF920F931F93DF93CF933E
:1026A00000D00F92CDB7DEB7082FD22E4A835B83BE
:1026B00069830E944D646981862F0E947F64802F08
:1026C00081600E9474644A815B81042F152FAA24C3
:1026D000BB24ED2CFF240894E108F1080FC0AE14D0
:1026E000BF0419F40E949A6402C00E949064F80129
:1026F00080830894A11CB11C0F5F1F4FAD1478F3A9
:102700000E9477640F900F900F90CF91DF911F91EF
:102710000F91FF90EF90DF90BF90AF900895AF9230
:10272000BF92CF92DF92EF92FF920F931F93DF93AE
:10273000CF93CDB7DEB760970FB6F894DEBF0FBE6C
:10274000CDBFB82EA42E662309F455C0AE014F5F4D
:102750005F4F80E1DA011D928A95E9F780EB68E925
:1027600028E00E944713BB2059F000D080EE92E091
:10277000EDB7FEB7928381830E9478A10F900F90EE
:102780008E010F5F1F4F38E0E32EF12CEC0EFD1E83
:1027900027EEC22E22E0D22ED8018D918D0100D0DD
:1027A00000D0EDB7FEB73196ADB7BEB71296DC924A
:1027B000CE921197828313820E9478A10F900F907E
:1027C0000F900F900E151F0539F700D000D0EDB710
:1027D000FEB731968CEE92E0ADB7BEB712969C93E1
:1027E0008E9311978885828313820E9478A10F901F
:1027F0000F900F900F90AA2009F457C0AE014F5FC1
:102800005F4F80E1FA0111928A95E9F780EB60E869
:1028100028E00E944713BB2069F000D082EF92E0CD
:10282000ADB7BEB712969C938E9311970E9478A174
:102830000F900F908E010F5F1F4F90E1E92EF12C4A
:10284000EC0EFD1E87EEC82E82E0D82EF801819195
:102850008F0100D000D0EDB7FEB73196ADB7BEB74F
:102860001296DC92CE921197828313820E9478A1F5
:102870000F900F900F900F900E151F0539F700D095
:1028800000D0EDB7FEB731968CEE92E0ADB7BEB793
:1028900012969C938E9311978885828313820E944F
:1028A00078A10F900F900F900F9060960FB6F8944C
:1028B000DEBF0FBECDBFCF91DF911F910F91FF9073
:1028C000EF90DF90CF90BF90AF9008950F931F933C
:1028D000DF93CF9300D0CDB7DEB71A8219828EEE88
:1028E0006AEA8E010F5F1F4FA80122E00E94471382
:1028F000398120E08A8190E0822B932B90930B1CEE
:1029000080930A1C8EEE6CEAA80122E00E94471315
:10291000398120E08A8190E0822B932B90930D1CCB
:1029200080930C1C8EEE6EEAA80122E00E944713F1
:10293000398120E08A8190E0822B932B90930F1CA9
:1029400080930E1C8EEE60EBA80122E00E944713DC
:10295000398120E08A8190E0822B932B90931D1C7B
:1029600080931C1C8EEE62EBA80122E00E944713AC
:10297000398120E08A8190E0822B932B90931F1C59
:1029800080931E1C8EEE64EBA80122E00E94471388
:10299000398120E08A8190E0822B932B9093211C37
:1029A0008093201C8EEE66EBA80122E00E94471364
:1029B000398120E08A8190E0822B932B9093111C27
:1029C0008093101C8EEE68EBA80122E00E94471352
:1029D000398120E08A8190E0822B932B9093131C05
:1029E0008093121C8EEE6AEBA80122E00E9447132E
:1029F000398120E08A8190E0822B932B9093171CE1
:102A00008093161C8EEE6CEBA80122E00E94471307
:102A1000398120E08A8190E0822B932B9093191CBE
:102A20008093181C8EEE6EEBA80122E00E944713E3
:102A3000398120E08A8190E0822B932B90931B1C9C
:102A400080931A1C0F900F90CF91DF911F910F91DF
:102A500008952F923F924F925F926F927F928F9242
:102A60009F92AF92BF92CF92DF92EF92FF920F931D
:102A70001F93DF93CF93CDB7DEB76C970FB6F89463
:102A8000DEBF0FBECDBFA82E4A8B2B8FFE01319625
:102A900083E0DF011D928A95E9F780912E1C88233F
:102AA00039F46C8F0E94661481E080932E1C6C8D2B
:102AB000662309F475C08EEE64EF4EE20E942F1378
:102AC00069E07AE180E090E00E94FE638EEE66EFBE
:102AD000AE014F5F5F4F22E00E944713698170E0B3
:102AE00080E090E0982F872F762F66272A8130E0AC
:102AF00040E050E0622B732B842B952B2091201CFF
:102B00003091211C40E050E0621B730B840B950B4D
:102B100020911E1C30911F1C40E050E00E947C9CC4
:102B20007B018C013FE015950795F794E7943A9562
:102B3000D1F76091181C7091191C882777FD80953A
:102B4000982F2BE0660F771F881F991F2A95D1F7C2
:102B500020911A1C30911B1C442737FD4095542F9F
:102B60002E0D3F1D401F511F0E94E49C2E0D3F1D46
:102B70003093151C2093141C285F3F4F14E03595AB
:102B800027951A95E1F779010027F7FC0095102F9A
:102B9000E092221CF092231C0093241C1093251C0D
:102BA000BA2DB295BB0FBB0FB07CBC5CB9872A2D88
:102BB00030E03E8B2D8B63E070E00A2C02C0660F84
:102BC000771F0A94E2F7882777FD8095982F25E3F1
:102BD00035E040E050E00E947C9CDC01CB01029695
:102BE000A11DB11D8A879B87AC87BD8720E533EC8B
:102BF00040E050E004C05595479537952795AA9435
:102C0000D2F72E873F87488B598B18861C821D82EE
:102C10001E821F8248E050E08D899E89481B590B17
:102C20005C8B4B8B69C18EEE64EF49850E942F133C
:102C30006A857B858C859D850E94FE638EEE66EF9E
:102C4000AE014F5F5F4F23E00E9447138091141C39
:102C50009091151C805A9F401C01442437FC4094DD
:102C6000542CC201B101A20191010E947C9C6F8B86
:102C7000788F898F9A8F20910E1C30910F1C4427DA
:102C800037FD4095542FC201B1010E947C9C7B010D
:102C90008C01BDE015950795F794E794BA95D1F7A7
:102CA00022E030E040E050E0E20EF31E041F151F6A
:102CB0006F89788D898D9A8DACE0959587957795FC
:102CC0006795AA95D1F72091101C3091111C4427CB
:102CD00037FD4095542F0E947C9CBC01992777FDBD
:102CE0009095892FE60EF71E081F191FE2E0159533
:102CF0000795F794E794EA95D1F780E090E8A0E093
:102D0000B0E0E80EF91E0A1F1B1F20911C1C309119
:102D10001D1C40E050E0C801B7010E947C9C3B01B3
:102D20004C017FE096948794779467947A95D1F7D5
:102D3000A980BB24CC24DD246501BB24AA248A817C
:102D400090E0A0E0B0E0BA2FA92F982F8827A82AFA
:102D5000B92ACA2ADB2A8B8190E0A0E0B0E0A82A39
:102D6000B92ACA2ADB2A0B8804C0D594C794B79421
:102D7000A7940A94D2F720910C1C30910D1C442783
:102D800037FD4095542FC201B1010E947C9C7B010C
:102D90008C014BE015950795F794E7944A95D1F788
:102DA00080910A1C90910B1CAA2797FDA095BA2F21
:102DB00032E0880F991FAA1FBB1F3A95D1F7E80E82
:102DC000F91E0A1F1B1F2091121C3091131C44274F
:102DD00037FD4095542F6F89788D898D9A8D0E948B
:102DE0007C9C27E195958795779567952A95D1F7EE
:102DF000E60EF71E081F191F0D8804C0EE0CFF1CFD
:102E0000001F111F0A94D2F722E030E040E050E0AA
:102E1000E20EF31E041F151F82E015950795F79427
:102E2000E7948A95D1F7AE18BF08C00AD10AC60147
:102E3000B5012E853F85488959890E947C9C97FD64
:102E40000BC0660F771F881F991FA40193010E9472
:102E5000C29C79018A010AC0A40193010E94C29C0C
:102E600079018A01EE0CFF1C001F111F552717FD69
:102E70005A95412F302F2F2DCA01B9010E947C9CF9
:102E80002EED3BE040E050E00E947C9C5B016C0139
:102E9000C801B70123E433EE4FEF5FEF0E947C9C43
:102EA000BC01992777FD9095892F6153714F8F4F02
:102EB0009F4F5601DD24B7FCD094CD2C6A0D7B1DAD
:102EC0008C1D9D1D44E095958795779567954A954E
:102ED000D1F76E0D7F1D801F911F2C813D814E818A
:102EE0005F81260F371F481F591F2C833D834E8358
:102EF0005F8338853F5F388748855A89451708F4CE
:102F000092CE552391F0252F30E040E050E06C81C7
:102F10007D818E819F810E94C29C2093261C3093CC
:102F2000271C4093281C5093291C8B8D8823C9F1A2
:102F30006091261C7091271C8091281C9091291C5F
:102F4000611571058105910561F10E94DE9920E806
:102F500036EE45EC57E40E940E9921E03EED42E446
:102F60005EE30E941F9C562F472F382F292F60E0C9
:102F700070E080E89FE3DA01F9012B2F3A2F4F2F01
:102F80005E2F0E9443982BE43AE34DEB57E30E94F7
:102F90000E9960932A1C70932B1C80932C1C909389
:102FA0002D1C6C960FB6F894DEBF0FBECDBFCF912F
:102FB000DF911F910F91FF90EF90DF90CF90BF9026
:102FC000AF909F908F907F906F905F904F903F90C9
:102FD0002F900895DF93CF9300D000D000D0CDB7CD
:102FE000DEB7FE01319686E0DF011D928A95E9F792
:102FF00080916C1B882399F486EA61E340E00E948B
:103000002F1386EA6CE24AE00E942F1381E080933E
:103010006C1B6CE77EE380E090E00E94FE6386EA32
:103020006DE248E00E942F136CE77EE380E090E0C1
:103030000E94FE6386EA62E3AE014F5F5F4F26E0C7
:103040000E94471386EA6DE247E00E942F139A819F
:1030500080E0498150E0482B592B5093671B4093E7
:10306000661B9C8180E02B8130E0282B392B30932C
:10307000691B2093681B7E8160E08D8190E0862B28
:10308000972B90936B1B80936A1B6DB77EB768502C
:1030900070400FB6F8947EBF0FBE6DBFEDB7FEB7A0
:1030A000319666EF72E0ADB7BEB712967C936E9321
:1030B00011975383428335832483978386830E94A9
:1030C00078A16DB77EB7685F7F4F0FB6F8947EBF6B
:1030D0000FBE6DBF26960FB6F894DEBF0FBECDBFF4
:1030E000CF91DF9108958F929F92AF92BF92CF922E
:1030F000DF92EF92FF920F931F93DF93CF9300D055
:1031000000D000D0CDB7DEB78E010F5F1F4F86E035
:10311000F80111928A95E9F78CE362E041E00E94A0
:103120002F138CE360E048E50E942F1362E174E303
:1031300080E090E00E94FE638CE363E0A80126E05B
:103140000E9447138CE362E043E00E942F139981B1
:1031500080E00A8110E0082B192B1093431B009389
:10316000421B9B8180E0EC80FF24E82AF92AF09240
:10317000451BE092441B9D8180E0CE80DD24C82A5F
:10318000D92AD092471BC092461BB701882777FDEA
:103190008095982F0E94DE994B015C01B801882729
:1031A00077FD8095982F0E94DE999B01AC01C501A7
:1031B000B4010E94B7982DB73EB72C5030400FB6DF
:1031C000F8943EBF0FBE2DBFADB6BEB60894A11C8D
:1031D000B11C24E033E0EDB7FEB732832183F50163
:1031E00013830283F582E482D782C68220EE3EE218
:1031F00045E652E40E94BC9B20E030E044E353E407
:103200000E944498F50160877187828793870E94A6
:1032100078A12DB73EB7245F3F4F0FB6F8943EBF5D
:103220000FBE2DBF26960FB6F894DEBF0FBECDBFE2
:10323000CF91DF911F910F91FF90EF90DF90CF9092
:10324000BF90AF909F908F900895CF93DF93EC0144
:1032500088819981009731F02EE08A35920709F034
:1032600071C00BC081E19AE060E870E00E94415BB0
:103270008AE59EE09983888369C081E19AE00E9493
:103280006C5B009709F462C08091080A9091090A6A
:1032900093FF3FC08091332082FF3BC083E061E019
:1032A00048E021E00E9429158DB79EB70A970FB616
:1032B000F8949EBF0FBE8DBFEDB7FEB731968FEC71
:1032C00091E0ADB7BEB712969C938E931197809103
:1032D000261C9091271CA091281CB091291C828348
:1032E0009383A483B58380912A1C90912B1CA09179
:1032F0002C1CB0912D1C86839783A087B1870E94D8
:103300008AA18DB79EB70A960FB6F8949EBF0FBEDE
:103310008DBF8091080A9091090A94FF06C08091A0
:10332000332083FF02C00E94EA178091080A90911F
:10333000090A95FF97CF8091332084FF93CF0E9495
:10334000731890CF1982188283E001C081E0DF9169
:10335000CF9108951F93182F8CEE0E947464812FD3
:103360000E947F6465E375E080E090E00E94FE6368
:103370008DEE0E9474640E949064182F0E949A64DB
:10338000512F40E0282F30E0242B352BC9011F910D
:103390000895EF92FF920F931F93182F8CEE0E94C7
:1033A0007464812F0E947F6462E174E380E090E0A6
:1033B0000E94FE638CEE0E94746480E00E947F6431
:1033C00065E375E080E090E00E94FE638DEE0E9470
:1033D00074640E949064182F0E949064E82E0E94EA
:1033E0009A64212F30E040E050E0A90133272227E2
:1033F000FF2400E010E0102F0F2DFE2CEE242E29CC
:103400003F29402B512B90E0A0E0B0E0282B392B36
:103410004A2B5B2BB901CA011F910F91FF90EF90CE
:1034200008952F923F924F925F926F927F928F9268
:103430009F92AF92BF92CF92DF92EF92FF920F9343
:103440001F93DF93CF93CDB7DEB7C654D0400FB6EE
:10345000F894DEBF0FBECDBF809188079091890799
:103460000097D1F110928907109288078CEE0E9484
:1034700074648EE10E947F646BE17EE480E090E002
:103480000E94FE6382EA0E94AA199093470A8093E1
:10349000460A84EA0E94AA199093450A8093440A36
:1034A00086EA0E94AA199093430A8093420A88EA06
:1034B0000E94AA199093410A8093400A8AEA0E94C6
:1034C000AA1990933F0A80933E0A8CEA0E94AA1997
:1034D00090933D0A80933C0A88E40E94C91969AB25
:1034E0007AAB8BAB9CAB88E50E94C9191B012C0100
:1034F00066247724430140913E0A50913F0A9A0185
:1035000040E050E060E070E080E090E0AA24BB245E
:10351000BA94CC24CA94DD24DA94EE24EA94FF24ED
:10352000FA940FEF1FEF0E94D78A220D2887E1E05F
:10353000221508F0E0E0330D21E0331508F020E01B
:10354000E30FEA87E1E0EA84E31608F0E0E02E2BDF
:10355000440D31E0441508F030E0240F2B8721E0C2
:10356000FB84F41608F020E0322B550D21E05515B0
:1035700008F020E0350F3C8731E00C85051708F096
:1035800030E0232B31E0661508F030E0260F2D8760
:1035900021E01D85161708F020E0322B21E0771579
:1035A00008F020E0370F3E8731E04E85471708F0DE
:1035B00030E0232B31E0881508F030E0280F2F870A
:1035C00021E05F85581708F020E0322B390F388B47
:1035D0002A85215031E06A85261708F030E09B8566
:1035E000915041E07B85971708F040E0390F81E06A
:1035F000391708F080E0842B9C85890F91E0AC8519
:103600008A1708F090E0BD859B0F41E09B1708F0FA
:1036100040E0EE854E0F51E04E1708F050E0FF8578
:103620005F0F61E05F1708F060E0E8886E0D01E071
:1036300010E027961FAF0EAF27976623A9F45523F6
:1036400099F4442389F4992379F4823068F4813021
:1036500039F43F3F29F42F3F19F41885112321F441
:1036600027961FAE1EAE279720903C0A30903D0A49
:1036700028853A854B855C856D857E858F85988903
:103680005101CC24DD24EE24FF2400E010E00E9450
:10369000D78AF901DA01162F072FF82EE92EE7FE57
:1036A00032C0215031E02E1708F030E08F2F8150CA
:1036B00041E08F1708F040E0380F91E0381708F02C
:1036C00090E0492B8A2F815851E08A1708F050E08A
:1036D000480F91E0481708F090E0592B5B0F61E02C
:1036E0005B1708F060E0610F71E0611708F070E0AF
:1036F000700F81E0701708F080E08F0D91E08F155A
:1037000008F090E09E0D07E10E94128C2C8B3D8BFF
:103710004E8B5F8B688F7DA38EA398AB20532F8336
:1037200091E03C89231708F090E08D89895F21E0C2
:103730004D89841708F020E0980F9A8391E05A8110
:10374000581708F090E0292B6E89260F298381E015
:10375000261708F080E07F89780F7B8381E09F89BE
:10376000791708F080E0A88DA80FAC8381E0B88DB0
:10377000AB1708F080E0EDA1E80FED8381E0FDA13B
:10378000EF1708F080E0EEA0E80EEE8281E0FEA0E8
:10379000EF1408F080E008A9080F09872F81205650
:1037A00091E01F81211708F090E03A81315F41E0FC
:1037B0005A81351708F040E0930F81E0931708F025
:1037C00080E0842B6981860F31E0861708F030E0B5
:1037D0007B81370F41E0371708F040E0AC814A0F9A
:1037E00051E04A1708F050E0BD815B0F61E05B17C4
:1037F00008F060E0EE816E0F71E06E1708F070E087
:10380000F9857F0F81F4662371F4552361F4442315
:1038100051F4332341F4882331F4913320F490336D
:1038200061F4253D50F027960EAD1FAD27970F5F31
:103830001F4F27961FAF0EAF27972090400A30905A
:10384000410A28853A854B855C856D857E858F8507
:1038500098895101CC24DD24EE24FF2400E010E0FF
:103860000E94D78AF901DA01162F072FF82EE92EC8
:10387000E7FE24C0215831E02E1708F030E03F0F5A
:1038800041E03F1708F040E04A0F51E04A1708F0C6
:1038900050E05B0F61E05B1708F060E0610F71E0E2
:1038A000611708F070E0700F81E0701708F080E099
:1038B0008F0D91E08F1508F090E09E0D07E00E94BB
:1038C000128C122FF32EE42ED52EC62EB72EA82E34
:1038D000992E4091440A5091450A9A0140E050E0E7
:1038E00060E070E080E090E000E10E94A18B210F99
:1038F000298B21E0A989A11708F020E03F0DE1E024
:103900003F1508F0E0E0230F298F21E0B98DB317B0
:1039100008F020E0E22B4E0D21E04E1508F020E0EB
:10392000E40FEA8F31E0E41708F030E0232B5D0D5F
:1039300031E05D1508F030E0250F2B8F21E0EB8D95
:10394000E51708F020E0322B6C0D21E06C1508F033
:1039500020E0360F3C8F31E0FC8DF61708F030E0A8
:10396000232B7B0D31E07B1508F030E0270F2D8FE6
:1039700021E0ED8CE71608F020E0322B8A0D21E0E3
:103980008A1508F020E0380F3E8F31E0FE8CF816E3
:1039900008F030E0232B990D290F2FA3098909A7DF
:1039A000198D1AA72A8D2BA73B8D3CA74C8D4DA7AF
:1039B0005D8D5EA76E8D6FA77FA17B8B402F4E5FC5
:1039C00051E0401708F050E0998D590F91E0A98D12
:1039D0005A1708F090E08A8D845061E0BA8D8B17F9
:1039E00008F060E0980F21E0981708F020E0622BC3
:1039F0008B8D815021E0EB8D8E1708F020E0680F51
:103A000031E0681708F030E0232B3C8D3F5F71E018
:103A1000FC8D3F1708F070E0230F81E0231708F0BA
:103A200080E0872BED8C8E0D31E08E1508F030E0B4
:103A3000FE8C3F0D71E03F1508F070E00FA1700F94
:103A400091F4332381F4882371F4253060F4243019
:103A5000A1F46F3F91F49A3F30F4993F71F45523EC
:103A600011F4433050F027962EAD3FAD27972F5FCE
:103A70003F4F27963FAF2EAF27972090420A3090B6
:103A8000430A28853A854B855C856D857E858F85C3
:103A900098895101CC24DD24EE24FF2400E010E0BD
:103AA0000E94D78AF901DA01162F072FF82EE92E86
:103AB000E7FE24C0215031E02E1708F030E03F0F20
:103AC00041E03F1708F040E04A0F51E04A1708F084
:103AD00050E05B0F61E05B1708F060E0610F71E0A0
:103AE000611708F070E0700F81E0701708F080E057
:103AF0008F0D91E08F1508F090E09E0D08E00E9478
:103B0000128C122FF32EE42ED52EC62EB72EA82EF1
:103B1000992E4091460A5091470A9A0140E050E0A0
:103B200060E070E080E090E00FE00E94A18B210F48
:103B30002A8B21E0AA89A11708F020E03F0DE1E0DF
:103B40003F1508F0E0E0230F2F8F21E0BF8DB31762
:103B500008F020E0E22B4E0D21E04E1508F020E0A9
:103B6000E40FE8A331E0E41708F030E0232B5D0D0B
:103B700031E05D1508F030E0250F29A321E0E9A12F
:103B8000E51708F020E0322B6C0D21E06C1508F0F1
:103B900020E0360F3AA331E0FAA1F61708F030E042
:103BA000232B7B0D31E07B1508F030E0270F2BA392
:103BB00021E0EBA0E71608F020E0322B8A0D21E08F
:103BC0008A1508F020E0380F3CA331E0FCA0F8167D
:103BD00008F030E0232B990D290F28A72A893F8D63
:103BE00048A159A16AA17BA18CA198A5C22EC3941A
:103BF000E1E0C21608F0E0E01F8DE10FF1E0E1170F
:103C000008F0F0E0F8A0AEEFFA0E01E0B8A1FB1664
:103C100008F000E0FF0D11E0FF1508F010E0012BA7
:103C200019A11150FF24F394E9A01E1508F0FF24F8
:103C3000B02EB10E01E0B11608F000E0F02A1AA192
:103C40001150DD24D3940AA1101708F0DD24AF2C05
:103C5000A10E01E0A11608F000E0D02A1BA111502E
:103C600001E0ABA11A1708F000E0D10EFF24F39495
:103C7000D11608F0FF240F291CA11150EE24E39463
:103C8000BCA11B1708F0EE24F02EF10E01E0F11696
:103C900008F000E00E2918A51150010FC9F4FF200B
:103CA000B9F4DD20A9F40A2D023090F40130C9F4F2
:103CB0001B2D103868F41F37A1F4FD3F48F4FC3F7A
:103CC00081F4E13828F4E03861F4AC2DA23048F0FA
:103CD0002796EEADFFAD279731962796FFAFEEAF53
:103CE0002797F9851F160CF4C8C5FF23F1F4EE8061
:103CF000EE2009F0C2C5FD80FF2009F0BEC50C8191
:103D0000002309F0BAC51B81112309F0B6C5A981AA
:103D1000AA2309F0B2C5BA81B83008F0AEC5B730F1
:103D200021F4EF81E03D08F0A8C528853A854B8550
:103D30005C856D857E858F85988959016A017B0137
:103D40008C010E94D78AAA24BB24CC24A0E8DA2EB6
:103D5000EE24FF2400E010E00E94C68C2DAB3EABA9
:103D60004FAB58AF69AF7AAF8BAF9CAF2F813A8121
:103D700049815B816C817D818E81998502E00E9401
:103D8000A18B0F81020FE1E0021708F0E0E02A8129
:103D9000230F11E0231708F010E03E2F320FE1E06F
:103DA000321708F0E0E01E2B2981240FB1E0241720
:103DB00008F0B0E0120F41E0121708F040E0B42B19
:103DC0002B81250FA1E0251708F0A0E0FB2EF20EB5
:103DD00041E0F21608F040E0A42B2C81260F51E0C0
:103DE000261708F050E0EA2EE20E41E0E21608F055
:103DF00040E0542B2D81270FF1E0271708F0F0E069
:103E0000E52FE20F41E0E21708F040E0F42B4E818D
:103E1000480F21E0481708F020E0F40F81E0F41784
:103E200008F080E0282B4985940F920F202F205115
:103E300051E0201708F050E0832F885241E08317AB
:103E400008F040E0352F380F51E0381708F050E007
:103E5000452B812F815051E0811708F050E0480F29
:103E600061E0481708F060E0562B8F2D815061E02B
:103E70008F1508F060E0580F71E0581708F070E0F7
:103E8000672B8E2D815071E08E1508F070E0680F61
:103E9000A1E0681708F0A0E07A2BAE2FA15081E0D6
:103EA000AE1708F080E07A0FE1E07A1708F0E0E062
:103EB0008E2BAF2FA150E1E0AF1708F0E0E08A0FA2
:103EC000F1E08A1708F0F0E0EF2B91509E0FAC88DC
:103ED000BD88CE88DF88E88CFDA00EA118A90E94BD
:103EE000D78A122F232EF42EE52ED62EC72EB82ECB
:103EF000A92EA7FE24C02F5F31E0211708F030E083
:103F0000320D41E0321508F040E04F0D51E04F1501
:103F100008F050E05E0D61E05E1508F060E06D0DA8
:103F200071E06D1508F070E07C0D81E07C1508F003
:103F300080E08B0D91E08B1508F090E09A0D01E088
:103F40000E94128C422E3A874B875C876D877E8752
:103F50008F879FA72EA339A74AA75BA76CA77DA72A
:103F60008EA79887212F322D4F2D5E2D6D2D7C2D04
:103F70008B2D9A2DA7FE24C02D5F31E0211708F06C
:103F800030E0320D41E0321508F040E04F0D51E0D5
:103F90004F1508F050E05E0D61E05E1508F060E03E
:103FA0006D0D71E06D1508F070E07C0D81E07C1501
:103FB00008F080E08B0D91E08B1508F090E09A0DF1
:103FC00002E00E94128C288B3B8B4C8B5D8B6E8B9E
:103FD0007F8B888F98ABF82FE92F89858F3F5CF115
:103FE0008F3F09F0BEC29E819F3F28F19F3F09F09D
:103FF000B8C2AD81AF3FF8F0AF3F09F0B2C2BC81AB
:10400000BF3FC8F0BF3F09F0ACC20B810F3F98F033
:104010000F3F09F0A6C219811F3F68F01F3F09F04A
:10402000A0C28A818A3F38F08A3F09F09AC29F81F4
:10403000943208F096C23F80ACED3A0E91E0BF8119
:104040003B1608F090E08A818B5F21E0EA818E17B1
:1040500008F020E0992E980E91E0981608F090E074
:10406000222E292AF9812F0E81E02F1608F080E0F8
:104070008B80880E81E0EB808E1408F080E07C80DD
:10408000780E81E0FC807F1408F080E06D80680E7F
:1040900081E00D81601608F080E05E80580E81E0BE
:1040A0001E81511608F080E02985280F2DA32F814D
:1040B0003A8149815B816C817D818E81998503E0A4
:1040C0000E94A18B022FAF810A1BF1E0201708F09C
:1040D000F0E0232FBA812B1BE1E0321708F0E0E07B
:1040E000322F3F1BF1E0231708F0F0E0EF2BF42F05
:1040F000E980FE1921E04F1708F020E01F2F1E1B5A
:1041000041E0F11708F040E0242BE52FFB80EF1988
:1041100041E05E1708F040E0BE2FB21B21E0EB1734
:1041200008F020E0422B562F2C81521B21E065170E
:1041300008F020E0A52FA41B41E05A1708F040E04A
:10414000242B572F4D81541B41E0751708F040E098
:10415000F52EF21A21E05F1508F020E0422B582FCF
:104160006E81561B21E0851708F020E0E52EE41A49
:1041700081E05E1508F080E0282B7985971B921B63
:10418000202F2C5F51E0201708F050E0832F875D2F
:1041900041E0831708F040E0352F380F51E0381721
:1041A00008F050E0452B410F51E0411708F050E076
:1041B0005B0F61E05B1708F060E06A0F71E06A175F
:1041C00008F070E07F0D81E07F1508F080E08E0D33
:1041D000E1E08E1508F0E0E09E0FA32CB92CC22C74
:1041E000D82CE72CF62C052D1DA10E94D78A240D72
:1041F000F1E0241508F0F0E0AA853A0FE1E03A1763
:1042000008F0E0E0F30FA1E0F31708F0A0E0EA2BDC
:10421000BB854B0F31E04B1708F030E0E40FA1E015
:10422000E41708F0A0E03A2BEC845E0D41E05E1547
:1042300008F040E0350FA1E0351708F0A0E04A2B68
:10424000FD846F0D51E06F1508F050E0142F160F2C
:1042500041E0161708F040E0542B0E85700F41E046
:10426000701708F040E0570F61E0571708F060E062
:10427000462B6F85860F61E07F85871708F060E029
:10428000480F71E0481708F070E0672B8FA5980F72
:104290002EA3F9A7EAA73BA71CA75DA74EA7690F06
:1042A00068872F813A8149815B816C817D818E8114
:1042B000998502E00E94A18B122FF32EE42ED52EB9
:1042C000C62EB72EA82E492E0E94A18BE22FE11BED
:1042D000F1E02E1708F0F0E0A32FAF1921E03A1714
:1042E00008F020E03A2F3F1BF1E0A31708F0F0E0C0
:1042F0002F2BA42FAE19F1E04A1708F0F0E0BA2FE7
:10430000B21B2B2F41E0AB1708F040E0F42B452FF8
:104310004D19A1E0541708F0A0E0542F5F1BF1E005
:10432000451708F0F0E0AF2BB62FBC1941E06B1732
:1043300008F040E00B2F0A1B61E0B01708F060E0C6
:10434000462BA72FAB1961E07A1708F060E0FA2E30
:10435000F41A41E0AF1508F040E0642B782F7A1989
:1043600041E0871708F040E0172F161B81E0711716
:1043700008F080E0482B9419941B4E2FFF814F1BAF
:1043800071E0E41708F070E0632FEA806E1981E0B5
:10439000361708F080E0E62EE71A31E06E1508F0D7
:1043A00030E0832B722F3981731B31E0271708F01F
:1043B00030E0672F681B81E0761708F080E0382B2B
:1043C000252F7B81271B81E0521708F080E0722F98
:1043D000731B31E0271708F030E0832B302FAC81BE
:1043E0003A1B21E0031708F020E0B32FB81B8B2FF6
:1043F00051E03B1708F050E0252B5F2DED815E1B4F
:1044000031E0F51608F030E0E52FE21B21E05E1701
:1044100008F020E0322B512FFE815F1B21E01517A1
:1044200008F020E0F52FF31B31E05F1708F030E0D3
:10443000232BF9849F19921B242F2C5831E0241729
:1044400008F030E05E2D505C41E05E1508F040E081
:10445000350FA1E0351708F0A0E04A2B460F51E0D8
:10446000461708F050E0570F61E0571708F060E07A
:10447000680F71E0681708F070E07E0F81E07E172A
:1044800008F080E08F0FE1E08F1708F0E0E09E0F6A
:10449000A32CB92CC22CD82CE72CF62C052D1DA151
:1044A0000E94D78A01E00E94128C0889200F01E047
:1044B0001889211708F000E01B89130FE1E03B8900
:1044C000131708F0E0E0302F310FF1E0311708F05A
:1044D000F0E0EF2B1C89140FF1E04C89141708F061
:1044E000F0E04E2F410FE1E0411708F0E0E0FE2B35
:1044F0001D89150FE1E05D89151708F0E0E05F2FD9
:10450000510FF1E0511708F0F0E0EF2BFE89F60FA4
:1045100011E06E89F61708F010E06E2F6F0FE1E0E2
:104520006F1708F0E0E01E2BEF89E70FF1E07F89BD
:10453000E71708F0F0E0712F7E0FA1E07E1708F07A
:10454000A0E0FA2BA88D8A0FE1E08A1708F0E0E0DE
:10455000F80FA1E0F81708F0A0E0EA2BB8A99B0F2C
:10456000E90FD988EEA0DE1891E0F988FD1408F073
:1045700090E0898D09A5801B11E0A98DA81708F08E
:1045800010E0E82EE91A91E08E1508F090E0192B62
:104590008A8DBAA58B1B91E0FA8CF81608F090E092
:1045A000F82EF11AA1E08F1508F0A0E09A2B8B8D60
:1045B0000BA5801B11E0AB8DA81708F010E0082FA9
:1045C000091B91E0801708F090E0192B8C8DBCA599
:1045D0008B1B91E0AC8DA81708F090E0B82FB11BB1
:1045E0001B2FA1E08B1708F0A0E09A2B8D8DADA5B5
:1045F0008A1BCC24C394BD8DB81708F0CC24B82EE8
:10460000B91A91E08B1508F090E0C92A9E8D8EA50D
:10461000981B81E0AE8DA91708F080E0A92EAC1898
:10462000CC24C3949A1508F0CC248C29BFA198857A
:10463000B91BD9A6EAA6FBA60CA71DA7BEA6AFA6C6
:10464000B81BBB8BAA89A21B2A2F91E0BA89BA1783
:1046500008F090E01F8D131B81E0EF8CE11608F04D
:1046600080E0312F391B91E0131708F090E0892B7F
:1046700018A1141B91E0F8A0F11608F090E0412F6A
:10468000481B81E0141708F080E0982B19A1151B36
:1046900081E009A1011708F080E0512F591B91E03A
:1046A000151708F090E0892B1AA1161B91E06AA15A
:1046B000611708F090E0612F681B81E0161708F081
:1046C00080E0982B1BA1171B81E07BA1711708F0DC
:1046D00080E0712F791B91E0171708F090E0892B8B
:1046E0009CA19F1BF1E0ACA1A91708F0F0E0B92F45
:1046F000B81B8B2FA1E09B1708F0A0E0FA2B98A520
:104700009E1B9F1B8F80EDA98E1A11E0FF81F8156B
:1047100008F010E0FA80EEA8FE1801E0AA81AF15BB
:1047200008F000E0AF2CA11A11E0FA1408F010E034
:10473000012B1981BFA91B1BB1E0E981E11708F02A
:10474000B0E0F12FF01B0F2FE1E01F1708F0E0E0C1
:10475000BE2B1B81E8AC1E19A1E0FB80F11608F00E
:10476000A0E0912E9B1AFF24F394191508F0FF2462
:10477000AF29FC8019ADF11A11E0BC81BF1508F01A
:1047800010E0EF2CEA1AE1E0FE1408F0E0E01E2B46
:10479000ED81FAADEF1BFF24F394AD81AE1708F065
:1047A000FF24BE2FB11B1B2FDD24D394EB1708F081
:1047B000DD24FD28DE80EBADDE1AE1E0FE81FD1593
:1047C00008F0E0E0CD2CCF18FF24F394DC1408F0BF
:1047D000FF24EF29F984ACADFA1AFE1AF0EADF2EB5
:1047E000D80CBB24B394D81408F0BB24EA2DE15FA5
:1047F000F1E0EA1508F0F0E0AB2DAE0FBB24B39466
:10480000AE1708F0BB24FB29F00FE1E0F01708F029
:10481000E0E0E90D01E0E91508F000E0B02FBE0D81
:1048200001E0BE1508F000E0010FEE24E39401174B
:1048300008F0EE241E2D1C0DEE24E3941C1508F048
:10484000EE24FE0C89F4112379F4002369F4BB23D0
:1048500059F4EE2349F4FF2339F4A13328F4A033AB
:1048600061F4BD2DB53D48F02796EEADFFAD27971D
:1048700031962796FFAFEEAF2797E9A8FAA80BA9C4
:104880001CA91701280157016201EE24FF2400E052
:1048900010E00E94D78AF901DA01162F072FF82EAF
:1048A000E92EE7FE32C0215031E02E1708F030E04B
:1048B0008F2F815041E08F1708F040E0380F91E0D2
:1048C000381708F090E0492B8A2F815E51E08A1753
:1048D00008F050E0480F91E0481708F090E0592B9D
:1048E0005B0F61E05B1708F060E0610F71E061173A
:1048F00008F070E0700F81E0701708F080E08F0D15
:1049000091E08F1508F090E09E0D05E10E94128C59
:10491000122FF9A41F19F1E0211708F0F0E0232F5E
:104920000AA5201BE1E0321708F0E0E0E22EEF1AC2
:1049300031E02E1508F030E0E32B342F2BA5321B8D
:1049400021E0431708F020E0F32EFE1A41E03F1566
:1049500008F040E0242B452F3CA5431B31E05417C1
:1049600008F030E0042F021B21E0401708F020E09F
:10497000322B462F5DA5451B21E0641708F020E08F
:10498000D42ED31A31E04D1508F030E0232B472FF9
:104990006EA5461B31E0741708F030E0C42EC21A31
:1049A00021E04C1508F020E0322B482F7FA5471B53
:1049B00021E0841708F020E0F42FF31B81E04F176B
:1049C00008F080E0282BE92F8B89E81BE21B212FC0
:1049D0003E2D4F2D502F6D2D7C2D8F2F9E2FE7FFBD
:1049E0002BC0215031E0211708F030E08E2D815886
:1049F00041E08E1508F040E0380F91E0381708F0DC
:104A000090E0492B4F0D51E04F1508F050E0500F4A
:104A100061E0501708F060E06D0D71E06D1508F071
:104A200070E07C0D81E07C1508F080E08F0F91E054
:104A30008F1708F090E09E0F0FE00E94128C022F5B
:104A4000F32ED42EB52EA62EC72EE82E192FE8E170
:104A50007E2E700EA1E0701608F0A0E0FF2DF4503D
:104A6000E1E0FF1508F0E0E0AF0FB1E0AF1708F0AC
:104A7000B0E0EB2B9D2C9A94F1E09D1408F0F0E04F
:104A8000BE2FB90DE1E0B91508F0E0E0FE2B9B2C3C
:104A90009A94E1E09B1408F0E0E06F2E690CF1E0DD
:104AA000691408F0F0E0EF2B962E9A94F1E0961638
:104AB00008F0F0E05E2E590CE1E0591408F0E0E057
:104AC000FE2B972E9A94E1E0971608F0E0E0F90D9E
:104AD00088248394F91508F08824E829882E8A947C
:104AE00099249394881608F09924E80D442443945B
:104AF000E81508F044249428892E8A94980C99F497
:104B0000EE2389F4FF2379F4552069F4662059F4E3
:104B1000B23048F4B13081F4A13D28F4A03D61F4F5
:104B2000A72DA93D48F02796EEADFFAD279731960A
:104B30002796FFAFEEAF27972DAF3EAF4FAF219631
:104B40005FAF219722966FAF229723967FAF23976F
:104B500024968FAF249725969FAF25970E94776460
:104B60002DAD3EAD4FAD21965FAD219722966FAD35
:104B7000229723967FAD239724968FAD2497259671
:104B80009FAD25972796AEADBFAD2797109709F437
:104B900053C0019521E0101608F020E0F19441E0A7
:104BA0001F1408F040E03F2D321B21E0F31608F0FF
:104BB00020E0422BD19451E01D1408F050E0BD2DAF
:104BC000B41B4B2F21E0DB1608F020E0522BB194F0
:104BD000E1E01B1408F0E0E0FB2DF51B5F2F21E066
:104BE000BF1608F020E0E22B6195F1E0161608F000
:104BF000F0E0A62EAE1A21E06A1508F020E0F22BB4
:104C00007195E1E0171608F0E0E0C72ECF1A21E019
:104C10007C1508F020E0E22B819561E0181608F081
:104C200060E0E82EEE1A21E08E1508F020E0622BFD
:104C3000192F1195202F161B6A2D7C2D8E2D912F4B
:104C40000E94D89920E030E048EC52E40E940E998E
:104C5000CA5BDF4F0FB6F894DEBF0FBECDBFCF915A
:104C6000DF911F910F91FF90EF90DF90CF90BF9059
:104C7000AF909F908F907F906F905F904F903F90FC
:104C80002F9008956F927F928F929F92AF92BF92D2
:104C9000CF92DF92EF92FF920F931F933B014C0153
:104CA00079018A01CA01B90123EC35EF4CE851E4DE
:104CB0000E94BC9B5B016C01C801B70128EB3EE17F
:104CC00043E753E40E9444989B01AC01C601B5013F
:104CD0000E940E990E947B995B016C01C401B30193
:104CE00020E030E048EC52E40E940E9921E835E9DA
:104CF00043EC50E40E94BC9BA60195010E94BC9B22
:104D00005B016C01C801B70123E333E948E853E4D0
:104D10000E9444989B01AC01C601B5010E940E9906
:104D200023E333EB48E553E40E94BC9B1F910F91B2
:104D3000FF90EF90DF90CF90BF90AF909F908F90BB
:104D40007F906F9008956F927F928F929F92AF9213
:104D5000BF92CF92DF92EF92FF920F931F93790150
:104D60008A010E943E9B20E030E040E050E40E9437
:104D7000439822E93CE54EED5EE30E940E993B012B
:104D80004C01C801B70123EC35EF4CE851E40E9417
:104D9000BC9B5B016C01C801B70128EB3EE143E716
:104DA00053E40E9444989B01AC01C601B5010E94E6
:104DB0000E999B01AC01C401B3010E9444988B0180
:104DC000A82EE92E712F28EB3EE143E753E40E9421
:104DD000BC9B3B014C0163EC75EF8CE891E4202F08
:104DE000312F4A2D5E2D0E9443989B01AC01C401D6
:104DF000B3010E940E991F910F91FF90EF90DF90E9
:104E0000CF90BF90AF909F908F907F906F900895BC
:104E10006F927F928F929F92AF92BF92CF92DF92CA
:104E2000EF92FF920F931F933B014C0179018A018E
:104E3000CA01B90123EC35EF4CE851E40E94BC9B58
:104E40005B016C01C801B70128EB3EE143E753E485
:104E50000E9444989B01AC01C601B5010E940E99C5
:104E60000E947B995B016C01C401B30120E030E03A
:104E700048EC52E40E940E99A60195010E94BC9B49
:104E800020E030E040E251E40E94439824EE38E311
:104E90004EE05FE30E94BC9B9B01AC01C801B701DF
:104EA0000E9444981F910F91FF90EF90DF90CF9058
:104EB000BF90AF909F908F907F906F900895AF922A
:104EC000BF92CF92DF92EF92FF920F931F9380E8F1
:104ED0000E9474648AEF0E947F648FE00E947F6466
:104EE00065E375E080E090E00E94FE6381E80E9447
:104EF00074640E949064E82E0E9490640E94906402
:104F0000F82E0E9490640E949064082F0E94906482
:104F10000E949A64182F0E949A6480E80E94746428
:104F20008CEF0E947F6489EC0E947F6465E375E0EA
:104F300080E090E00E94FE6381E80E9474640E9419
:104F40009064C82E0E949064D82E0E9490640E94A3
:104F50009064A82E0E949064B82E0E949A648DB727
:104F60009EB742970FB6F8949EBF0FBE8DBFEDB7A8
:104F7000FEB7319629E133E0ADB7BEB712963C9348
:104F80002E931197A2821382B4821582E682178231
:104F9000F08611860287138614871586C6861786C3
:104FA000D08A118A0E9478A18DB79EB742960FB61B
:104FB000F8949EBF0FBE8DBF0E94776420E030E062
:104FC00040E050E060E070E080E090E01F910F91E1
:104FD000FF90EF90DF90CF90BF90AF9008950F9328
:104FE0001F93CF93DF93EC0180E80E9474642097B5
:104FF00041F085EE0E947F6461E077E980E090E017
:1050000007C083EE0E947F6469E97AEB81E090E05B
:105010000E94FE6381E80E9474640E949064082FDD
:105020000E949064182F0E949A640E947764302F27
:1050300020E0612F70E0622B732B6C7F80E090E0AA
:10504000209769F00E94DC9920E030E04AEF5AE3B3
:105050000E94BC9B20E030E040EC50E40CC00E9479
:10506000DC9922E538EB4FE25BE30E94BC9B26E62D
:1050700036E64BE352E40E944398DF91CF911F91B3
:105080000F910895EF92FF920F931F93CF93DF93A9
:10509000729A8091EF0683FD06C0C0E5D0E00E94C1
:1050A000BA0B2197E1F78EE40E9411648823B1F0D6
:1050B0008091392490913A24A0913B24B0913C24D2
:1050C0000196A11DB11D8093392490933A24A09399
:1050D0003B24B0933C2421E030E087C0C0E5D0E021
:1050E0000E94BA0B2197E1F78FE40E9411640E949D
:1050F0009064982F92959695969593709130A9F417
:1051000020913D2430913E2440913F2450914024F1
:105110002F5F3F4F4F4F5F4F20933D2430933E24EE
:1051200040933F245093402416C09230A0F0209129
:1051300041243091422440914324509144242F5FD4
:105140003F4F4F4F5F4F2093412430934224409371
:105150004324509344241FE3E12EE8220E949064EC
:10516000F82E0E949064082F0E949A64182F0E94C3
:1051700077648091EF0683FF72987E2D60E06F0D5B
:10518000711D80E090E00E94DC9920E134E048EC61
:105190005BE30E94BC9B60932F1C7093301C809338
:1051A000311C9093321C702F60E0610F711D769559
:1051B00067957695679580E090E00E94DC9924EAF7
:1051C0003CEF44E25CE30E94BC9B20E030E040E224
:1051D00052E40E9443986093B2287093B32880935E
:1051E000B4289093B52820E030E0C901DF91CF9139
:1051F0001F910F91FF90EF9008957298729A8EE42C
:105200000E94116480EA0E947F6480E00E947F64B3
:1052100080E00E947F648FE40E9411640E94906489
:1052200082958695869583708130A9F420913D24DE
:1052300030913E2440913F24509140242F5F3F4FB6
:105240004F4F5F4F20933D2430933E2440933F24A3
:105250005093402416C08230A0F020914124309118
:10526000422440914324509144242F5F3F4F4F4F9D
:105270005F4F209341243093422440934324509322
:10528000442400D000D0EDB7FEB7319628E433E0D7
:10529000ADB7BEB712963C932E93119782831382BB
:1052A0000E9478A10F900F900F900F908EE40E94B3
:1052B000116480E80E947F6480E00E947F6480E047
:1052C0000E947F640E94776480E090E0089500D09F
:1052D00081E09DE0ADB7BEB712969C938E93119777
:1052E0000E948AA12091D1060F900F902223A9F04D
:1052F00000D000D0EDB7FEB731968EEF9CE0ADB791
:10530000BEB712969C938E931197228313820E94AC
:105310008AA10F900F900F900F90089500D089ED03
:105320009CE0EDB7FEB7928381830E948AA181EB56
:105330009CE0EDB7FEB7928381830E948AA18AE840
:105340009CE0EDB7FEB7928381830E948AA18FE42F
:105350009CE0EDB7FEB7928381830E948AA18DE124
:105360009CE0EDB7FEB7928381830E948AA181EE13
:105370009BE0EDB7FEB7928381830E948AA18BEBFD
:105380009BE0EDB7FEB7928381830E948AA185E8F6
:105390009BE0EDB7FEB7928381830E948AA1809142
:1053A000332090913420827091700F900F9000976D
:1053B00059F000D085E59BE0EDB7FEB7928381837D
:1053C0000E948AA10F900F9000D089E29BE0EDB778
:1053D000FEB7928381830E948AA180E09BE0EDB7B3
:1053E000FEB7928381830E948AA185ED9AE0EDB792
:1053F000FEB7928381830E948AA186EA9AE0EDB784
:10540000FEB7928381830E948AA184E79AE0EDB778
:10541000FEB7928381830E948AA183E49AE0EDB76C
:10542000FEB7928381830E948AA18FE09AE0EDB754
:10543000FEB7928381830E948AA18FED99E0EDB738
:10544000FEB7928381830E948AA183EB99E0EDB736
:10545000FEB7928381830E948AA184E899E0EDB728
:10546000FEB7928381830E948AA18BE499E0EDB715
:10547000FEB7928381830E948AA182E199E0EDB711
:10548000FEB7928381830E948AA18BED98E0EDB7ED
:10549000FEB7928381830E948AA18AEA98E0EDB7E1
:1054A000FEB7928381830E948AA18BE798E0EDB7D3
:1054B000FEB7928381830E948AA18CE498E0EDB7C5
:1054C000FEB7928381830E948AA185E298E0EDB7BE
:1054D000FEB7928381830E948AA18FEE97E0EDB799
:1054E000FEB7928381830E948AA186EC97E0EDB794
:1054F000FEB7928381830E948AA18BE997E0EDB782
:10550000FEB7928381830E948AA10F900F90089525
:1055100088E593E00E94AAA108952F923F924F92AE
:105520005F926F927F928F929F92AF92BF92CF9233
:10553000DF92EF92FF920F931F93CF93DF936091CF
:105540003524709136248091372490913824A0908E
:105550003524B0903624C0903724D0903824609001
:1055600035247090362480903724909038242090F1
:1055700035243090362440903724509038242DB76D
:105580003EB72A5030400FB6F8943EBF0FBE2DBF35
:10559000CDB7DEB7219625E737E0EDB7FEB732830A
:1055A000218340E8E42E41E5F42E41E0042F112D43
:1055B000A80197010E94C29C3B832A83C601B501C2
:1055C000A80197010E94C29C30E1E32E3EE0F32E39
:1055D000012D112DA80197010E94C29C332727FDA0
:1055E00030953D832C83C401B301A80197010E942B
:1055F000C29C2CE3E22EF12C012D112DA801970164
:105600000E94C29C332727FD30953F832E83C20121
:10561000B101A80197010E94C29C772767FD709590
:10562000798768870E948AA12DB73EB7265F3F4FD2
:105630000FB6F8943EBF0FBE2DBFDF91CF911F91E3
:105640000F91FF90EF90DF90CF90BF90AF909F9021
:105650008F907F906F905F904F903F902F90089524
:10566000E7E7F1E38081918122E482349207B9F087
:1056700000D000D087E597E0ADB7BEB712969C93F7
:105680008E931197E757F1431496FC93EE9313977B
:105690000E948AA10F900F900F900F9008953A9654
:1056A000B1E4E53FFB07F0F208950F931F93CF930A
:1056B000DF93EC018C9A0E949C0C00D000D000D0AB
:1056C0002BE437E0EDB7FEB7328321836383748325
:1056D000858396830E948AA18DB79EB706960FB6E2
:1056E000F8949EBF0FBE8DBF209719F00E94AD0D9C
:1056F0000BC000D089E497E0EDB7FEB792838183B9
:105700000E948AA10F900F9081E00E944E0C00D061
:1057100000D000D00DB71EB70F5F1F4F2DE337E04D
:10572000EDB7FEB7328321832091C9063091CA06B6
:105730004091CB065091CC060E94BC9BF80162833D
:105740007383848395830E948AA18DB79EB7069642
:105750000FB6F8949EBF0FBE8DBF209719F00E9420
:10576000AD0D0BC000D08BE397E0EDB7FEB7928391
:1057700081830E948AA10F900F9082E00E944E0CBC
:1057800000D000D000D00DB71EB70F5F1F4F2FE223
:1057900037E0EDB7FEB7328321832091CD063091FB
:1057A000CE064091CF065091D0060E94BC9BF801D6
:1057B00062837383848395830E948AA18DB79EB789
:1057C00006960FB6F8949EBF0FBE8DBF209719F0B6
:1057D0000E94AD0D0BC000D08DE297E0EDB7FEB793
:1057E000928381830E948AA10F900F9083E00E9490
:1057F0004E0C00D000D000D02EE137E0EDB7FEB760
:105800003283218363837483858396830E948AA174
:105810008C988DB79EB706960FB6F8949EBF0FBEB4
:105820008DBF209719F00E94AD0D0BC000D08CE108
:1058300097E0EDB7FEB7928381830E948AA10F9013
:105840000F908091332087FFA4C080ED61E042E19A
:1058500021E00E94E76500D000D000D02FE037E0C3
:10586000EDB7FEB732832183638374838583968388
:105870000E948AA18DB79EB706960FB6F8949EBF78
:105880000FBE8DBF209719F00E94AD0D0BC000D048
:105890008DE097E0EDB7FEB7928381830E948AA1E5
:1058A0000F900F9080ED62E042E121E00E94E765F9
:1058B00000D000D000D020E037E0EDB7FEB7328353
:1058C000218363837483858396830E948AA18DB725
:1058D0009EB706960FB6F8949EBF0FBE8DBF209759
:1058E00019F00E94AD0D0BC000D08EEF96E0EDB721
:1058F000FEB7928381830E948AA10F900F9080ED62
:1059000063E042E121E00E94E76500D000D000D0D2
:1059100021EF36E0EDB7FEB73283218363837483D2
:10592000858396830E948AA18DB79EB706960FB68F
:10593000F8949EBF0FBE8DBF209719F00E94AD0D49
:105940000BC000D08FEE96E0EDB7FEB79283818357
:105950000E948AA10F900F9080ED64E042E121E067
:105960000E94E76500D000D000D022EE36E0EDB70F
:10597000FEB73283218363837483858396830E9479
:105980008AA18DB79EB706960FB6F8949EBF0FBE3C
:105990008DBF209711F40E94AD0DDF91CF911F9123
:1059A0000F9108950F931F93CF93DF93882389F06E
:1059B00086EA98E26FEF70E049E050E00E94F3A0C1
:1059C00086EA98E269E170E049E050E00E94D3A2E3
:1059D0001CC0C6EAD8E20DED16E0899100D000D0D7
:1059E000EDB7FEB73196ADB7BEB712961C930E93C6
:1059F0001197828313820E948AA10F900F900F90BB
:105A00000F90B8E2CE3ADB0741F70E94AD0DDF916F
:105A1000CF911F910F910895EF92FF920F931F93D3
:105A20006091D7067091D80680E090E00E94E5A0D2
:105A300063E773E00E94FAA0009709F0B6C08DE416
:105A400090E2A1E0B0E08093E9069093EA06A0938B
:105A5000EB06B093EC0689EE96E06EE070E044E071
:105A600050E00E94D3A28CE390E09093EE068093E6
:105A7000ED068DEE96E062E170E042E050E00E94BB
:105A8000D3A28AE090E49093F0068093EF068FEE25
:105A900096E064E170E042E050E00E94D3A21092F0
:105AA000090A1092080A88E09AE060E070E042E09B
:105AB00050E00E94D3A20F2EF2E2EF2EFFEFFF2E56
:105AC000FCEC0F2FFBE31F2FF02DE092C906F092A4
:105AD000CA060093CB061093CC0689EC96E066E0EC
:105AE00070E044E050E00E94D3A2E092CD06F09234
:105AF000CE060093CF061093D0068DEC96E06AE0B8
:105B000070E044E050E00E94D3A287ED94E3AFEE52
:105B1000BCE38093C5069093C606A093C706B093D6
:105B2000C80685EC96E062E070E044E050E00E9438
:105B3000D3A210920D0A80E090E00E94E36F8DE006
:105B40009AE066E170E041E050E00E94D3A28AE171
:105B50008093F1068AE190E00E945B6E81EF96E00F
:105B600067E170E041E050E00E94D3A28FE08093B3
:105B7000F20682EF96E068E170E041E050E00E94BA
:105B8000D3A288E59BE12AE0FC0111922A95E9F76E
:105B900062E270E04AE050E00E94D3A281E00E94FD
:105BA000D22C80E090E00E94770F1F910F91FF9020
:105BB000EF900895EF92FF920F931F93CF93DF938F
:105BC0007B018C01CB0181709070009749F080E0DF
:105BD00090E06AE773E00E94900B81E090E002C0E1
:105BE00080E090E0E1FE07C0EC0121966FE773E0F2
:105BF0000E94900BCE01E2FE07C0EC01219667E8FF
:105C000073E00E94900BCE01E3FE07C0EC012196E9
:105C10006FE873E00E94900BCE01E4FE07C0EC0138
:105C2000219663E973E00E94900BCE01E5FE07C068
:105C3000EC01219666E973E00E94900BCE01E6FE2E
:105C400007C0EC0121966AE973E00E94900BCE0137
:105C5000E7FE07C0EC01219660EA73E00E94900B1A
:105C6000CE01F0FE07C0EC01219668EA73E00E94C5
:105C7000900BCE01F1FE07C0EC01219660EB73E0C2
:105C80000E94900BCE01F2FE07C0EC01219664EB5E
:105C900073E00E94900BCE0120913320309134208C
:105CA000247032702115310549F0F3FE07C0EC0174
:105CB00021966AEB73E00E94900BCE012091332075
:105CC00023FF09C0F4FE07C0EC0121966FEB73E0DF
:105CD0000E94900BCE012091332024FF09C0F5FED5
:105CE00007C0EC01219665EC73E00E94900BCE0199
:105CF000F6FE05C06DEC73E00E94900B10C0E1143D
:105D0000F1040105110559F400D088ED96E0EDB7D6
:105D1000FEB7928381830E948AA10F900F90DF913A
:105D2000CF911F910F91FF90EF900895EF92FF9206
:105D30000F931F93CF93DF938C01C0E0D0E081C01D
:105D4000C80163ED76E00E94D1A0009709F4C1601C
:105D5000C8016BEC76E00E94D1A0009709F4C26004
:105D6000C80163EC76E00E94D1A0009709F4C460FA
:105D7000C8016FEB76E00E94D1A0009709F4C860DB
:105D8000C8016CEB76E00E94D1A0009709F4C061D5
:105D9000C80168EB76E00E94D1A0009709F4C062C8
:105DA000C80162EB76E00E94D1A0009709F4C064BC
:105DB000C8016AEA76E00E94D1A0009709F4C068A1
:105DC000C80162EA76E00E94D1A0009709F4D16090
:105DD000C8016EE976E00E94D1A0009709F4D26074
:105DE000C80168E976E00E94D1A0009709F4D46068
:105DF000C80163E976E00E94D1A0009709F4D86059
:105E0000C8016DE876E00E94D1A0009709F4D06146
:105E1000C80165E876E00E94D1A0009709F4D0623D
:105E2000C8016AE776E00E94D1A0009709F4D06427
:105E30006091D7067091D80680E090E00E94E5A0BE
:105E40008C010115110509F07BCFCE01DF91CF91B7
:105E50001F910F91FF90EF900895EF92FF920F9393
:105E60001F93CF93DF937B018C01CB0181709070E6
:105E7000009749F080E090E068ED73E00E94900B9D
:105E800081E090E002C080E090E02091332020FF8C
:105E900009C0E2FE07C0EC0121966CED73E00E94A0
:105EA000900BCE01E1FE07C0EC01219660EE73E09D
:105EB0000E94900BCE01E3FE07C0EC01219663EE39
:105EC00073E00E94900BCE01E4FE07C0EC01219626
:105ED00065EE73E00E94900BCE01E5FE07C0EC0179
:105EE000219668EE73E00E94900BCE01E6FE07C09B
:105EF000EC0121966EEE73E00E94900BCE01E7FE5E
:105F000007C0EC01219664EF73E00E94900BCE0174
:105F1000F0FE07C0EC01219667EF73E00E94900B42
:105F2000CE01F1FE07C0EC0121966CEF73E00E94F8
:105F3000900BCE01F2FE07C0EC0121966FEF73E0EB
:105F40000E94900BCE01F3FE07C0EC01219664E0A5
:105F500074E00E94900BCE012091332021FF09C0F4
:105F6000F4FE07C0EC0121966BE074E00E94900BF8
:105F7000CE01209133203091342030FF09C012FF30
:105F800007C0EC0121966EE074E00E94900BCE01F8
:105F9000209133203091342030FF09C013FF07C017
:105FA000EC01219661E174E00E94900BCE012091FA
:105FB00033203091342030FF09C014FF07C0EC01BA
:105FC000219667E174E00E94900BCE01F5FE07C0B8
:105FD000EC01219662E274E00E94900BCE01F6FE85
:105FE00007C0EC01219667E274E00E94900BCE019D
:105FF000F7FE07C0EC0121966AE274E00E94900B64
:10600000CE0100FF07C0EC0121966DE274E00E9412
:10601000900BCE012091332027FF09C001FF07C05C
:10602000EC01219660E374E00E94900BCE01209178
:10603000332027FF09C002FF07C0EC01219664E36B
:1060400074E00E94900BCE012091332027FF09C0FD
:1060500003FF07C0EC01219668E374E00E94900BF7
:10606000CE012091332027FF09C004FF07C0EC01B7
:1060700021966CE374E00E94900BCE0120913320B6
:1060800022FF09C005FF07C0EC01219660E474E01F
:106090000E94900BCE012091332022FF09C006FF01
:1060A00007C0EC01219662E474E00E94900BCE01DF
:1060B000209133203091342030FF09C007FF07C002
:1060C000EC01219665E474E00E94900BCE012091D2
:1060D00033203091342030FF09C010FF07C0EC019D
:1060E00021966DE474E00E94900BCE012091332044
:1060F0003091342031FF07C011FF05C066E574E020
:106100000E94900B10C0E114F1040105110559F42F
:1061100000D085E796E0EDB7FEB7928381830E94B9
:106120008AA10F900F90DF91CF911F910F91FF9057
:10613000EF900895EF92FF920F931F93CF93DF9309
:10614000EC0160E776E00E94D1A0009709F04DC015
:106150008091332082FF08C06DE4E62E60E2F62EC7
:1061600061E2062F112D07C05DE4E52E50E2F52E09
:1061700051E0052F112D81FF08C020E030E140E003
:1061800050E0E22AF32A042B152B89E290E06BE21F
:1061900070E04AE250E026E00E94216181E090E058
:1061A0000E94210D882341F080E190E0A0E0B0E062
:1061B000E82AF92A0A2B1B2B809133209091342056
:1061C00090FF08C020E030E040E851E0E22AF32AE6
:1061D000042B152B91FFC9C180E090E0A0E0B2E054
:1061E000E82AF92A0A2B1B2BC0C1EE24FF248701C1
:1061F000BCC1CE016CE676E00E94D1A0009741F4CC
:1062000021E030E040E050E0E22AF32A042B152B95
:10621000CE0168E676E00E94D1A0009741F484E0C8
:1062200090E0A0E0B0E0E82AF92A0A2B1B2BCE016F
:1062300065E676E00E94D1A0009741F422E030E0CC
:1062400040E050E0E22AF32A042B152BCE0163E64E
:1062500076E00E94D1A0009741F488E090E0A0E0B1
:10626000B0E0E82AF92A0A2B1B2BCE0160E676E083
:106270000E94D1A0009741F420E130E040E050E0DE
:10628000E22AF32A042B152BCE016AE576E00E9460
:10629000D1A0009741F480E290E0A0E0B0E0E82ACD
:1062A000F92A0A2B1B2BCE0164E576E00E94D1A0CF
:1062B000009741F420E430E040E050E0E22AF32A85
:1062C000042B152BCE0161E576E00E94D1A000974A
:1062D00041F480E890E0A0E0B0E0E82AF92A0A2B37
:1062E0001B2BCE016CE476E00E94D1A0009741F414
:1062F00020E031E040E050E0E22AF32A042B152BA5
:10630000CE0169E476E00E94D1A0009741F480E0DC
:1063100092E0A0E0B0E0E82AF92A0A2B1B2BCE017C
:1063200064E476E00E94D1A0009741F420E034E0DC
:1063300040E050E0E22AF32A042B152BCE016DE356
:1063400076E00E94D1A0009741F480E098E0A0E0C0
:10635000B0E0E82AF92A0A2B1B2BCE016AE376E08B
:106360000E94D1A0009741F420E030E140E050E0ED
:10637000E22AF32A042B152BCE0165E376E00E9476
:10638000D1A0009741F480E090E2A0E0B0E0E82ADC
:10639000F92A0A2B1B2BCE0162E376E00E94D1A0E2
:1063A000009741F420E030E440E050E0E22AF32A94
:1063B000042B152BCE016FE276E00E94D1A000974E
:1063C00041F480E090E8A0E0B0E0E82AF92A0A2B46
:1063D0001B2BCE016CE276E00E94D1A0009741F425
:1063E00020E030E041E050E0E22AF32A042B152BB4
:1063F000CE0168E276E00E94D1A0009741F480E0EF
:1064000090E0A2E0B0E0E82AF92A0A2B1B2BCE018B
:1064100064E276E00E94D1A0009741F420E030E0F1
:1064200044E050E0E22AF32A042B152BCE0160E26F
:1064300076E00E94D1A0009741F480E090E0A8E0CF
:10644000B0E0E82AF92A0A2B1B2BCE016CE176E09A
:106450000E94D1A0009741F420E030E040E150E0FC
:10646000E22AF32A042B152BCE016AE176E00E9482
:10647000D1A0009741F480E090E0A0E2B0E0E82AEB
:10648000F92A0A2B1B2BCE0167E176E00E94D1A0EE
:10649000009741F420E030E040E450E0E22AF32AA3
:1064A000042B152BCE016FE076E00E94D1A000975F
:1064B00041F480E090E0A0E8B0E0E82AF92A0A2B55
:1064C0001B2BCE0166E076E00E94D1A0009741F43C
:1064D00020E030E040E051E0E22AF32A042B152BC3
:1064E000CE016DEF75E00E94D1A0009741F480E0ED
:1064F00090E0A0E0B2E0E82AF92A0A2B1B2BCE019B
:106500006AEF75E00E94D1A0009741F420E030E0EE
:1065100040E054E0E22AF32A042B152BCE0164EF6D
:1065200075E00E94D1A0009741F480E090E0A0E0E7
:10653000B8E0E82AF92A0A2B1B2BCE0169EE75E098
:106540000E94D1A0009741F420E030E040E050E10B
:10655000E22AF32A042B152B6091D7067091D806F6
:1065600080E090E00E94E5A0EC01209709F041CE88
:10657000B701C801DF91CF911F910F91FF90EF906C
:10658000089500D089ED95E0ADB7BEB712969C9303
:106590008E9311970E948AA10F900F900E94882AD3
:1065A00000D000D081ED95E0EDB7FEB792838183F6
:1065B00088E59BE1948383830E948AA10F900F90CA
:1065C0008DEC95E0ADB7BEB712969C938E93119764
:1065D0000E948AA10F900F9080E00E94D22C00D0E0
:1065E00088EC95E0EDB7FEB7928381830E948AA183
:1065F0000F900F900E9400128091332080FF05C001
:1066000081E061E041E00E948F130E948D2A00D05A
:1066100000D0EDB7FEB731968FEB95E0ADB7BEB7C2
:1066200012969C938E9311978091F1068283138228
:106630000E948AA1EDB7FEB7319686EB95E0ADB723
:10664000BEB712969C938E93119780910D0A828308
:1066500013820E948AA18EE995E0EDB7FEB792837E
:10666000818380E490E0948383830E948AA100D098
:10667000EDB7FEB731968BE895E0ADB7BEB7129691
:106680009C938E9311978091B62882831382809178
:10669000B728848315820E948AA10F900F90EDB7CE
:1066A000FEB7319682E895E0ADB7BEB712969C93DF
:1066B0008E9311978091F206828313820E948AA1A1
:1066C0008091EF069091F0060F900F900F900F9031
:1066D00096FF03C08FE594E002C082E694E000D00C
:1066E00000D028E735E0EDB7FEB7328321839483ED
:1066F00083830E948AA183E695E0ADB7BEB7129668
:106700009C938E9311978091ED069091EE061496CE
:106710009C938E9313970E948AA10F900F908BE504
:1067200095E0EDB7FEB7928381830E948AA10F9016
:106730000F906091E9067091EA068091EB069091C6
:10674000EC060E942D2F0E94AD0D1D9B03C08FE50E
:1067500094E002C082E694E000D000D02FE435E05F
:10676000ADB7BEB712963C932E93119714969C9397
:106770008E9313970E948AA10F900F9085E495E065
:10678000EDB7FEB7928381830E948AA18091EF06C4
:106790000F900F9081FF0EC000D08FE395E0ADB752
:1067A000BEB712969C938E9311970E948AA10F9068
:1067B0000F9017C080FF03C08FE594E002C082E60F
:1067C00094E000D000D02BE335E0EDB7FEB7328384
:1067D0002183948383830E948AA10F900F900F904E
:1067E0000F9000D084E395E0ADB7BEB712969C93AE
:1067F0008E9311970E948AA16091080A7091090AEC
:106800000F900F9080E090E00E94DA2D0E94AD0D75
:10681000779903C08FE594E002C082E694E000D04F
:1068200000D02BE235E0EDB7FEB7328321839483AD
:1068300083830E948AA10F900F900F900F900E9467
:106840008F086091E9067091EA068091EB069091BD
:10685000EC060E94D30C0E94B00C00D000D000D0F7
:106860002DE135E0ADB7BEB712963C932E9311974C
:10687000EDB7FEB763837483858396830E948AA1F4
:106880008DB79EB706960FB6F8949EBF0FBE8DBF0C
:1068900081E090E00E94552B809191289091922860
:1068A000A0919328B091942800D000D000D02FE080
:1068B00035E0EDB7FEB73283218383839483A583CC
:1068C000B6830E948AA18BEF94E0ADB7BEB7129653
:1068D0009C938E93119780919E2890919F28A091D0
:1068E000A028B091A128EDB7FEB783839483A58338
:1068F000B6830E948AA18091952890919628A091B4
:106900009728B09198282DEE34E0EDB7FEB732838A
:10691000218383839483A583B6830E948AA189ED12
:1069200094E0ADB7BEB712969C938E931197809169
:10693000A2289091A328A091A428B091A528EDB7F2
:10694000FEB783839483A583B6830E948AA18DB703
:106950009EB706960FB6F8949EBF0FBE8DBF80E01F
:1069600090E061E070E00E94B90D81E090E061E0AC
:1069700070E00E94B90D08952F923F924F925F925E
:106980006F927F928F929F92AF92BF92CF92DF923F
:10699000EF92FF920F931F93DF93CF9300D0CDB769
:1069A000DEB79A838983DC018D919C9111970097C2
:1069B00011F00C94AD476091D7067091D80681E52F
:1069C00094E20E94E5A081E594E260E470E00E9418
:1069D00012A1009759F460917131709172318AE07F
:1069E00090E00E944CA181E00C94B3478130910566
:1069F00049F42090512433244424552466247724D8
:106A00004301BEC18230910599F430915124209107
:106A10005224932F80E0820F911D1C01892F880F33
:106A2000880B482E582E682E782E882E982EA8C1B6
:106A30008330910509F09CC020915124A0905224EC
:106A40008090532430E040E050E060E070E080E06F
:106A500090E000E10E94A18BF22E132FE42ED52EA0
:106A6000C62EB72E282E992E2A2D30E040E050E079
:106A700060E070E080E090E008E00E94A18B2F0DC4
:106A8000B1E02F1508F0B0E0310FE1E0311708F068
:106A9000E0E0B30FF1E0B31708F0F0E0EF2B4E0D9C
:106AA00031E04E1508F030E0E40FF1E0E41708F0B3
:106AB000F0E03F2B5D0D41E05D1508F040E0A32FB5
:106AC000A50F31E0A51708F030E0432B6C0D31E045
:106AD0006C1508F030E0F42FF60F41E0F61708F0DF
:106AE00040E0342B7B0D41E07B1508F040E0532F54
:106AF000570F31E0571708F030E0432B820D31E09B
:106B0000821508F030E0480F61E0481708F060E0B7
:106B1000362B990D930F022F080D11E0021708F084
:106B200010E01B0F81E01B1708F080E0B82FBE0FAC
:106B300071E0BE1708F070E07A0F61E07A1708F094
:106B400060E06F0F31E06F1708F030E0350F21E0A3
:106B5000351708F020E0240F81E0241708F080E0CA
:106B600018014B2E572E662E732E822E982EFDC0A6
:106B7000843091050CF4FBC020915124A090522444
:106B8000709053248090542430E040E050E060E066
:106B900070E080E090E008E10E94A18BF22E132FBC
:106BA000E42ED52EC62EB72E282E992E2A2D30E073
:106BB00040E050E060E070E080E090E000E10E94A2
:106BC000A18B2F0DF1E02F1508F0F0E0310FE1E07F
:106BD000311708F0E0E0F30FA1E0F31708F0A0E0B0
:106BE000EA2B4E0D31E04E1508F030E0E40FA1E045
:106BF000E41708F0A0E03A2B5D0D41E05D1508F0C8
:106C000040E0B32FB50F31E0B51708F030E0432B6B
:106C10006C0D31E06C1508F030E0A42FA60F41E0B8
:106C2000A61708F040E0342B7B0D41E07B1508F0FF
:106C300040E0532F570F31E0571708F030E0432B57
:106C4000820D31E0821508F030E0480F61E048170E
:106C500008F060E0362B990E930E222E280C81E06E
:106C6000221608F080E0E82EEF0E11E0EF1608F093
:106C700010E01E0F81E01E1708F080E0F82EFB0EDA
:106C800081E0FB1608F080E0D82EDA0E81E0DA16FB
:106C900008F080E0C82EC50E81E0C51608F080E03F
:106CA000B82EB40E81E0B41608F080E0980E272DBF
:106CB00030E040E050E060E070E080E090E008E02C
:106CC0000E94A18B220DE1E0221508F0E0E03E0DCC
:106CD000F1E03E1508F0F0E0E30FA1E0E31708F063
:106CE000A0E0FA2B410F31E0411708F030E0F40F3B
:106CF000A1E0F41708F0A0E03A2B5F0D41E05F152A
:106D000008F040E0A32FA50F31E0A51708F030E010
:106D1000432B6D0D31E06D1508F030E0542F560F08
:106D200041E0561708F040E0342B7C0D41E07C1523
:106D300008F040E0632F670F31E0671708F030E09C
:106D4000432B8B0D31E08B1508F030E0480F71E0DC
:106D5000481708F070E0372B990D222E3E2E4F2E4B
:106D60005A2E652E762E842E932E990E09C01AE087
:106D7000212E3324442455246624772488249924FE
:106D80000E94AD0DB22DB73691F4E32DEF3679F4B4
:106D9000F42DFC3661F4552051F4662041F477203F
:106DA00031F4882021F4992011F40C94EB419101E5
:106DB000A201B301C401B7E6AB2EAFE6BA2EFCE6E2
:106DC000CF2EDD24EE24FF2400E010E00E94838C0F
:106DD000823008F0A4C2822D893689F4932D92372F
:106DE00071F4442061F4552051F4662041F4772079
:106DF00031F4882021F4992011F40C9484449101F9
:106E0000A201B301C401E9E6AE2E02E7B02ECC2404
:106E1000DD24EE24FF2400E010E00E94838C823009
:106E200008F023C1A22DA53681F4B32DB43669F440
:106E3000442059F4552049F4662039F4772029F488
:106E4000882019F4992009F437C79101A201B301F0
:106E5000C40115E6A12EB4E6BB2ECC24DD24EE241D
:106E6000FF2400E010E00E94838C823008F07DC097
:106E7000E22DE53781F4332071F4442061F455208C
:106E800051F4662041F4772031F4882021F49920D0
:106E900011F40C94913F9101A201B301C401A5E743
:106EA000AA2EBB24CC24DD24EE24FF2400E010E035
:106EB0000E94838C823010F5F22DF83611F00C947C
:106EC000AB47332011F00C94AB47442011F00C94E5
:106ED000AB47552011F00C94AB47662011F00C9491
:106EE000AB47772011F00C94AB47882011F00C943D
:106EF000AB47992011F00C94AB4733C7822D8637EE
:106F000081F4332071F4442061F4552051F466205B
:106F100041F4772031F4882021F4992011F40C9465
:106F2000A13F922D943611F00C94AB47A32DA136BE
:106F300011F00C94AB47442011F00C94AB47552052
:106F400011F00C94AB47662011F00C94AB477720FE
:106F500011F00C94AB47882011F00C94AB479920AA
:106F600011F00C94AB470C94F544B22DB73789F46B
:106F7000E32DEF3671F4442061F4552051F466207E
:106F800041F4772031F4882021F4992011F40C94F5
:106F900025439101A201B301C401F7E7AF2EEFE64B
:106FA000BE2ECC24DD24EE24FF2400E010E00E945D
:106FB000838C8230B8F5F22DF43681F4832D893636
:106FC00069F4442059F4552049F4662039F47720B7
:106FD00029F4882019F4992009F482C7922D953656
:106FE00011F00C94AB47A32DAE3611F00C94AB47C7
:106FF000442011F00C94AB47552011F00C94AB4792
:10700000662011F00C94AB47772011F00C94AB473D
:10701000882011F00C94AB47992011F00C94AB47E9
:107020000C944F43B22DB33389F4E32DE13771F45F
:10703000442061F4552051F4662041F4772031F466
:10704000882021F4992011F40C94F544F22DF536A2
:1070500011F00C94AB47832D823711F00C94AB47A1
:10706000442011F00C94AB471EC2922D923689F445
:10707000A32DA53671F4B42DB43659F4552049F436
:10708000662039F4772029F4882019F4992009F42E
:1070900013C69101A201B301C40102E6A02E15E6B8
:1070A000B12EB4E6CB2EDD24EE24FF2400E010E068
:1070B0000E94838C823008F098C0E22DE13389F47D
:1070C000F32DF43671F4842D813659F4552049F4AA
:1070D000662039F4772029F4882019F4992009F4DE
:1070E000FFC39101A201B301C401A1E3AA2EF4E6FA
:1070F000BF2EE1E6CE2EDD24EE24FF2400E010E0DA
:107100000E94838C8230C0F5922D933789F4A32D91
:10711000A23771F4442061F4552051F4662041F403
:10712000772031F4882021F4992011F40C94D7446D
:10713000B22DB33711F00C94AB47E32DE33711F0C8
:107140000C94AB47442011F00C94AB47552011F040
:107150000C94AB47662011F00C94AB47772011F0EC
:107160000C94AB47882011F00C94AB47992011F098
:107170000C94AB470C94E644F22DF33691F4832D36
:10718000843679F4942D913661F4552051F46620BB
:1071900041F4772031F4882021F4992011F40C94E3
:1071A000F544A22DA83711F00C94AB47B32DB4369B
:1071B00011F00C94AB47E42DE13611F00C94AB4781
:1071C000552011F00C94AB47662011F00C94AB479E
:1071D000772011F00C94AB47882011F00C94AB474A
:1071E000992011F00C94AB4777C3F22DFD3691F442
:1071F000832D853779F4942D983661F4552051F418
:10720000662041F4772031F4882021F4992011F48C
:107210000C9406459101A201B301C4010DE6A02E14
:1072200015E7B12EB8E6CB2EDD24EE24FF2400E0D6
:1072300010E00E94838C8230C8F5A22DA23791F411
:10724000B32DB23779F4E42DE53661F4552051F4CD
:10725000662041F4772031F4882021F4992011F43C
:107260000C944842F22DF33611F00C94AB47832D69
:107270008D3611F00C94AB47942D983611F00C9488
:10728000AB47552011F00C94AB47662011F00C94DD
:10729000AB47772011F00C94AB47882011F00C9489
:1072A000AB47992011F00C94AB473EC3A22DA336F7
:1072B00089F4B32DB23371F4E42DE93659F4552035
:1072C00049F4662039F4772029F4882019F49920AC
:1072D00009F426C3F22DF43611F00C94AB47832D3C
:1072E000833611F00C94AB47942D9C3611F00C941E
:1072F000AB47552011F00C94AB47662011F00C946D
:10730000AB47772011F00C94AB47882011F00C9418
:10731000AB47992011F00C94AB470C94E841A22D97
:10732000A63391F4B32DB93679F4E42DE53761F441
:10733000F52DF53649F4662039F4772029F48820B4
:1073400019F4992009F411C59101A201B301C401F6
:10735000A6E3AA2EF9E6BF2EE5E7CE2E05E6D02E4F
:10736000EE24FF2400E010E00E94838C823008F0BD
:107370004CC1822D8C3691F4932D943779F4A42D41
:10738000A43761F4552051F4662041F4772031F49C
:10739000882021F4992011F40C94DC469101A2017B
:1073A000B301C4011CE6A12EB4E7BB2EA4E7CA2E8C
:1073B000DD24EE24FF2400E010E00E94838C823064
:1073C00008F087C0B22DB03391F4E32DE13379F4A6
:1073D000F42DF13761F4552051F4662041F4772003
:1073E00031F4882021F4992011F40C944842910141
:1073F000A201B301C401F0E3AF2EE1E3BE2E01E729
:10740000C02EDD24EE24FF2400E010E00E94838CD7
:10741000823028F5822D853711F00C94AB47932DDF
:10742000933611F00C94AB47A42DAD3611F00C94AB
:10743000AB47552011F00C94AB47662011F00C942B
:10744000AB47772011F00C94AB47882011F00C94D7
:10745000AB47992011F00C94AB470C94AB42B22D82
:10746000B13391F4E32DE13379F4F42DF13761F484
:10747000552051F4662041F4772031F4882021F41E
:10748000992011F40C94AB42822D803711F00C94AA
:10749000AB47932D953611F00C94AB47A42DA23732
:1074A00011F00C94AB47552011F00C94AB476620BB
:1074B00011F00C94AB47772011F00C94AB47882067
:1074C00011F00C94AB47992011F00C94AB470C943D
:1074D0002344B22DB43791F4E32DEF3679F4F42D33
:1074E000FF3661F4852D823649F4662039F4772021
:1074F00029F4882019F4992009F484C59101A20186
:10750000B301C40114E7A12EBFE6BB2EAFE6CA2E1D
:10751000F2E6DF2EEE24FF2400E010E00E94838CD0
:107520008230C8F5922D943789F4A32DA83771F4D1
:10753000B42DB43759F4552049F4662039F4772036
:1075400029F4882019F4992009F45FC5E22DE43765
:1075500011F00C94AB47F32DF43611F00C94AB47BB
:10756000842D873711F00C94AB47552011F00C9403
:10757000AB47662011F00C94AB47772011F00C94C8
:10758000AB47882011F00C94AB47992011F00C9474
:10759000AB470C943C47922D993691F4A32DAC3611
:1075A00079F4B42DB13661F4E52DE33649F4662063
:1075B00039F4772029F4882019F4992009F4E0C1DE
:1075C000F22DFE3611F00C94AB47832D813611F06D
:1075D0000C94AB47942D983611F00C94AB47A52D25
:1075E000A33611F00C94AB47662011F00C94AB4716
:1075F000772011F00C94AB47882011F00C94AB4726
:10760000992011F00C94AB47D2C4B22DB13691F44D
:10761000E32DEC3679F4F42DF53661F4852D8237BF
:1076200049F4662039F4772029F4882019F4992048
:1076300009F4B2C39101A201B301C401E1E6AE2E87
:107640000CE6B02E15E6C12EB2E7DB2EEE24FF24A9
:1076500000E010E00E94838C823008F09FC0922DE1
:10766000923791F4A32DA73779F4B42DB03761F494
:10767000E52DE03749F4662039F4772029F4882095
:1076800019F4992009F454C19101A201B301C40174
:10769000A2E7AA2EF7E7BF2EE0E7CE2E00E7D02E16
:1076A000EE24FF2400E010E00E94838C8230D0F5AD
:1076B000F22DF03791F4832D8C3679F4942D953694
:1076C00061F4A52DA83649F4662039F4772029F411
:1076D000882019F4992009F444C3B22DB13611F071
:1076E0000C94AB47E32DED3611F00C94AB47F42D21
:1076F000F53711F00C94AB47852D883611F00C94BA
:10770000AB47662011F00C94AB47772011F00C9436
:10771000AB47882011F00C94AB47992011F00C94E2
:10772000AB47ACC7922D933799F4A32DA53681F4BE
:10773000B42DB23769F4E52DE03751F4662041F4F9
:10774000772031F4882021F4992011F40C94F84525
:10775000F22DF33711F00C94AB47832D823711F0E3
:107760000C94AB47942D973711F00C94AB47A52D93
:10777000A03711F00C94AB47662011F00C94AB4786
:10778000772011F00C94AB47882011F00C94AB4794
:10779000992011F00C94AB470C94EF43B22DB737FE
:1077A00091F4E32DE03779F4F42DF83761F4852D69
:1077B000843749F4662039F4772029F4882019F4B5
:1077C000992009F4CEC39101A201B301C40117E7C6
:1077D000A12EB0E7BB2EA8E7CA2EF4E7DF2EEE24D9
:1077E000FF2400E010E00E94838C8230D0F5922DBF
:1077F000943791F4A32DA33779F4B42DB53661F401
:10780000E52DE23749F4662039F4772029F4882001
:1078100019F4992009F4E0C7F22DF43711F00C9413
:10782000AB47832D833711F00C94AB47942D9536DD
:1078300011F00C94AB47A52DA43711F00C94AB4775
:10784000662011F00C94AB47772011F00C94AB47F5
:10785000882011F00C94AB47992011F00C94AB47A1
:10786000FBC3B22DB23791F4E32DE73679F4F42D52
:10787000F03761F4852D853749F4662039F4772097
:1078800029F4882019F4992009F471C5922D9C36A9
:1078900011F00C94AB47A32DA13611F00C94AB471B
:1078A000B42DB43711F00C94AB47E52DE83711F047
:1078B0000C94AB47662011F00C94AB47772011F085
:1078C0000C94AB47882011F00C94AB47992011F031
:1078D0000C94AB470C94A1460E94EA170C94AD4758
:1078E00080ED61E04CE021E00E94E76580ED61E021
:1078F0004EE021E00E94E76580ED61E040E121E09B
:107900000E94E76580ED61E042E121E00E94E765C9
:1079100080ED61E040E122E00E94E7650C94AD4714
:107920000E9400120C94AD470E9473180C94AD474E
:107930006091D7067091D80680E090E00E94E5A0A3
:107940008C016FE574E00E94FAA0009719F4779813
:107950000C94AD47C80162E674E00E94FAA000975B
:1079600019F4779A0C94AD47779903C08FE594E0AA
:1079700002C082E694E000D000D021ED33E07DC566
:107980006091D7067091D80680E090E00E94E5A053
:107990008C0167E274E00E94FAA0009709F052C0DF
:1079A0006091D7067091D80680E090E00E94E5A033
:1079B0008C01009711F40C94AD4766E674E00E94C8
:1079C000FAA0009729F482E29FEFACECBBE30BC076
:1079D000C8016CE674E00E94FAA0009789F482E284
:1079E0009FEFACECBAE38093C9069093CA06A093CC
:1079F000CB06B093CC0689EC96E066E070E0DCC084
:107A0000C8010E94CF9F7B018C0120E030E0A901DA
:107A10000E940A99882391F081E00E944E0C9B01FC
:107A2000AC01C801B7010E940E996093C90670931A
:107A3000CA068093CB069093CC06DDCF00D081E1BF
:107A400094E08CC0C8016AE274E00E94FAA000973A
:107A500009F052C06091D7067091D80680E090E09E
:107A60000E94E5A08C01009711F40C94AD4766E6E6
:107A700074E00E94FAA0009729F482E29FEFACEC38
:107A8000BBE30BC0C8016CE674E00E94FAA000974B
:107A900069F482E29FEFACECBAE38093CD06909359
:107AA000CE06A093CF06B093D0061DC0C8010E9499
:107AB000CF9F7B018C0120E030E0A9010E940A9950
:107AC0008823B1F082E00E944E0C9B01AC01C801FA
:107AD000B7010E940E996093CD067093CE068093F5
:107AE000CF069093D0068DEC96E06AE070E064C01B
:107AF00000D084E094E067C0C80162E274E00E94B4
:107B0000FAA0009709F06BC06091D7067091D80673
:107B100080E090E00E94E5A08C01009711F40C94A5
:107B2000AD4766E674E00E94FAA0009769F487ED1D
:107B300094E3AFEEBCE38093C5069093C606A09392
:107B4000C706B093C80634C0C8016CE674E00E9452
:107B5000FAA0009741F400D085EF93E0EDB7FEB7AF
:107B60009283818336C0C8010E94CF9F7B018C0124
:107B700020E030E0A9010E940A99882309F180E001
:107B80000E944E0C1B012C01C801B70121EE3AE7FF
:107B900044E95EE30E944398A20191010E940E997C
:107BA0006093C5067093C6068093C7069093C80677
:107BB00085EC96E062E070E044E050E00C947F4792
:107BC00000D088EE93E0ADB7BEB712969C938E932B
:107BD00011970E948AA10F900F900C94AD470E94BC
:107BE0009C0C00D000D000D021EE33E0EDB7FEB702
:107BF00032832183ADB7BEB713966D937D938D937A
:107C00009C9316970E948AA1EDB7FEB736960FB6E1
:107C1000F894FEBF0FBEEDBF81E00E944E0C209194
:107C2000C9063091CA064091CB065091CC060E94FD
:107C3000BC9B7B018C0182E00E944E0C9B01AC013D
:107C40008DB79EB70A970FB6F8949EBF0FBE8DBF33
:107C5000CDB6DEB60894C11CD11C85ED93E0ADB75E
:107C6000BEB712969C938E9311978E2D9F2DA02FA9
:107C7000B12FF60182839383A483B583CA01B9012E
:107C80002091CD063091CE064091CF065091D0067E
:107C90000E94BC9BD60116966D937D938D939C9309
:107CA00019970E948AA1EDB7FEB73A960FB6F894DD
:107CB000FEBF0FBEEDBF51C06091D7067091D806D0
:107CC00080E090E00E94E5A00097F9F00E94962ED7
:107CD0002091080A3091090A8217930759F190936D
:107CE000090A8093080A88E09AE060E070E042E0C8
:107CF00050E00E94D3A200D08AEC93E0ADB7BEB7AB
:107D000012969C938E93119707C000D083EC93E05A
:107D1000EDB7FEB7928381830E948AA16091080A21
:107D20007091090A0F900F9080E090E00E94DA2D88
:107D30000E94AD0D00D088EB93E0ADB7BEB71296B0
:107D40009C938E9311970E948AA10F900F906FEFD2
:107D50007FEF80E090E00E94DA2D0E94AD0D0C9440
:107D6000AD470E948E290C94AD47809155248433F1
:107D700029F480E061E040E00E948F132091D10659
:107D8000222311F40C94AD4700D000D0EDB7FEB71C
:107D9000319685EB93E09AC080915524893709F09C
:107DA00088C06091D7067091D80680E090E00E946C
:107DB000E5A08C016FE574E00E94FAA0009731F411
:107DC0008091EF069091F00690640CC0C80162E6C5
:107DD00074E00E94FAA0009791F48091EF069091D0
:107DE000F0069F7B9093F0068093EF068FEE96E06F
:107DF00064E170E042E050E00E94D3A25AC0C801A2
:107E000061E774E00E94FAA00097A1F5EDB7FEB714
:107E10003A970FB6F894FEBF0FBEEDBF319682E2DF
:107E200094E0ADB7BEB712969C938E931197809154
:107E30006D1B90916E1B9383828380916F1B909139
:107E4000701B958384838091711B9091721B978323
:107E500086838091731B9091741B918780870E9409
:107E60008AA1EDB7FEB73A960FB6F894FEBF0FBEE3
:107E7000EDBF1FC08091EF069091F00696FF03C002
:107E80008FE594E002C082E694E000D000D02EE1BD
:107E900034E0ADB7BEB712963C932E93119714966B
:107EA0009C938E9313970E948AA10F900F900F902E
:107EB0000F902091D106222311F40C94AD4700D0ED
:107EC00000D0EDB7FEB7319682EB93E0ADB7BEB709
:107ED00012969C938E931197228313820C94A4473D
:107EE0006091D7067091D80680E090E00E94E5A0EE
:107EF00066E674E00E94FAA0009711F481E001C0E8
:107F000080E00E94D22C2091D106222311F40C94FF
:107F1000AD4700D000D0EDB7FEB731968FEA93E0C1
:107F2000D5CF0E948D2A2091D106222311F40C94E2
:107F3000AD4700D000D0EDB7FEB731968CEA93E0A4
:107F4000C5CF0E94882A2091D106222311F40C94D7
:107F5000AD4700D000D0EDB7FEB7319689EA93E087
:107F6000B5CF6091D7067091D80680E090E00E946E
:107F7000E5A00E94D39F803150F480930D0A90E0D9
:107F80000E94E36F8DE09AE066E170E027C000D0C8
:107F900000D0EDB7FEB731968DE494E0ADB7BEB733
:107FA00012969C938E93119780910D0A29C060912F
:107FB000D7067091D80680E090E00E94E5A00E946C
:107FC000D39F982F9B50903160F48093F10690E0FE
:107FD0000E945B6E81EF96E067E170E041E050E067
:107FE0008EC700D000D0EDB7FEB7319687E594E09C
:107FF000ADB7BEB712969C938E9311978091F10600
:1080000082836BCF0C940000A8C76091D706709153
:10801000D80680E090E00E94E5A0BC01009769F0DE
:1080200088E59BE14AE050E00E9403A188E59BE1DE
:1080300062E270E04AE050E062C700D000D087E71B
:1080400094E0EDB7FEB79283818388E59BE194834A
:1080500083830E9478A17AC76091D7067091D80671
:1080600080E090E00E94E5A08C016FE774E00E9440
:10807000FAA0009739F4219A8091EF069091F006CA
:10808000806133C7C80161E874E00E94FAA00097DC
:1080900039F4229A8091EF069091F006806225C70C
:1080A000C80163E874E00E94FAA0009739F4239AAB
:1080B0008091EF069091F006806417C7C80165E8CB
:1080C00074E00E94FAA0009739F4239A8091EF0699
:1080D0009091F006806809C7C80167E874E00E94C3
:1080E000FAA0009781F581E080934A248091E90607
:1080F0009091EA06A091EB06B091EC0680934B2498
:1081000090934C24A0934D24B0934E24109250246D
:1081100010924F248091EF069091F0069160909319
:10812000F0068093EF068FEE96E064E170E042E0A7
:1081300050E00E94D3A283E397E062E14AE454E274
:108140000E948B580AC7C80169E874E00E94FAA02F
:10815000009771F4E5E7FBE1119211928BE1E539AB
:10816000F807D1F78091EF069091F0069260BDC6B6
:10817000C80162E674E00E94FAA09C018091EF06BB
:108180009091F00621153105A9F48F709C7F909392
:10819000F0068093EF062B9A8FEE96E064E170E094
:1081A00042E050E00E94D3A280919D2890E00E947E
:1081B000706ED3C684FF03C08FE594E002C082E6F0
:1081C00094E000D000D027E934E0ADB7BEB71296F6
:1081D0003C932E93119714969C938E9313970E9421
:1081E0008AA18091EF060F900F900F900F9085FF5E
:1081F00003C08FE594E002C082E694E000D000D096
:108200002CE834E0EDB7FEB7328321839483838377
:108210000E948AA18091EF060F900F900F900F900F
:1082200086FF03C08FE594E002C082E694E000D0B0
:1082300000D021E834E0ADB7BEB712963C932E9340
:10824000119714969C938E9313970E948AA1809104
:10825000EF060F900F900F900F9087FF03C08FE5F0
:1082600094E002C082E694E000D000D026E734E03B
:10827000EDB7FEB732832183948383830E948AA162
:108280008091EF069091F0060F900F900F900F9055
:1082900090FF03C08FE594E002C082E694E000D036
:1082A00000D02BE634E0ADB7BEB712963C932E93C8
:1082B000119714969C938E9313970E948AA1809194
:1082C000EF069091F0060F900F900F900F9091FF96
:1082D00003C08FE594E002C082E694E000D000D0B5
:1082E00020E634E0EDB7FEB73283218394838383A5
:1082F0000E948AA18091EF069091F0060F900F9056
:108300000F900F9091FF29C68BE894E00E94AAA1DC
:1083100005E71BE1EBE0CE2ED12C73E9E72E74E0EC
:10832000F72ED8018D919D918D0100D000D000D005
:10833000EDB7FEB73196ADB7BEB71296FC92EE928E
:108340001197D382C282958384830E9478A1089476
:10835000C11CD11CEDB7FEB736960FB6F894FEBF20
:108360000FBEEDBFFBE1CF16D104D9F6F6C500D0A4
:1083700085EA93E0ADB7BEB712969C938E931197A2
:108380000E948AA12091D1060F900F902223A9F07C
:1083900000D000D0EDB7FEB7319682EA93E0ADB7DA
:1083A000BEB712969C938E931197228313820E94DC
:1083B0008AA10F900F900F900F9088E10FB6F8945C
:1083C00080936000109260000FBE0C94007CC5C5C5
:1083D0000E949D65C2C56091D7067091D80680E065
:1083E00090E00E94E5A07C016FE574E00E94FAA095
:1083F000009749F40E943A6D8091EF069091F00643
:1084000081608D7F72C5C70162E674E00E94FAA0A8
:10841000009741F40E949C6C8091EF069091F006C9
:108420008C7F63C50EE914E0C701B8010E94FAA071
:10843000009749F40E949C6C8091EF069091F006A1
:108440008E7F826052C58091EF0681FF0BC000D005
:1084500000D086EA94E0EDB7FEB79283818314835F
:10846000038372C580FF03C08FE594E002C082E6FB
:1084700094E000D000D022EA34E0ADB7BEB7129647
:108480003C932E93119714969C938E9313975CC5EF
:1084900000D088E793E0EDB7FEB7928381830E9416
:1084A0008AA18DB79EB740970FB6F8949EBF0FBEB6
:1084B0008DBFEDB7FEB731968AE593E0ADB7BEB795
:1084C00012969C938E931197809145249091462407
:1084D000A0914724B091482482839383A483B583D9
:1084E0008091392490913A24A0913B24B0913C246E
:1084F00086839783A087B18780913D2490913E2405
:10850000A0913F24B091402482879387A487B587A8
:108510008091412490914224A0914324B09144241D
:1085200086879787A08BB18B0E948AA12091D10664
:10853000EDB7FEB772960FB6F894FEBF0FBEEDBF53
:10854000222309F40AC500D000D0EDB7FEB731965A
:1085500087E593E0BBCCF89481E090E00E94880826
:10856000182F80E090E00E948808082F7894F894F3
:1085700083E090E00E948808F82E82E090E00E945C
:108580008808E82E789400D000D000D02DE433E0A5
:10859000EDB7FEB7328321832091E61B3091E71BB4
:1085A0004091E81B5091E91BADB7BEB713962D93D0
:1085B0003D934D935C9316970E948AA100D000D002
:1085C000EDB7FEB7319626E233E0ADB7BEB71296EF
:1085D0003C932E931197E2821382F48215820683D4
:1085E0001782108711860E948AA1EDB7FEB73A96CE
:1085F0000FB6F894FEBF0FBEEDBF0E94302B209146
:10860000660000D000D0EDB7FEB731968AE193E066
:10861000ADB7BEB712969C938E93119722831382A7
:108620000E948AA10F900F900F900F900E94AD0DA5
:108630002091D106222309F490C400D000D0EDB7D8
:10864000FEB7319687E193E041CC80E090E060E0B6
:1086500070E00E94B90D81E090E060E070E00E945F
:10866000B90D2091D106222309F477C400D000D09F
:10867000EDB7FEB7319684E193E028CC0E94FD2847
:108680000E94AD0D2091D106222309F466C400D0CA
:1086900000D0EDB7FEB7319681E193E017CC609141
:1086A000D7067091D80680E090E00E94E5A063EACA
:1086B00074E00E94FAA0009741F5F8948DE29AE0E8
:1086C0000E9482590CC0C8010F960E94CE5C80E8BF
:1086D00097E0B8010E943C59C8010E94485A082FEF
:1086E000192F0115110579F704C08DE29AE00E9457
:1086F000C3598DE29AE00E94285A0097B1F78DE2A3
:108700009AE00E947E5978945AC08DE29AE00E94C5
:108710008259482F592F7A0109EA14E04CC0EDB76D
:10872000FEB774970FB6F894FEBF0FBEEDBF31963B
:10873000ADB7BEB712961C930E931197D7011A9638
:108740008C911A978283138212968C91129784834C
:10875000158213968C9113978683178214968C91A9
:1087600014978087118617968C91179782871386A6
:1087700019968C9119978487158615968C91159763
:108780008687178618968C911897808B118A169673
:108790008C91828B138A0E9478A1EDB7FEB77496F4
:1087A0000FB6F894FEBF0FBEEDBFC7010E94485A36
:1087B000482F592F7A01E114F10409F0B0CF20912C
:1087C000D106222309F4C9C300D000D0EDB7FEB70B
:1087D00031968EE093E07ACB0E940C2DBEC360915F
:1087E000D7067091D80680E090E00E94E5A08C0149
:1087F00068EE74E00E94FAA0009731F48091EF06D1
:108800009091F006937F71C3C8016CE674E00E94FA
:10881000FAA0009739F48091EF069091F006937FCB
:10882000986063C3C8016DEE74E00E94FAA00097DF
:1088300039F48091EF069091F006937F946055C3D0
:108840000E948F088AC36091D7067091D80680E095
:1088500090E00E94E5A0009751F10E949A3020918B
:10886000E9063091EA064091EB065091EC0662175A
:1088700073078407950739F16093E9067093EA0658
:108880008093EB069093EC0689EE96E06EE070E044
:1088900044E050E00E94D3A200D086E093E0EDB720
:1088A000FEB7928381830E948AA10F900F906091FE
:1088B000E9067091EA068091EB069091EC060E9421
:1088C0002D2F0E94AD0D00D08AEF92E0ADB7BEB75C
:1088D00012969C938E9311970E948AA10F900F90ED
:1088E0006FEF7FEFCB010E942D2F0E94AD0D2091E5
:1088F000D106222309F431C300D000D0EDB7FEB772
:10890000319687EF92E0E2CA6091D7067091D8065F
:1089100080E090E00E94E5A0009741F160E070E007
:108920004AE050E00E94C19E7093EE066093ED060F
:1089300000D000D0EDB7FEB731962AED32E0ADB7EA
:10894000BEB712963C932E931197738362830E9455
:108950008AA10F900F900F900F908DEE96E062E13C
:1089600070E042E050E00E94D3A214C000D000D0DA
:1089700089EB92E0EDB7FEB7928381838091ED069B
:108980009091EE06948383830E948AA10F900F90AA
:108990000F900F902091D106222309F4DEC200D05F
:1089A00000D0EDB7FEB7319686EB92E08FCA0E94F9
:1089B0000B5D2091D106222309F4CFC200D000D054
:1089C000EDB7FEB7319683EB92E080CA0E94C132C8
:1089D0002091D106222309F4C0C200D000D0EDB707
:1089E000FEB7319680EB92E071CA80E090E00E9481
:1089F000552B2091D106222309F4AFC200D000D01C
:108A0000EDB7FEB731968DEA92E060CA80913320CF
:108A100081FF3BC00E9442280097B9F500D000D0EA
:108A200000D082EA92E0EDB7FEB792838183809115
:108A30002F1C9091301CA091311CB091321C83836B
:108A40009483A583B6830E948AA185E992E0ADB79D
:108A5000BEB712969C938E9311978091B2289091F5
:108A6000B328A091B428B091B528EDB7FEB78383A1
:108A70009483A583B6830E948AA18DB79EB706967C
:108A80000FB6F8949EBF0FBE8DBF0E94AD0D8091B2
:108A900033209091342090FF9CC081E090E00E94B0
:108AA000EF271B012C0180E090E00E94EF277B0163
:108AB0008C010E945F2700D000D000D084E892E0B3
:108AC000ADB7BEB712969C938E931197EDB7FEB7D4
:108AD00023823482458256820E948AA184E792E0F2
:108AE000ADB7BEB712969C938E931197EDB7FEB7B4
:108AF000E382F482058316830E948AA18DB79EB714
:108B000006960FB6F8949EBF0FBE8DBFC201B1018D
:108B1000A80197010E94422600D000D000D029E68B
:108B200032E0ADB7BEB712963C932E931197EDB7D6
:108B3000FEB763837483858396830E948AA18DB771
:108B40009EB706960FB6F8949EBF0FBE8DBFC201AA
:108B5000B101A80197010E94A32600D000D000D047
:108B60002BE532E0ADB7BEB712963C932E9311972A
:108B7000EDB7FEB763837483858396830E948AA1D1
:108B80008DB79EB706960FB6F8949EBF0FBE8DBFE9
:108B9000C201B101A80197010E94082700D000D0AE
:108BA00000D028E432E0ADB7BEB712963C932E93C6
:108BB0001197EDB7FEB763837483858396830E9414
:108BC0008AA18DB79EB706960FB6F8949EBF0FBECA
:108BD0008DBF0E94AD0D2091D106222309F4BDC1A5
:108BE00000D000D0EDB7FEB7319685E492E06EC9B3
:108BF0008091332082FF3BC083E061E048E021E0C8
:108C00000E942915EDB7FEB73A970FB6F894FEBF4C
:108C10000FBEEDBF31968EE292E0ADB7BEB71296B1
:108C20009C938E9311978091261C9091271CA09164
:108C3000281CB091291C82839383A483B5838091DF
:108C40002A1C90912B1CA0912C1CB0912D1C86836A
:108C50009783A087B1870E948AA1EDB7FEB73A96A5
:108C60000FB6F894FEBF0FBEEDBF0E94AD0D809110
:108C700033209091342091FF57C00E94111A7B013C
:108C80008C0120E030E048EC52E40E94BC9B20E8DC
:108C900036EE45EC57E40E940E9921E03EED42E4A9
:108CA0005EE30E941F9C6B01582F492F8DB79EB722
:108CB0000A970FB6F8949EBF0FBE8DBFADB6BEB675
:108CC0000894A11CB11C25E132E0ADB7BEB71296E5
:108CD0003C932E931197F501E282F382048315836E
:108CE00060E070E080E89FE3FA012C2D3D2D4F2FCE
:108CF0005E2F0E9443982BE43AE34DEB57E30E942A
:108D00000E99D50116966D937D938D939C9319972B
:108D10000E948AA1EDB7FEB73A960FB6F894FEBF4F
:108D20000FBEEDBF0E94AD0D2091D106222309F4A4
:108D300014C100D000D0EDB7FEB7319682E192E0C9
:108D4000C5C86091D7067091D80680E090E00E9477
:108D5000E5A068EF74E00E94FAA00097B1F460917A
:108D6000D7067091D80680E090E00E94E5A00097B9
:108D700009F4F3C00E94D39F803108F0EEC09091B7
:108D80005201982B90935201E8C08091520100D07B
:108D900000D028EC34E0EDB7FEB73283218390E0B9
:108DA0008F709070948383830E948AA10F900F909C
:108DB0000F900F900C94AD3E6091D7067091D8063D
:108DC00080E090E00E94E5A0009781F160E070E013
:108DD0004AE050E00E94949D603100F56093F206F5
:108DE00000D000D0EDB7FEB7319685E092E0ADB788
:108DF000BEB712969C938E931197628313820E9442
:108E00008AA10F900F900F900F9082EF96E068E18B
:108E100070E041E050E00E94D3A21FC000D000D01B
:108E2000EDB7FEB731968CEF91E007C000D000D0CF
:108E3000EDB7FEB7319683EF91E0ADB7BEB71296AE
:108E40009C938E9311978091F206828313820E94E5
:108E50008AA10F900F900F900F900E94AD0D20915E
:108E6000D106222309F479C000D000D0EDB7FEB7B7
:108E7000319680EF91E02AC86091D7067091D806AC
:108E800080E090E00E94E5A08C016FE574E00E9414
:108E9000FAA0009741F40E947E6B8091EF069091BA
:108EA000F006906122C0C80162E674E00E94FAA058
:108EB000009741F5F8940E948C6B88E10FB6F89406
:108EC00080936000109260000FBE84B7877F84BFDC
:108ED00080916000886180936000109260007894B7
:108EE0008091EF069091F0069F7E9093F00680931C
:108EF000EF068FEE96E064E170E042E050E00E9401
:108F0000D3A22BC0C8016DEF74E00E94FAA09C01AF
:108F10008091EF069091F0062115310521F494FF20
:108F20001CC0F894FFCF94FF03C08FE594E002C00B
:108F300082E694E000D000D025ED34E0EDB7FEB736
:108F400032832183948383830E948AA10F900F90A0
:108F50000F900F9002C00E946729A981BA811196D3
:108F60001C921E9283E00F900F90CF91DF911F9182
:108F70000F91FF90EF90DF90CF90BF90AF909F90B8
:108F80008F907F906F905F904F903F902F900895BB
:108F9000F89491E2E0E0F0E0909357008491E2E0F1
:108FA000F0E0909357002491E4E0F0E090935700B4
:108FB000E49190E0A0E0B0E0DC019927882730E060
:108FC00040E050E0542F432F322F2227820F931F6F
:108FD000A41FB51F8E0F911DA11DB11D8093E61B0F
:108FE0009093E71BA093E81BB093E91B7894089536
:108FF000DF93CF93CDB7DEB761970FB6F894DEBF9E
:109000000FBECDBFCE0104966EE070E044E050E0AC
:109010000E94B5A28C819D81AE81BF818F3F2FEFD1
:1090200092072FEFA2072FEFB20749F489EE96E0DF
:109030006EE070E044E050E00E94D3A208C080934C
:10904000E9069093EA06A093EB06B093EC06CE01F6
:10905000029662E170E042E050E00E94B5A28A818F
:109060009B812FEF8F3F920779F48CE390E09093F0
:10907000EE068093ED068DEE96E062E170E042E050
:1090800050E00E94D3A204C09093EE068093ED06B8
:10909000CE01029664E170E042E050E00E94B5A289
:1090A0008A819B812FEF8F3F920779F48AE090E4C9
:1090B0009093F0068093EF068FEE96E064E170E007
:1090C00042E050E00E94D3A204C09093F006809347
:1090D000EF06CE01029660E070E042E050E00E94B0
:1090E000B5A28A819B812FEF8F3F920769F410927E
:1090F000090A1092080A88E09AE060E070E042E015
:1091000050E00E94D3A204C09093090A8093080AF9
:1091100086EA98E269E170E049E050E00E94B5A279
:109120000E94630FCE01049666E070E044E050E0D8
:109130000E94B5A28C819D81AE81BF818F3F2FEFB0
:1091400092072FEFA2072FEFB20749F489EC96E0C0
:1091500066E070E044E050E00E94D3A208C089ECD1
:1091600096E066E070E044E050E00E94B5A2CE01D7
:1091700004966AE070E044E050E00E94B5A28C8161
:109180009D81AE81BF818F3F2FEF92072FEFA20706
:109190002FEFB20749F48DEC96E06AE070E044E00E
:1091A00050E00E94D3A208C08DEC96E06AE070E027
:1091B00044E050E00E94B5A2CE01049662E070E067
:1091C00044E050E00E94B5A28C819D81AE81BF81B8
:1091D0008F3F2FEF92072FEFA2072FEFB20749F42F
:1091E00085EC96E062E070E044E050E00E94D3A29B
:1091F00008C085EC96E062E070E044E050E00E9438
:10920000B5A2CE01019666E170E041E050E00E9417
:10921000B5A289818F3F49F48DE09AE066E170E064
:1092200041E050E00E94D3A208C08DE09AE066E1E0
:1092300070E041E050E00E94B5A2CE01019667E1E6
:1092400070E041E050E00E94B5A289818F3F49F46F
:1092500081EF96E067E170E041E050E00E94D3A228
:1092600008C081EF96E067E170E041E050E00E94C5
:10927000B5A2CE01019668E170E041E050E00E94A5
:10928000B5A289818F3F49F482EF96E068E170E0F2
:1092900041E050E00E94D3A208C082EF96E068E16E
:1092A00070E041E050E00E94B5A2CE01089662E273
:1092B00070E04AE050E00E94B5A288858F3F49F4F3
:1092C00088E59BE162E270E04AE050E00E94D3A2B0
:1092D00008C088E59BE162E270E04AE050E00E944D
:1092E000B5A261960FB6F894DEBF0FBECDBFCF9189
:1092F000DF9108950E94726B6C9A6B9A6A9A6F9ACA
:10930000729A749A739A779A809880B3897F80BB97
:109310008398849887E080937E00549A0E94C8477F
:109320000E94F84781E00E94C20B80E090E00E941A
:10933000770F0E940B648091EF0686FD239A0895B3
:10934000CF93DF93EC0188819981009731F02EE073
:109350008B34920709F099C08FC00E947A4980919E
:10936000EF0680FD06C081FF02C01D9902C00E9469
:109370009C6C809170008C7F809370008091B6000F
:1093800080628093B6001092B20082E08093B100B8
:109390008091B60090E0877090700097C9F7809137
:1093A000700081608093700080E090E066EB78E070
:1093B0000E94556B0E94882A80E00E94D22C00D027
:1093C0008AEE91E0ADB7BEB712969C938E9311973B
:1093D0000E948AA10F900F900E940012809133206A
:1093E00086FF02C00E94486580910D0A90E00E94AD
:1093F000E36F8091F10690E00E945B6E0E94586ED0
:1094000080933B0A8091F10690E00E945B6E00D051
:1094100000D000D0EDB7FEB7319682E095E0ADB751
:10942000BEB712969C938E93119780913B0A8283CC
:10943000138280910D0A848315820E9478A1109274
:109440003A0A1092390AEDB7FEB736960FB6F8947D
:10945000FEBF0FBEEDBF8FEF96E09093B0288093D4
:10946000AF2883E290E09093320A8093310A8BE434
:109470009EE0998388830DC0633259F489E39AE0B2
:1094800060E070E00E94BC34E6CF1982188283E06D
:1094900001C081E0DF91CF9108958436910534F1C8
:1094A00000D000D024E135E0EDB7FEB73283218350
:1094B000948383830E9478A18091452490914624CF
:1094C000A0914724B09148240196A11DB11D80931D
:1094D000452490934624A0934724B09348240F90AA
:1094E0000F900F900F9021E030E002C020E030E0BC
:1094F000C90108952F923F924F925F926F927F928F
:109500008F929F92AF92BF92CF92DF92EF92FF9293
:109510000F931F93DF93CF93CDB7DEB7C35AD040DD
:109520000FB6F894DEBF0FBECDBFC457DF4F99838F
:109530008883CC58D040633871F489E19AE0CD55E6
:10954000DF4F6883C35AD0400E94C256CD55DF4FCB
:109550006881C35AD040C457DF4FA881B981CC5825
:10956000D0402D913C911197BDE02E3F3B0711F467
:109570000C94CE55EDE02F3F3E0750F421153105F8
:10958000A9F0FCE02F383F0711F00C9425561AC0C3
:109590004EE02F30340711F40C94F7555EE026317D
:1095A000350711F00C9425560C94145689E19AE075
:1095B00061E870E04CE757E00E94A7568FE89CE016
:1095C0000C94C455623111F00C9430568091EF0622
:1095D0009091F00691FDF2CF80914A24813079F488
:1095E000C0904B24D0904C24E0904D24F0904E2419
:1095F000C657DF4F19821882CA58D04014C0823033
:10960000E9F6C0904B24D0904C24E0904D24F0908B
:109610004E24E0914F24F0915024C657DF4FF98338
:10962000E883CA58D040A70196012070307041707D
:109630005070CE56DF4F288339834A835B83C259EB
:10964000D040E0FC8C9AC701B6010E94D30CD70130
:10965000C60180709071A070B070CA56DF4F8883C9
:109660009983AA83BB83C659D040D4FE02C00E940E
:109670004228A70196012070307240705070C65683
:10968000DF4F288339834A835B83CA59D040D5FE94
:109690000AC00E949C0C6093992870939A2880932A
:1096A0009B2890939C28C601817090700097A9F127
:1096B0004DB75EB7485050400FB6F8945EBF0FBE2E
:1096C0004DBFEDB7FEB73196CE014396ADB7BEB7ED
:1096D00012969C938E93119787E790E093838283F1
:1096E00088E295E09583848388E59BE19783868370
:1096F0000E94E1A1A82E092FEDB7FEB738960FB64C
:10970000F894FEBF0FBEEDBF0E944D4A009709F0CE
:1097100055CF802F0A2D182F02C000E010E0C1FEA7
:109720005FC063E1862E912C8C0E9D1E00D000D070
:1097300000D0EDB7FEB73196C401800F911FADB7D1
:10974000BEB712969C938E93119787E790E0938310
:10975000828380E395E0958384830E94E1A1080FD2
:10976000191F56EAA52E58E2B52EEDB7FEB736966C
:109770000FB6F894FEBF0FBEEDBF47E7642E712C05
:1097800037EE432E32E0532ED5012D915D01EDB71A
:10979000FEB738970FB6F894FEBF0FBEEDBF3196F7
:1097A000C401800F911FADB7BEB712969C938E93E4
:1097B00011977382628255824482268317820E94A7
:1097C000E1A1080F191FEDB7FEB738960FB6F89450
:1097D000FEBF0FBEEDBFFEEAAF16F8E2BF06A1F670
:1097E000C2FE6EC023E1822E912C8C0E9D1E00D0F5
:1097F00000D000D0EDB7FEB73196C401800F911FA5
:10980000ADB7BEB712969C938E93119787E790E001
:109810009383828384E395E0958384830E94E1A10E
:10982000080F191F5E010894A11CB11C80E1F5010D
:1098300011928A95E9F72DB73EB72A5F3F4F0FB6D1
:10984000F8943EBF0FBE2DBF80EB68E9A50128E06C
:109850000E94471399E0692E712C6C0E7D1E87E7DC
:10986000482E512CB7EE2B2EB2E03B2ED5012D9178
:109870005D01EDB7FEB738970FB6F894FEBF0FBE87
:10988000EDBF3196C401800F911FADB7BEB71296E0
:109890009C938E9311975382428235822482268331
:1098A00017820E94E1A1080F191FEDB7FEB7389685
:1098B0000FB6F894FEBF0FBEEDBFA614B704B1F605
:1098C000A70196012070307040705072C256DF4F71
:1098D000288339834A835B83CE59D040F5FC30C05E
:1098E0004DB75EB7485050400FB6F8945EBF0FBEFC
:1098F0004DBFEDB7FEB73196CE014396800F911F55
:10990000ADB7BEB712969C938E93119787E790E000
:109910009383828389E395E09583848380910B0A06
:1099200090910C0A978386830E94E1A1080F191F6A
:10993000EDB7FEB738960FB6F894FEBF0FBEEDBF79
:10994000C3FE50C089E290E06BE270E04AE250E072
:1099500027E00E94216186EA98E20E9491632DB778
:109960003EB72A5030400FB6F8943EBF0FBE2DBF11
:10997000ADB6BEB60894A11CB11C9E012D5E3F4F32
:10998000200F311FADB7BEB712963C932E9311979F
:1099900027E730E0F5013383228320E435E0358387
:1099A00024839C01B901882777FD8095982F0E9418
:1099B000DE9920E030E048EC52E40E940E99D50197
:1099C00016966D937D938D939C9319970E94E1A1B8
:1099D000080F191FEDB7FEB73A960FB6F894FEBF01
:1099E0000FBEEDBFC4FE56C089E290E06BE270E0AE
:1099F0004AE250E026E00E94216181E090E00E946E
:109A0000210D80930F0A8EE99BE10E9491632DB78F
:109A10003EB72A5030400FB6F8943EBF0FBE2DBF60
:109A2000ADB6BEB60894A11CB11C9E012D5E3F4F81
:109A3000200F311FADB7BEB712963C932E931197EE
:109A400027E730E0F501338322832AE435E03583CC
:109A500024839C01B901882777FD8095982F0E9467
:109A6000DE9920E030E048EC52E40E940E99D501E6
:109A700016966D937D938D939C9319970E94E1A107
:109A8000080F191FEDB7FEB73A960FB6F894FEBF50
:109A90000FBEEDBFC5FE36C02DB73EB72A503040D1
:109AA0000FB6F8943EBF0FBE2DBFEDB7FEB731968F
:109AB000CE014396800F911FADB7BEB712969C930F
:109AC0008E93119787E790E09383828385E595E0F5
:109AD000958384838091621B9091631BA091641B8A
:109AE000B091651B86839783A087B1870E94E1A10F
:109AF000080F191FEDB7FEB73A960FB6F894FEBFE0
:109B00000FBEEDBFC6FE31C00E94B00C2DB73EB7F0
:109B10002A5030400FB6F8943EBF0FBE2DBFEDB7B0
:109B2000FEB731969E012D5E3F4F200F311FADB71E
:109B3000BEB712963C932E93119727E730E03383FC
:109B4000228323E635E03583248366837783808709
:109B500091870E94E1A1080F191FEDB7FEB73A9651
:109B60000FB6F894FEBF0FBEEDBFC7FE3AC0F89423
:109B70008091912890919228A0919328B091942857
:109B800078942DB73EB72A5030400FB6F8943EBFB8
:109B90000FBE2DBF4DB75EB74F5F5F4F9E012D5E6D
:109BA0003F4F200F311FEDB7FEB73283218327E7E8
:109BB00030E0FA013383228321E735E035832483C3
:109BC00086839783A087B1870E94E1A1080F191FA0
:109BD0002DB73EB7265F3F4F0FB6F8943EBF0FBE7E
:109BE0002DBFD0FEAAC08091ED069091EE060097A1
:109BF00009F4A3C0F8948091912890919228A091A3
:109C00009328B0919428C257DF4F88839983AA8301
:109C1000BB83CE58D04078948091961B9091971B2F
:109C2000A091981BB091991BC257DF4F28813981B1
:109C30004A815B81CE58D040281B390B4A0B5B0B05
:109C4000CA01B9010E94DC99862EA72E682E492EE2
:109C50006091ED067091EE0680E090E00E94DC9944
:109C60009B01AC01682D7A2D862D942D0E940E99B2
:109C7000882EA92E4DB75EB74A5050400FB6F894C3
:109C80005EBF0FBE4DBFEDB7FEB73196CE01439616
:109C9000800F911FADB7BEB712969C938E9311970C
:109CA00087E790E0938382838CE795E095838483B4
:109CB000262F372F482D5A2D2683378340875187EB
:109CC000CD55DF4F6883C35AD040CE55DF4F7883E0
:109CD000C25AD0400E94E1A1080F191FCD55DF4F95
:109CE0006881C35AD040CE55DF4F7881C25AD040E8
:109CF000862F972FA82DBA2D80939E2890939F286A
:109D0000A093A028B093A128C257DF4F28813981A2
:109D10004A815B81CE58D0402093961B3093971B8D
:109D20004093981B5093991B4DB75EB7465F5F4FAA
:109D30000FB6F8945EBF0FBE4DBFD1FE3DC0F89484
:109D40008091952890919628A0919728B091982875
:109D50007894EDB7FEB73A970FB6F894FEBF0FBEF2
:109D6000EDBF4DB75EB74F5F5F4F9E012D5E3F4F1A
:109D7000200F311F3283218327E730E0FA0133833C
:109D8000228329E835E03583248386839783A0875F
:109D9000B1870E94E1A1080F191F2DB73EB7265FBA
:109DA0003F4F0FB6F8943EBF0FBE2DBFC8010E94B3
:109DB0004D4A009709F002CCD2FEAAC08091ED0670
:109DC0009091EE06009709F4A3C0F894809195282D
:109DD00090919628A0919728B0919828C257DF4F6C
:109DE00088839983AA83BB83CE58D040789480918E
:109DF0009A1B90919B1BA0919C1BB0919D1BC257DD
:109E0000DF4F288139814A815B81CE58D040281BA1
:109E1000390B4A0B5B0BCA01B9010E94DC99862EF3
:109E2000A72E682E492E6091ED067091EE0680E017
:109E300090E00E94DC999B01AC01682D7A2D862D63
:109E4000942D0E940E99882EA92E4DB75EB74A50C8
:109E500050400FB6F8945EBF0FBE4DBFEDB7FEB7D2
:109E60003196CE014396800F911FADB7BEB71296C3
:109E70009C938E93119787E790E09383828384E984
:109E800095E095838483262F372F482D5A2D2683DE
:109E9000378340875187CD55DF4F6883C35AD04001
:109EA000CE55DF4F7883C25AD0400E94E1A1080FFF
:109EB000191FCD55DF4F6881C35AD040CE55DF4FB3
:109EC0007881C25AD040862F972FA82DBA2D809323
:109ED000A2289093A328A093A428B093A528C257A2
:109EE000DF4F288139814A815B81CE58D040209351
:109EF0009A1B30939B1B40939C1B50939D1B4DB70B
:109F00005EB7465F5F4F0FB6F8945EBF0FBE4DBFA2
:109F1000D3FE3BC08091352490913624A091372404
:109F2000B0913824EDB7FEB73A970FB6F894FEBF5C
:109F30000FBEEDBF4DB75EB74F5F5F4F9E012D5E09
:109F40003F4F200F311F3283218327E730E0FA0192
:109F50003383228321EA35E0358324838683978304
:109F6000A087B1870E94E1A1080F191F2DB73EB746
:109F7000265F3F4F0FB6F8943EBF0FBE2DBFC801FE
:109F80000E944D4A009709F019CBCA56DF4F8881CD
:109F90009981AA81BB81C659D0400097A105B1051E
:109FA000C9F1ADB7BEB71A970FB6F894BEBF0FBED2
:109FB000ADBFEDB7FEB73196CE014396800F911F2E
:109FC00012969C938E93119787E790E093838283F8
:109FD0008CEA95E09583848380912F1C9091301CAE
:109FE000A091311CB091321C86839783A087B187E2
:109FF0000E94E1A1080F191FEDB7FEB73A960FB600
:10A00000F894FEBF0FBEEDBFC8010E944D4A0097F5
:10A0100009F0D4CAC656DF4F288139814A815B8155
:10A02000CA59D0402115310541055105E1F14DB71F
:10A030005EB74A5050400FB6F8945EBF0FBE4DBF9A
:10A04000EDB7FEB73196CE014396800F911FADB7A5
:10A05000BEB712969C938E93119787E790E09383F7
:10A06000828387EB95E095838483809199289091F2
:10A070009A28A0919B28B0919C2886839783A087DB
:10A08000B1870E94E1A1080F191FEDB7FEB73A96FC
:10A090000FB6F894FEBF0FBEEDBFC8010E944D4A37
:10A0A000009709F08BCAD6FE48C081E00E944E0C92
:10A0B0002DB73EB72A5030400FB6F8943EBF0FBEC2
:10A0C0002DBFADB6BEB60894A11CB11C9E012D5E7D
:10A0D0003F4F200F311FADB7BEB712963C932E9362
:10A0E000119727E730E0F5013383228324EC35E034
:10A0F000358324832091C9063091CA064091CB064E
:10A100005091CC060E94BC9BD50116966D937D9311
:10A110008D939C9319970E94E1A1080F191FEDB729
:10A12000FEB73A960FB6F894FEBF0FBEEDBFC8015A
:10A130000E944D4A009709F041CAD7FE48C082E00C
:10A140000E944E0C2DB73EB72A5030400FB6F894FF
:10A150003EBF0FBE2DBFADB6BEB60894A11CB11C4C
:10A160009E012D5E3F4F200F311FADB7BEB7129637
:10A170003C932E93119727E730E0F5013383228338
:10A1800021ED35E0358324832091CD063091CE0634
:10A190004091CF065091D0060E94BC9BD5011696E7
:10A1A0006D937D938D939C9319970E94E1A1080F65
:10A1B000191FEDB7FEB73A960FB6F894FEBF0FBE63
:10A1C000EDBFC8010E944D4A009709F0F7C9CE566D
:10A1D000DF4F288139814A815B81C259D0402115E6
:10A1E000310541055105C9F183E00E944E0C4DB780
:10A1F0005EB74A5050400FB6F8945EBF0FBE4DBFD9
:10A20000EDB7FEB731969E012D5E3F4F200F311FF7
:10A21000ADB7BEB712963C932E93119727E730E067
:10A22000338322832EED35E0358324836683778361
:10A23000808791870E94E1A1080F191F8C98EDB7C4
:10A24000FEB73A960FB6F894FEBF0FBEEDBFC80139
:10A250000E944D4A009709F0B1C9E1FE3FC08091CC
:10A26000332087FF3BC080ED61E042E121E00E94A6
:10A27000E7652DB73EB72A5030400FB6F8943EBF81
:10A280000FBE2DBFEDB7FEB731969E012D5E3F4F3D
:10A29000200F311FADB7BEB712963C932E93119786
:10A2A00027E730E0338322832BEE35E035832483A8
:10A2B00066837783808791870E94E1A1080F191F29
:10A2C000EDB7FEB73A960FB6F894FEBF0FBEEDBFDE
:10A2D000C8010E944D4A009709F070C9E2FE3FC0D4
:10A2E0008091332087FF3BC080ED62E042E121E0B6
:10A2F0000E94E7652DB73EB72A5030400FB6F8945C
:10A300003EBF0FBE2DBFEDB7FEB731969E012D5E4D
:10A310003F4F200F311FADB7BEB712963C932E931F
:10A32000119727E730E03383228329EF35E0358327
:10A33000248366837783808791870E94E1A1080F39
:10A34000191FEDB7FEB73A960FB6F894FEBF0FBED1
:10A35000EDBFC8010E944D4A009709F02FC9E3FEE6
:10A360003FC08091332087FF3BC080ED63E042E136
:10A3700021E00E94E7652DB73EB72A5030400FB666
:10A38000F8943EBF0FBE2DBFEDB7FEB731969E01CC
:10A390002D5E3F4F200F311FADB7BEB712963C93D5
:10A3A0002E93119727E730E03383228327E036E0AE
:10A3B0003583248366837783808791870E94E1A118
:10A3C000080F191FEDB7FEB73A960FB6F894FEBF07
:10A3D0000FBEEDBFC8010E944D4A009709F0EEC8BC
:10A3E000E4FE3FC08091332087FF3BC080ED64E0F6
:10A3F00042E121E00E94E7652DB73EB72A50304088
:10A400000FB6F8943EBF0FBE2DBFEDB7FEB7319625
:10A410009E012D5E3F4F200F311FADB7BEB7129684
:10A420003C932E93119727E730E03383228325E175
:10A4300036E03583248366837783808791870E9403
:10A44000E1A1080F191FEDB7FEB73A960FB6F894C1
:10A45000FEBF0FBEEDBFC8010E944D4A009709F034
:10A46000ADC8812C912CA0E2AA2EB12C8C209D206D
:10A47000AE20BF20E5FE0AC08091332082FF06C0D7
:10A4800083E061E046E020E00E942915412C512C38
:10A49000F0E46F2E712C4C205D206E207F20E6FEB4
:10A4A0000AC08091332082FF06C083E061E046E06D
:10A4B00021E00E94291581149104A104B10409F43A
:10A4C00040C08091332082FF3CC02DB73EB72A5058
:10A4D00030400FB6F8943EBF0FBE2DBFEDB7FEB7AC
:10A4E0003196CE014396800F911FADB7BEB712963D
:10A4F0009C938E93119787E790E09383828383E206
:10A5000096E0958384838091261C9091271CA091CE
:10A51000281CB091291C86839783A087B1870E944D
:10A52000E1A1080F191FEDB7FEB73A960FB6F894E0
:10A53000FEBF0FBEEDBFC8010E944D4A009709F053
:10A540003DC8411451046104710409F441C0809173
:10A55000332082FF3DC02DB73EB72A5030400FB6A2
:10A56000F8943EBF0FBE2DBFEDB7FEB73196CE01BA
:10A570004396800F911FADB7BEB712969C938E93F2
:10A58000119787E790E0938382838BE296E095832F
:10A59000848380912A1C90912B1CA0912C1CB0913B
:10A5A0002D1C86839783A087B1870E94E1A1080FA5
:10A5B000191FEDB7FEB73A960FB6F894FEBF0FBE5F
:10A5C000EDBFC8010E944D4A009711F00C94DE4A7D
:10A5D000E7FE40C0809133209091342090FF3AC034
:10A5E00080E090E00E94EF272DB73EB72A50304020
:10A5F0000FB6F8943EBF0FBE2DBFEDB7FEB7319634
:10A600009E012D5E3F4F200F311FADB7BEB7129692
:10A610003C932E93119727E730E03383228326E380
:10A6200036E03583248366837783808791870E9411
:10A63000E1A1080F191FEDB7FEB73A960FB6F894CF
:10A64000FEBF0FBEEDBFC8010E944D4A009711F03A
:10A650000C94DE4AF0FE40C080913320909134206B
:10A6600090FF3AC081E090E00E94EF272DB73EB7FF
:10A670002A5030400FB6F8943EBF0FBE2DBFEDB745
:10A68000FEB731969E012D5E3F4F200F311FADB7B3
:10A69000BEB712963C932E93119727E730E0338391
:10A6A000228326E436E0358324836683778380879C
:10A6B00091870E94E1A1080F191FEDB7FEB73A96E6
:10A6C0000FB6F894FEBF0FBEEDBFC8010E944D4A01
:10A6D000009711F00C94DE4AF2FE51C080913320B5
:10A6E0009091342090FF4BC081E090E00E94EF27D2
:10A6F0004B015C0160E070E0CB010E94A799DC0196
:10A70000CB010E94EF279B01AC01C501B4010E945F
:10A7100042262DB73EB72A5030400FB6F8943EBFC0
:10A720000FBE2DBFEDB7FEB731969E012D5E3F4F98
:10A73000200F311FADB7BEB712963C932E931197E1
:10A7400027E730E03383228327E536E0358324830F
:10A7500066837783808791870E94E1A1080F191F84
:10A76000EDB7FEB73A960FB6F894FEBF0FBEEDBF39
:10A77000C8010E944D4A009711F00C94DE4AF3FE86
:10A7800051C0809133209091342090FF4BC081E0E4
:10A7900090E00E94EF274B015C0160E070E0CB018C
:10A7A0000E94A799DC01CB010E94EF279B01AC011D
:10A7B000C501B4010E94A3262DB73EB72A503040F0
:10A7C0000FB6F8943EBF0FBE2DBFEDB7FEB7319662
:10A7D0009E012D5E3F4F200F311FADB7BEB71296C1
:10A7E0003C932E93119727E730E03383228322E6B0
:10A7F00036E03583248366837783808791870E9440
:10A80000E1A1080F191FEDB7FEB73A960FB6F894FD
:10A81000FEBF0FBEEDBFC8010E944D4A009711F068
:10A820000C94DE4AF4FE51C0809133209091342084
:10A8300090FF4BC081E090E00E94EF274B015C014C
:10A8400060E070E0CB010E94A799DC01CB010E947F
:10A85000EF279B01AC01C501B4010E9408272DB769
:10A860003EB72A5030400FB6F8943EBF0FBE2DBF02
:10A87000EDB7FEB731969E012D5E3F4F200F311F81
:10A88000ADB7BEB712963C932E93119727E730E0F1
:10A890003383228320E736E03583248366837783FE
:10A8A000808791870E94E1A1080F191FEDB7FEB7BD
:10A8B0003A960FB6F894FEBF0FBEEDBFC8010E94D6
:10A8C0004D4A009711F00C94DE4AF1FE3EC0809193
:10A8D00033209091342091FF38C00E94111A2DB777
:10A8E0003EB72A5030400FB6F8943EBF0FBE2DBF82
:10A8F000EDB7FEB731969E012D5E3F4F200F311F01
:10A90000ADB7BEB712963C932E93119727E730E070
:10A910003383228323E836E0358324836683778379
:10A92000808791870E94E1A1080F191FEDB7FEB73C
:10A930003A960FB6F894FEBF0FBEEDBFC8010E9455
:10A940004D4A009711F00C94DE4AC256DF4F288121
:10A9500039814A815B81CE59D040211531054105AD
:10A96000510509F44AC04DB75EB74E5050400FB67E
:10A97000F8945EBF0FBE4DBFEDB7FEB73196CE0166
:10A980004396800F911FADB7BEB712969C938E93DE
:10A99000119787E790E09383828384E996E095831B
:10A9A0008483C657DF4FA881B981CA58D040129618
:10A9B0008C9112978683178213968C9113978087B8
:10A9C000118615968C9115978287138616968C9111
:10A9D000848715860E94E1A1080F191FEDB7FEB705
:10A9E0003E960FB6F894FEBF0FBEEDBFC8010E94A1
:10A9F0004D4A009711F00C94DE4A779A8091080A2C
:10AA00009091090A92FD749AC114D104E104F104F1
:10AA1000E9F18091080A9091090A82FD08C08091AD
:10AA2000EF0680FD04C081FF31C01D9B2FC000D008
:10AA300000D08BEA96E0ADB7BEB712969C938E938A
:10AA40001197CE01439614969C938E9313970E9470
:10AA500078A12091D1060F900F900F900F90222394
:10AA6000A9F000D000D0EDB7FEB7319684EE91E0AA
:10AA7000ADB7BEB712969C938E9311972283138223
:10AA80000E948AA10F900F900F900F908091F20674
:10AA90008061898B80912C0A8A8BFE01E00FF11F67
:10AAA000138A58010894A11CB11C8091080A909146
:10AAB000090A80FF12C000D000D082EB96E0EDB70B
:10AAC000FEB7928381830D5F1F4F148303830E941F
:10AAD00078A10F900F900F900F90E2E0CE2ED12C26
:10AAE000CA0CDB1C8E010F5E1F4FC801B6010E940D
:10AAF0001F608091EF0682FF08C089ED96E0B801E3
:10AB0000A60121E934E20E94A4648091080A909190
:10AB1000090A82FD73980E943A6D89E19AE00E94C9
:10AB2000C5568091EF069091F00690FF48C00091C5
:10AB3000ED061091EE060E94586EC82E1092EE0699
:10AB40001092ED0689E190E00E94706E29C0739822
:10AB500080912C0A8F5F80932C0A8A8BB5016F5FDE
:10AB60007F4FCE0141960E941F6089E19AE00E94CA
:10AB7000C55680914E1290914F1265E840E050E02A
:10AB80000E948B588EEF9DE0C457DF4FA881B9819A
:10AB9000CC58D04011969C938E9362C0AA24BB24BB
:10ABA0002091EF063091F00630FDD1CF8C2D90E052
:10ABB0000E94706E1093EE060093ED06739A8091DA
:10ABC0000B0A90910C0A009711F00E949C6C8091E6
:10ABD0002C0A8F5F80932C0A8091080A9091090AB1
:10ABE00082FD02C00C94DE4A739A0C94DE4A84E221
:10ABF0009AE00E946C5B009799F10E943A6D8091F7
:10AC0000EF0687FD2B9884E29AE060E470E00E94F2
:10AC1000415B86E19EE0C457DF4FE881F981CC5863
:10AC2000D040918380831CC084E29AE00E946C5BD8
:10AC30000097B1F00E949C6C8091EF0687FD02C0E6
:10AC40000C94DE4A2B9A0C94DE4AC457DF4FA8813D
:10AC5000B981CC58D04011961C921E9283E001C05D
:10AC600081E0CD55DF4F0FB6F894DEBF0FBECDBFEC
:10AC7000CF91DF911F910F91FF90EF90DF90CF90D8
:10AC8000BF90AF909F908F907F906F905F904F900C
:10AC90003F902F9008950E94EF5608950895FC016B
:10ACA000DB018C91808311968C911197818308959B
:10ACB000FC01DB0190818C91981741F421E030E098
:10ACC000918111968C911197981711F020E030E046
:10ACD000C9010895FC0180818093B6288181809309
:10ACE000B7280895DC011996ED91FC911A9702801E
:10ACF000F381E02D309709F009950895EF92FF92C6
:10AD00000F931F93DF93CF9300D0CDB7DEB78C01A5
:10AD100088E10E949A60BC017E010894E11CF11C4C
:10AD2000C7010E944F56D8011996ED91FC911A97D0
:10AD30000190F081E02DC801B70109950F900F90A7
:10AD4000CF91DF911F910F91FF90EF900895EF92B7
:10AD5000FF920F931F93CF93DF93EC018B017A0146
:10AD60004EE857E00E94D356FA86E986C80162E9A8
:10AD700077E00E943257DF91CF911F910F91FF90A2
:10AD8000EF9008950E94EC560895CF93DF93EC0165
:10AD900088E166EB78E20E949060CE010E94EF5657
:10ADA000DF91CF910895EF92FF920F931F93CF936E
:10ADB000DF93EC018B017A010E940B57F886EF823A
:10ADC000C80166E977E00E943257DF91CF911F9169
:10ADD0000F91FF90EF9008950E94145708950E94DC
:10ADE00011730895FC01A781B0852D913C91F90163
:10ADF00009950895DC011796ED91FC911897028052
:10AE0000F381E02D309709F0099508958AE492E1E5
:10AE10000E947E590895FC01738362838AE492E163
:10AE2000BF010E94095A0895BC018AE492E10E9480
:10AE3000D0590895CF93DF93EC018AE492E10E9408
:10AE4000825908C0828193818C179D0739F0CF0108
:10AE50000E94485AE82FF92F3097A1F7CF01DF91D0
:10AE6000CF9108950F931F93CF93DF938B010E948F
:10AE70001A57EC01009731F01D830C83C8010E9422
:10AE800069758E83DF91CF911F910F9108951F9364
:10AE9000CF93DF93EC01162F888580FF1DC0EC81D6
:10AEA000FD813097C9F0D0934F12C0934E1282E0CB
:10AEB0008887CE0106960995992787FD9095029778
:10AEC0008230910510F0133829F4CE01BE010E94A2
:10AED000705702C081E08887DF91CF911F9108955C
:10AEE000CF92DF92EF92FF920F931F93CF93DF9356
:10AEF000EC017B01C0904E12D0904F1200914C1289
:10AF000010914D12F80103C00190F081E02DEC1773
:10AF1000FD0719F03097C1F746C0209709F443C0E8
:10AF20008885882309F118860BC0C017D10729F03E
:10AF3000C80167E8AE010E944757F80100811181FE
:10AF40000115110591F7EC81FD81309769F0CE155F
:10AF5000DF0551F0D0934F12C0934E12CE010696EA
:10AF600063E840E050E00995E0914C12F0914D12F9
:10AF7000CE17DF0791F48881998190934D128093C9
:10AF80004C120DC0808191818C179D0729F4888116
:10AF900099819183808303C0FC01309799F7D09207
:10AFA0004F12C0924E12DF91CF911F910F91FF90DF
:10AFB000EF90DF90CF9008951F93CF93DF9310927F
:10AFC0005012C0914C12D0914D1211E00EC08985E3
:10AFD000882341F018871986CE0162E840E050E0EE
:10AFE0000E9447570990D881C02D209781F7DF91A3
:10AFF000CF911F9108958091FB12982F9F5F90939E
:10B00000FB12089560914E1270914F120E9470577A
:10B0100008958AE88093FB121092521210925112F6
:10B0200010924D1210924C1210924F1210924E121A
:10B03000089580915012882311F00E94DC5770917E
:10B040005112772309F455C02091521230E0F901D2
:10B05000EE0FFF1FEE0FFF1FE20FF31FED5AFD4E25
:10B0600060816093FA12418152815093F9124093AA
:10B07000F812838194819093F7128093F6122F5FD8
:10B080003F4F2F71307020935212715070935112B4
:10B09000009741F580914C1290914D1218C080910B
:10B0A0005012882311F00E94DC574091F812509101
:10B0B000F9128091F4129091F5126091FA120E94A7
:10B0C0004757E091F412F091F512808191819093AD
:10B0D000F5128093F4128091F4129091F51200977A
:10B0E000F1F607C0613819F421E0FC0120870E94C5
:10B0F0004757809150122091511230E0280F311D96
:10B10000C9010895809150122091511230E0280F0A
:10B11000311DC9010895709151127032D9F02091FA
:10B120005212270F2F712093F31230E0F901EE0F26
:10B13000FF1FEE0FFF1FE20FF31FED5AFD4E60835E
:10B1400052834183948383837F5F7093511220E005
:10B1500030E002C021E030E0C9010895CF93DF93D1
:10B16000C0914E12D0914F120E944757D0934F1268
:10B17000C0934E12DF91CF910895FC01AB019091E5
:10B180004C1280914D129C01A32FB22F03C00D9041
:10B19000BC91A02DAE17BF0791F01097C1F7309763
:10B1A00071F090838183F0934D12E0934C1281E013
:10B1B000808717821682CF0161E80E94AE580895F9
:10B1C000FC01009741F080858150823020F481E0BD
:10B1D000818780935012089521E030E0FC01808542
:10B1E000882311F420E030E0C9010895CF93DF9364
:10B1F000EC014A815B818C819D8160E070E00E945E
:10B20000F3A04A815B8188819981489F9001499F81
:10B21000300D589F300D11248E819F8160E070E0C9
:10B22000A9010E94F3A0DF91CF910895FC018281D2
:10B23000938120E030E019C0A481B581A20FB31F33
:10B240004C91442381F481E08C9340815181249F6F
:10B25000C001259F900D349F900D112426813781C8
:10B26000280F391F07C02F5F3F4F2817390720F3DA
:10B2700020E030E0C9010895FC0126813781428138
:10B28000538180E090E018C02617370781F4A4812D
:10B29000B581A80FB91F2C91121614F421502C93CC
:10B2A0000480F581E02DE80FF91F80810895A081C9
:10B2B000B1812A0F3B1F01968417950728F38FEF62
:10B2C0000895FC01CB01268137816217730790F046
:10B2D000A081B18162817381A69FA001A79F500DBB
:10B2E000B69F500D1124420F531F21E030E0841708
:10B2F000950710F020E030E0C9010895FC011182AB
:10B3000010820895FC01808191810895FB012081C4
:10B310003181FC01318320830895FC01208131813A
:10B320002115310511F407C09C01F901808191813B
:10B330000097D1F702C020E030E0C9010895CF9313
:10B34000DF93DC012D913C91119721153105A9F076
:10B35000F90180819181009729F411961C921E9227
:10B360000EC0F90120813181D9018D919C911197F5
:10B370000097B9F71182108202C020E030E0C901C5
:10B38000DF91CF910895DC01ED91FC9111973097F9
:10B3900029F08081918111969C938E93CF0108951D
:10B3A000CF93DF93FC01A081B1811097D9F0C0E069
:10B3B000D0E016C0A617B70771F48D919C91119734
:10B3C000209719F49183808302C099838883119612
:10B3D0001C921E9207C0ED0198818981A92FB82F78
:10B3E000109741F7DF91CF9108950F931F93CF935B
:10B3F000DF938C01EB010E94D059F801808191818B
:10B4000099838883D183C083DF91CF911F910F915E
:10B410000895EF92FF920F931F93CF93DF93EC0168
:10B420007B010E94D059F70111821082CE010E9447
:10B430008D59FC01009719F4E882F98202C0F1826B
:10B44000E082DF91CF911F910F91FF90EF900895CF
:10B45000DC01ED91FC91119720E030E005C02F5FF9
:10B460003F4F0190F081E02D3097C9F7C901089551
:10B47000FB01309721F4BA010E94F5590895DA01D1
:10B480008081918111969C938E935183408308957E
:10B49000009721F0FC012081318102C020E030E0E2
:10B4A000C90108958091FC129091FD12009729F432
:10B4B0001092FF121092FE1208950E94FE69E09110
:10B4C000FC12F091FD122281338140815181240FC1
:10B4D000351F281B390B0CC042815381608171815B
:10B4E000460F571F481B590B4217530708F49A0180
:10B4F0000480F581E02D309779F7280F391F3093BC
:10B50000FF122093FE12089584EA97E00E94E0580B
:10B510000895CF92DF92EF92FF920F931F93CF93F4
:10B52000DF937C01FC0180819181009729F08A35AD
:10B53000910509F06EC00BC01092FD121092FC1222
:10B540008AE590E0F7019183808381E066C06738E7
:10B5500049F5CA01E091FC12F091FD1203C004808C
:10B56000F581E02D309741F326813781281739077F
:10B57000B1F3E093FC12F093FD120FC016962D91DB
:10B580003C9117972817390739F414962D913C915F
:10B59000159735832483DF01FD01A481B5811097C0
:10B5A00069F7CECF623861F6C091FC12D091FD12DE
:10B5B00000E010E02BC0CE010E9461790097F1F00D
:10B5C0008E819F8168E8AE010E948B580097A1F49C
:10B5D0001F821E828C819D810115110521F0F801C9
:10B5E0009583848304C09093FD128093FC121D8286
:10B5F0001C820E94525AD8CF0E94845A8E019C818C
:10B600008D81C92EE6016E01D82EE601209799F6AC
:10B6100097CFF7011182108283E0DF91CF911F91C4
:10B620000F91FF90EF90DF90CF900895CF93DF932D
:10B63000EC010E94845A8E819F81009769F0E0910D
:10B64000FC12F091FD1206C0EC17FD07A9F0048072
:10B65000F581E02D3097C1F780914E1290914F12F5
:10B660009F838E838091FC129091FD129D838C8329
:10B67000D093FD12C093FC120E94525ADF91CF91D9
:10B680000895CF93DF93EC010E944179CE010E948F
:10B69000165BDF91CF910895CF93DF93EC010E9469
:10B6A0004D79CE010E94165BDF91CF910895CF9323
:10B6B000DF93EC010E945779CE010E94165BDF9167
:10B6C000CF910895FC0180819181860F971F91830E
:10B6D00080830E94525A089521E030E0FC01868167
:10B6E0009781009711F020E030E0C9010895FC0136
:10B6F0002281338180819181280F391FC9010895EA
:10B70000FC0180819181089521E030E08091FC125C
:10B710009091FD12009711F420E030E0C9010895E6
:10B720008091FC129091FD12009729F02091FE1259
:10B730003091FF1202C020E030E0C9010895CF939C
:10B74000DF93EC01E091FC12F091FD128E179F0740
:10B7500041F48C819D819093FD128093FC1214C062
:10B76000FC01309731F0848195818C179D07C1F7DA
:10B7700007C01D821C821F821E82DF91CF91089517
:10B780008C819D81958384830E94525AF2CFCF92FF
:10B79000DF92EF92FF920F931F93CF93DF938C0171
:10B7A0007A01FC0180819181009729F08B34910509
:10B7B00009F051C01EC081E093E10E948259C82E59
:10B7C000E6017E01F92EE70109C06C817D81CE0181
:10B7D00002960E94415B0990D881C02D2097A9F75D
:10B7E00081E0809300138BE490E0F80191838083E3
:10B7F00037C06838A9F581E093E10E948259C82ECC
:10B80000E6016E01D92EE60123C0CE010296E816AC
:10B81000F906D9F481E093E1BE010E94D059E0908D
:10B820004E12F0904F128A859B8590934F12809311
:10B830004E12EC85FD85309719F08E859F85099510
:10B84000F0924F12E0924E12CECF0990D881C02DC7
:10B850002097D9F6C8CFF8011182108283E001C089
:10B8600081E0DF91CF911F910F91FF90EF90DF90DA
:10B87000CF9008951092001381E093E10E947E59C9
:10B880008DEB97E060E070E00E94BD5808950F9343
:10B890001F93CF93DF93EC0100914E1210914F1242
:10B8A0001B870A875D874C873F872E87809100130F
:10B8B000882379F08DEB97E090934F1280934E128E
:10B8C000CE0102960E94415B10934F1200934E12DC
:10B8D00002C07D836C8381E093E1BE010E94D05958
:10B8E00081E093E1BE010E94095ADF91CF911F913F
:10B8F0000F9108950F931F93CF93DF93EC018091E5
:10B900000013882391F000914E1210914F128DEB8D
:10B9100097E090934F1280934E12CE0102960E94B0
:10B920004C5B10934F1200934E1281E093E1BE01E5
:10B930000E94D05981E093E1BE010E94095ADF9133
:10B94000CF911F910F9108950F931F93CF93DF9382
:10B95000EC0180910013882391F000914E12109118
:10B960004F128DEB97E090934F1280934E12CE01C1
:10B9700002960E94575B10934F1200934E1281E083
:10B9800093E1BE010E94D05981E093E1BE010E9483
:10B99000095ADF91CF911F910F910895CF93DF93B3
:10B9A000EC0180910013882329F0CE0102960E94B9
:10B9B0009F5B04C01F821E821986188681E093E176
:10B9C000BE010E94D059DF91CF910895CF93DF93AC
:10B9D000EC0180910013882331F0CE0102960E9481
:10B9E0006C5B9C0114C081E093E10E948259E82FB6
:10B9F000F92F06C0EC17FD0741F00190F081E02D12
:10BA00003097C1F721E030E002C020E030E0C9010A
:10BA1000DF91CF9108950F931F930091B628109155
:10BA2000B7280E942B6A2DB73EB7225530400FB67B
:10BA3000F8943EBF0FBE2DBFEDB7FEB731962CED8B
:10BA40003DE0ADB7BEB712963C932E93119702839B
:10BA50001382148315826683778380879187809110
:10BA6000A92A9091AA2AA091AB2AB091AC2A8287E8
:10BA70009387A487B5878091AD2A9091AE2AA09133
:10BA8000AF2AB091B02A86879787A08BB18B80911F
:10BA9000B12A9091B22AA091B32AB091B42A828B94
:10BAA000938BA48BB58B8091B52A9091B62AA091E7
:10BAB000B72AB091B82A868B978BA08FB18F8091CF
:10BAC000B92A9091BA2AA091BB2AB091BC2A828F40
:10BAD000938FA48FB58F8091BD2A9091BE2AA0919B
:10BAE000BF2AB091C02A868F978FA0A3B1A380915F
:10BAF000C12A9091C22AA091C32AB091C42A82A3DC
:10BB000093A3A4A3B5A38091C52A9091C62AA0911E
:10BB1000C72AB091C82A86A397A3A0A7B1A78091EE
:10BB2000C92A9091CA2AA091CB2AB091CC2A82A787
:10BB300093A7A4A7B5A78091CD2A9091CE2AA091D2
:10BB4000CF2AB091D02A86A797A7A0ABB1AB80919E
:10BB5000D12A9091D22AA091D32AB091D42A82AB33
:10BB600093ABA4ABB5AB8091D52A9091D62AA09186
:10BB7000D72AB091D82A86AB97ABA0AFB1AF80914E
:10BB8000D92A9091DA2AA091DB2AB091DC2A82AFDF
:10BB900093AFA4AFB5AFEDB7FEB7FF968091DD2AA6
:10BBA0009091DE2AA091DF2AB091E02A80839183D0
:10BBB000A283B383EDB7FEB7ED5BFF4F8091E12A1F
:10BBC0009091E22AA091E32AB091E42A80839183A4
:10BBD000A283B383EDB7FEB7E95BFF4F8091E52AFF
:10BBE0009091E62AA091E72AB091E82A8083918378
:10BBF000A283B383EDB7FEB7E55BFF4F8091E92ADF
:10BC00009091EA2AA091EB2AB091EC2A808391834B
:10BC1000A283B383EDB7FEB7E15BFF4F8091ED2ABE
:10BC20009091EE2AA091EF2AB091F02A808391831F
:10BC3000A283B3830E948AA10091B6281091B728ED
:10BC40002DB73EB72E5A3F4F0FB6F8943EBF0FBEEA
:10BC50002DBF0E942B6AADB7BEB7D2970FB6F8942E
:10BC6000BEBF0FBEADBFEDB7FEB731962DE63DE0CE
:10BC700012963C932E93119702831382148315829C
:10BC800066837783808791878091F12A9091F22A49
:10BC9000A091F32AB091F42A82879387A487B5876D
:10BCA0008091F52A9091F62AA091F72AB091F82A6E
:10BCB00086879787A08BB18B8091F92A9091FA2A79
:10BCC000A091FB2AB091FC2A828B938BA48BB58B1D
:10BCD0008091FD2A9091FE2AA091FF2AB091002B1D
:10BCE000868B978BA08FB18F8091012B9091022B27
:10BCF000A091032BB091042B828F938FA48FB58FCB
:10BD00008091052B9091062BA091072BB091082BC9
:10BD1000868F978FA0A3B1A38091092B90910A2BB6
:10BD2000A0910B2BB0910C2B82A393A3A4A3B5A33A
:10BD300080910D2B90910E2BA0910F2BB091102B79
:10BD400086A397A3A0A7B1A78091192B90911A2B36
:10BD5000A0911B2BB0911C2B82A793A7A4A7B5A7DA
:10BD600080911D2B90911E2BA0911F2BB091202B09
:10BD700086A797A7A0ABB1AB0E948AA12DB73EB70B
:10BD80002E5C3F4F0FB6F8943EBF0FBE2DBF1F91E4
:10BD90000F91089580E3809303130895EF92FF922B
:10BDA000CF93DF932091031330E0C0E3D0E0C21BB8
:10BDB000D30B285F3C4EB901AE010E94EAA0CE0130
:10BDC000DF91CF91FF90EF900895AF92BF92CF9205
:10BDD000DF92EF92FF920F931F93CF93DF937C013B
:10BDE000C0900413D09005132091031330E0860116
:10BDF000005D1F4F021B130B01381105E0F4C0E377
:10BE0000D0E0C21BD30B285F3C4EB901AE010E94AB
:10BE1000EAA0CE0DDF1D209106133091071380910B
:10BE2000BA139091BB13280F391FCE01B901A60197
:10BE30000E94EAA002C000E010E0C801DF91CF91AB
:10BE40001F910F91FF90EF90DF90CF90BF90AF9038
:10BE5000089590910313980F9093031308954091C0
:10BE60000413509105139C014817590798F08091CD
:10BE7000BA139091BB13820F931F9093BB138093BF
:10BE8000BA13421B530B509305134093041321E044
:10BE900030E002C020E030E0C9010895909305131E
:10BEA0008093041308952091BA133091BB13285C3A
:10BEB0003C4EC90108952091031330E0285F3C4EA9
:10BEC000C901089521E030E0809106139091071395
:10BED00043E18833940711F420E030E0C90108956C
:10BEE0000E94625F009771F028E333E160910613CE
:10BEF000709107134091041350910513C9010E94DA
:10BF0000EAA00895A091BA13B091BB131097B9F0AD
:10BF10002091041330910513205D3F4FA85CBC4E67
:10BF2000E8E3F3E180E390E003C04D914193019693
:10BF300082179307D4F31092BB131092BA1308958B
:10BF400080910613909107130895809104139091A6
:10BF5000051308959091031380E3891B089580E3EE
:10BF600090910313891B2091041330910513280F1E
:10BF7000311DC90108951F93CF93DF93EC011091F8
:10BF80000313812F90E08C179D076CF00E94AF5F28
:10BF90008C0F9D1F8138910530F41C1B10930313E7
:10BFA00021E030E002C020E030E0C901DF91CF9114
:10BFB0001F910895CF93DF93E0ECF8E21192119274
:10BFC00088E2E03FF807D1F7C0E0D0E0CE01880F6B
:10BFD000991F8854974D6CE877E00E944F56219640
:10BFE000C430D10599F7DF91CF9108951092BB131A
:10BFF0001092BA13109205131092041380E38093E9
:10C00000031388E393E190930713809306130E9430
:10C01000DA5F08950F931F93CF93DF93EC018B01A9
:10C020000E94F65FD0930713C09306131093051375
:10C0300000930413DF91CF911F910F910895CF9238
:10C04000DF92EF92FF920F931F93DF93CF9300D075
:10C05000CDB7DEB78C0169837A830E94F65F698170
:10C060007A81C62ED72E21E8C216D10418F030E806
:10C07000C32ED12C8091061390910713B801A6010D
:10C080000E94EAA0D0920513C0920413C6010F903B
:10C090000F90CF91DF911F910F91FF90EF90DF9064
:10C0A000CF900895282F392FD901E0ECF8E280E3F2
:10C0B00001900D928150E1F7862F972FDC01E8EB7C
:10C0C000F8E288E001900D928150E1F70895E0ECEC
:10C0D000F8E2282F392FD90180E30D900192815089
:10C0E000E1F7A8EBB8E2862F972FFC0188E00190DA
:10C0F0000D928150E1F70895E82FF0E0EE0FFF1F59
:10C10000E054F74D7183608381E090E00895E82F5B
:10C11000F0E0EE0FFF1FE054F74D8081918108950C
:10C1200090E0880F991F8857974D0E944F5681E0E5
:10C1300090E00895282F30E0220F331F2857374D05
:10C14000C90108958115910511F00197F1F708953E
:10C15000E091F328F091F42890818091F2288923CE
:10C160000895E091F028F091F12880819091F228D3
:10C17000892B8083E091F528F091F62880819091B9
:10C18000F228892B80830895E091F028F091F1281E
:10C1900090818091F228809589238083E091F52811
:10C1A000F091F62890818091F228809589238083F0
:10C1B0000895FF920F931F93E091F028F091F128DA
:10C1C00090818091F228809589238083E091F528E1
:10C1D000F091F62880819091F228892B80838FEB53
:10C1E00093E00E94A260FFB6F894E091F528F091E8
:10C1F000F62890818091F22880958923808383E8B6
:10C2000090E00E94A260E091F328F091F428008170
:10C210001091F228FFBE78948BE393E00E94A26015
:10C22000E091F328F091F42880819091F2288923FD
:10C2300019F0802F812301C081E01F910F91FF90A1
:10C2400008955093F6284093F5287093F128609351
:10C25000F0289093F4288093F32881E090E002C0C6
:10C26000880F991F2A95E2F78093F2280E94D960DF
:10C2700008950F931F93182F0FB7F894E091F528A6
:10C28000F091F62880819091F228892B808383E0B9
:10C2900090E00E94A260112351F0E091F528F09106
:10C2A000F62890818091F22880958923808387E108
:10C2B00090E00E94A260E091F328F091F428808140
:10C2C0009091F228892309F410E089E590E00E941A
:10C2D000A260E091F528F091F62890818091F228F3
:10C2E0008095892380830FBF8BE390E00E94A2603A
:10C2F000812F1F910F9108950F931F93182F08E01E
:10C30000812F81700E94396116958111106801504A
:10C31000B9F7812F1F910F9108958FEF0E947C61D3
:10C320000895DF92EF92FF920F931F93CF93DF93C5
:10C33000182FEB010E94D960882389F580EF0E94B5
:10C340007C61EE2400E498EFD92ED00E81E00E94AB
:10C350003961F82E81E00E943961882319F0FF20AD
:10C3600069F020C0FF2051F4011728F0888180FF78
:10C3700005C0101719F0E02EFF24F3948F2D0E94B2
:10C380003961888186958883FF2011F080688883D1
:10C3900001500D15D9F6002339F02196D4CFEE24A3
:10C3A000EA9402C08EEFE82E8E2DDF91CF911F917F
:10C3B0000F91FF90EF90DF9008950F931F93CF930D
:10C3C000DF93182FEB010E94D960209751F085E58B
:10C3D0000E947C6108E089910E947C610150D9F73C
:10C3E00003C08CEC0E947C61812F0E947C61DF91F4
:10C3F000CF911F910F9108950F931F93CF93DF93C8
:10C40000FB01DA01E801408150E0718160E0462BD8
:10C41000572B803171F4BA016E7F13E0660F771FDE
:10C420001A95E1F796814CE050E0491B5109460FFF
:10C43000571F57FF06C091E09C93509541955F4F61
:10C4400001C01C92883289F4848190E0BC0160763E
:10C4500070706036710549F086FF02C04E7F05C0DE
:10C4600085FF02C04C7F01C0487FCA0154E0969509
:10C4700087955A95E1F7F90180834F70488380E0F2
:10C48000DF91CF911F910F9108950F931F93CF9339
:10C49000DF938C01EB01F8018081BE010E94916164
:10C4A000F801808381508D3F28F48881883211F013
:10C4B000803189F7DF91CF911F910F9108951F93DC
:10C4C000CF93DF93EC010E94D96084EBBE010E9400
:10C4D000DD6181E00E943961182F0E94D96081E0FE
:10C4E000112309F480E0DF91CF911F9108951F93EC
:10C4F000CF93DF93182FEB010E94D9600E94A860B0
:10C50000882349F084E4BE010E94DD61113029F0E6
:10C510000E94B16002C082E001C080E0DF91CF9153
:10C520001F9108956F927F928F929F92AF92BF92C8
:10C53000CF92DF92EF92FF920F931F93DF93CF93EF
:10C54000CDB7DEB729970FB6F894DEBF0FBECDBFCB
:10C550007C014B013A0159010E94D9608EEBB70171
:10C560000E94DD618E010F5F1F4F8AE0C82ED12C23
:10C57000CC0EDD1E0E948D61F80181938F01EC15B8
:10C58000FD05C1F78E010F5F1F4FC80169E070E024
:10C590000E94127E882351F4F7018081B801A40122
:10C5A000930185010E94FC6180E001C083E029962F
:10C5B0000FB6F894DEBF0FBECDBFCF91DF911F91B4
:10C5C0000F91FF90EF90DF90CF90BF90AF909F9032
:10C5D0008F907F906F9008957F928F929F92AF92ED
:10C5E000BF92CF92DF92EF92FF920F931F93DF9350
:10C5F000CF93CDB7DEB729970FB6F894DEBF0FBE45
:10C60000CDBF782E5B014A0179018EEB60E070E0CE
:10C610000E94DD618E010F5F1F4F9AE0C92ED12C61
:10C62000CC0EDD1E0E948D61F80181938F01EC1507
:10C63000FD05C1F78E010F5F1F4FC80169E070E073
:10C640000E94127E882349F4872DB801A501940128
:10C6500087010E94FC6180E001C083E029960FB64B
:10C66000F894DEBF0FBECDBFCF91DF911F910F9128
:10C67000FF90EF90DF90CF90BF90AF909F908F9002
:10C680007F9008950F931F93DF93CF93CDB7DEB7BD
:10C6900028970FB6F894DEBF0FBECDBF182F062F18
:10C6A000DE011196EFECF7E088E001900D928150E9
:10C6B000E1F7242F332727FD309541E752E0249FEF
:10C6C000C001259F900D349F900D112464E670E009
:10C6D0000E94AF9CAB0164E6069FB0011124460F97
:10C6E000571FFE013196CE010996619170E0261721
:10C6F000370719F44F5F5F4F03C0E817F907A9F731
:10C70000112319F0509541955F4FCA0128960FB635
:10C71000F894DEBF0FBECDBFCF91DF911F910F9177
:10C7200008950F931F93DF93CF93CDB7DEB72B9769
:10C730000FB6F894DEBF0FBECDBF182F092F885F4C
:10C74000612F792F0E947762882309F049C066E43F
:10C7500071E48FE090E00E94FE63812F902FBE0174
:10C760006F5F7F4FAE014E5F5F4F9E012D5F3F4F6A
:10C770000E9492628823A1F5DE011496E7ECF7E0AF
:10C7800088E001900D928150E1F74B81642F70E0B9
:10C7900021E732E0629FC001639F900D729F900D70
:10C7A000112464E670E00E94AF9C9A8184E6989F11
:10C7B000C0011124680F791FFE013496CE010C963A
:10C7C0002191421719F46F5F7F4F03C0E817F907F3
:10C7D000B9F78981882331F0709561957F4F02C048
:10C7E00064E371E2CB012B960FB6F894DEBF0FBE67
:10C7F000CDBFCF91DF911F910F910895DC01CB0147
:10C8000081159105A105B10529F081509040A04006
:10C81000B040D9F708951092B90080E28093B80033
:10C82000089594EA9093BC0020EA36E841E050E095
:10C8300005C02150304040405040F1F09091BC0084
:10C8400097FFF7CF1DC09031B9F48093BB0084E807
:10C850008093BC0080EA96E8A1E0B0E004C00197B4
:10C86000A109B10959F02091BC0027FFF8CF0EC0F3
:10C8700081E0903421F40FC081E0089581E00895B3
:10C880009091B900987F9830F1F6DFCF9091B90080
:10C89000987F983169F780E0089544EA34E824E904
:10C8A0004093BC009091BC0097FFFCCF9091B900E1
:10C8B000987F983011F0903199F78093BB003093B6
:10C8C000BC009091BC0097FFFCCF9091B900987F7D
:10C8D000903211F0983539F42093BC009091BC004F
:10C8E00094FDFCCFDDCF08950E941164089584E982
:10C8F0008093BC008091BC0084FDFCCF08958093A0
:10C90000BB0084E88093BC008091BC0087FFFCCF13
:10C910009091B900987F81E0983209F480E0089501
:10C9200084EC8093BC008091BC0087FFFCCF809199
:10C93000BB00089584E88093BC008091BC0087FF11
:10C94000FCCF8091BB000895E82FF92F80E19191F1
:10C9500090933F018150D9F780913C018F7D809366
:10C960003C0180913C01877F80933C01862F972F6B
:10C97000FC0180E1919190933E018150D9F7809123
:10C980003C01806880933C0180913D0180FFFCCF99
:10C990004051504080913C01806280933C018091E5
:10C9A0003C01877F80933C0114C0862F972FFC01A8
:10C9B00080E1919190933E018150D9F780913C01A3
:10C9C000806880933C0180913D0180FFFCCF405105
:10C9D0005040141615064CF3822F932FFC0180E172
:10C9E00090913E0191938150D9F781E090E00895B4
:10C9F0000F931F93CF93DF938C018CE70E944D64BC
:10CA00008CE70E947F64C0E0D0E0F80181918F0143
:10CA10000E947F642196C031D105B9F70E947764E6
:10CA2000DF91CF911F910F910895813039F48CE7F8
:10CA300090E060E070E040E050E006C08CE790E0FD
:10CA400060E070E040EC50E00E942F1308958130C8
:10CA500039F48CE790E060E070E04EE050E006C012
:10CA60008CE790E060E070E048E050E00E942F1317
:10CA700008958CE790E060E070E041E050E00E94B3
:10CA80002F136AE67AE080E090E00E94FE6308954A
:10CA90008CE790E060E070E048E350E00E942F13E4
:10CAA0008CE790E060E070E049E350E00E942F13D3
:10CAB0008CE790E060E070E044E150E00E942F13CA
:10CAC0008CE790E060E070E048E750E00E942F13B0
:10CAD0008CE790E060E070E04EE550E00E942F139C
:10CAE0008CE790E060E070E04DE650E00E942F138C
:10CAF0006CE17AE186E090E00E94FE638CE790E0D2
:10CB000060E070E04CE050E00E942F138CE790E072
:10CB100060E070E041E050E00E942F138CE790E06D
:10CB200060E070E046E050E00E942F136AE67AE091
:10CB300080E090E00E94FE630895DF93CF93CDB72D
:10CB4000DEB7A2970FB6F894DEBF0FBECDBFDE01F1
:10CB50001196E7EDF7E081E101900D928150E1F748
:10CB6000DE015296E8EEF7E081E101900D928150EE
:10CB7000E1F70E944865CE0101960E94F86482E0C8
:10CB80000E9415656AE67AE080E090E00E94FE630C
:10CB9000CE0142960E94F86460E17EEA88E290E06D
:10CBA0000E94FE6380E00E94276560E17EEA88E2E1
:10CBB00090E00E94FE6381E00E942765A2960FB676
:10CBC000F894DEBF0FBECDBFCF91DF910895DF9205
:10CBD000EF92FF920F931F93DF93CF9300D00F92AA
:10CBE000CDB7DEB7F82E042F122F213031F02230CE
:10CBF00031F0243031F0283031F080E005C081E0A0
:10CC000003C082E001C083E00C3059F00E3011F413
:10CC1000846007C0003111F4886003C0023109F458
:10CC20008C60613059F0623011F4806207C063306B
:10CC300011F4806403C0643009F48066682F606872
:10CC40008F2D90E070E0AE014F5F5F4F23E030E04A
:10CC50000E94471369E07AE180E090E00E94FE6361
:10CC600081E0F82A8F2D0E9411640E9490648983CC
:10CC70000E9490648A83023119F40E9490648B832D
:10CC80000E94906487FDF1CF0E949A640E947764AD
:10CC900069E07AE180E090E00E94FE638F2D0E94BF
:10CCA00011640E94906489830E9490648A83023197
:10CCB00019F40E9490648B830E9490642981023150
:10CCC00081F5622F70E080E090E03B814A8121FF96
:10CCD00012C0CB0177276627630F711D811D911D3F
:10CCE000342F20E040E050E0620F731F841F951F37
:10CCF0008C6F9F6F0FC0CB0177276627630F711D65
:10CD0000811D911D342F20E040E050E0620F731F21
:10CD1000841F951F0E94DE9920E83FEF4FEF57E4F4
:10CD20001FC0722F60E08A81680F711D882777FD10
:10CD30008095982F0E94DE990C3029F420E030EE87
:10CD40004FEF54E40DC00E3029F420E038EF4FEFE0
:10CD500055E406C0003131F420E03EEF4FEF56E4D9
:10CD60000E940E992FE632E143E050E40E94BC9B02
:10CD7000D62EE72EF82E092F612F70E0882777FD39
:10CD80008095982F0E94DE999B01AC016D2D7E2D20
:10CD90008F2D902F0E940E990F900F900F90CF9192
:10CDA000DF911F910F91FF90EF90DF900895E6E4DF
:10CDB000F1E08081208190813081829586958695F1
:10CDC000837022952F70822B832B92959F70892BD5
:10CDD0000895DF92EF92FF920F931F93DF93CF930B
:10CDE00000D0CDB7DEB780E06CE046E00E94BF6ABD
:10CDF00089E18093C4001092C50082E08093C00056
:10CE000080E00E94696B0E94EE6984B784B784B7A2
:10CE100084B784B7E7E7F1E322E432E43183208387
:10CE20003A968DB79EB70A97E817F907B8F300D07E
:10CE300000D089E29FE0ADB7BEB712969C938E9367
:10CE4000119789EF97E014969C938E9313970E9405
:10CE50008AA10F900F900F900F900E942B7A0E9442
:10CE6000095884EA97E060E070E00E94BD580E9493
:10CE70003A5CE0914408F091450809950E94D76614
:10CE800090E00E94697ACE0101960E941C69882375
:10CE900059F000D089E09FE0EDB7FEB7928381831F
:10CEA0000E948AA10F900F908E010F5F1F4FC80143
:10CEB0000E946A560E9426697C010E942B69BC016F
:10CEC000C701A8010E94766E0E9484680E945B6E72
:10CED0000E9430690E94E36F00D08CEF9EE0ADB7F6
:10CEE000BEB712969C938E9311970E948AA100D090
:10CEF000EDB7FEB7319608EF1EE0ADB7BEB712969C
:10CF00001C930E9311978A81828313820E948AA1B7
:10CF1000EDB7FEB73196ADB7BEB712961C930E9320
:10CF200011978981828313820E948AA10F900F90AA
:10CF300086EF9EE0EDB7FEB7928381830E948AA1BF
:10CF40000F900F900E946F7AE091C708F091C80887
:10CF50000995E091AE08F091AF080995E09170084D
:10CF6000F09171080995E090AC08F090AD0800913F
:10CF7000C5081091C6080E94586ED82E0E94EB6F0B
:10CF80002DB73EB72A5030400FB6F8943EBF0FBEC3
:10CF90002DBFEDB7FEB731962BED3EE0ADB7BEB776
:10CFA00012963C932E931197F382E28215830483A9
:10CFB000D6821782808711860E948AA1E091D108CB
:10CFC000F091D2082DB73EB7265F3F4F0FB6F894C9
:10CFD0003EBF0FBE2DBF3097D1F00995BC0100D0E8
:10CFE00000D088EC9EE0ADB7BEB712969C938E93AE
:10CFF000119780E890E00E949B9CEDB7FEB7748388
:10D0000063830E948AA10F900F900F900F9000D021
:10D0100086EC9EE0ADB7BEB712969C938E931197A7
:10D020000E948AA10F900F9080EF98E060E070E07E
:10D030000E94BD5880E797E00E94157900D08EEBE2
:10D040009EE0EDB7FEB7928381830E948AA10F9084
:10D050000F900F900F90CF91DF911F910F91FF9044
:10D06000EF90DF900895EF92FF920F931F9380E867
:10D0700080936100109261000E94E9660E94195835
:10D080000E948A6B8091F7289091F828009729F0E8
:10D0900001979093F8288093F728E090F928F09072
:10D0A000FA280091FB281091FC280E942B6AE616B2
:10D0B000F7060807190711F30E942B6A6093F928F5
:10D0C0007093FA288093FB289093FC28D7CF00D048
:10D0D00000D000D0EDB7FEB7319628EB3EE0ADB7FB
:10D0E000BEB712963C932E931197938382837583D8
:10D0F00064830E948AA18DB79EB706960FB6F894F6
:10D100009EBF0FBE8DBF08950F931F93DF93CF93E4
:10D11000CDB7DEB7A2970FB6F894DEBF0FBECDBF76
:10D120008EE490E00E94CDA289839A83982F9B5031
:10D13000903108F08A839A819095891709F470C01C
:10D1400000D084E69FE0ADB7BEB712969C938E9355
:10D1500011970E948AA18E010D5F1F4F0F900F90B3
:10D16000D80180E090E0FC01EC5BF04FE491ED939E
:10D17000019688309105B9F7F894CE0103966CE2D8
:10D1800070E048E050E00E94D3A2D80180E090E037
:10D19000FC01E45BF04FE491ED9301968E30910534
:10D1A000B9F7CE01039664E370E04EE050E00E94D0
:10D1B000D3A280E090E0FC01E65AF04FE491D80160
:10D1C000ED938D0101968A309105A9F7CE01039662
:10D1D00062E470E04AE050E00E94D3A280E590E073
:10D1E0006DEC7BEA0E94EBA282E590E060E070E0EB
:10D1F0000E94EBA284E590E060E00E94DDA28CE456
:10D2000090E060E070E00E94EBA28AE1898385EE05
:10D210008A8369817A818EE490E00E94EBA27894FF
:10D220008981A2960FB6F894DEBF0FBECDBFCF9115
:10D23000DF911F910F910895F8946CE270E042E045
:10D2400050E00E94B5A2789480E0089580E590E0D7
:10D250000E94CDA2089582E590E00E94CDA208959B
:10D2600084E590E00E94C5A208952091052930919F
:10D270000629409107295091082990E0A0E0B0E0EC
:10D28000280F391F4A1F5B1F209305293093062959
:10D2900040930729509308292091012930910229B0
:10D2A0004091032950910429280F391F4A1F5B1F01
:10D2B0002093012930930229409303295093042994
:10D2C0002091A52A2223A1F02091FD283091FE284B
:10D2D0004091FF2850910029280F391F4A1F5B1FDA
:10D2E0002093FD283093FE284093FF285093002977
:10D2F00008951F920F920FB60F920BB60F92112442
:10D300002F933F934F935F936F937F938F939F934D
:10D31000AF93BF93EF93FF938091BC139091BD1394
:10D3200001969093BD138093BC138091BE138F5FC1
:10D330008093BE138091BE138038A9F41092BE135F
:10D340008091052990910629A0910729B09108297B
:10D350000196A11DB11D8093052990930629A093E4
:10D360000729B09308298091A52A8823F1F080919C
:10D37000BF138F5F8093BF138091BF138038A9F4D0
:10D380001092BF138091FD289091FE28A091FF2854
:10D39000B09100290196A11DB11D8093FD289093A5
:10D3A000FE28A093FF28B09300290E94845B009779
:10D3B00011F00E94845AFF91EF91BF91AF919F911C
:10D3C0008F917F916F915F914F913F912F910F902E
:10D3D0000BBE0F900FBE0F901F901895F8941092EF
:10D3E000B60016BC83EF87BD82E084BD94E095BD96
:10D3F00095B395BB80936E00789408952091BC13EB
:10D400003091BD138091BC139091BD13281739073B
:10D41000A9F7C901089507C022E330E000002150B8
:10D420003040E1F701970097B9F708950F931F93E4
:10D43000CF93DF938C010E94FE69EC010E94FE698C
:10D440008C1B9D0B80179107C8F3DF91CF911F9123
:10D450000F91089508952091052930910629409152
:10D460000729509108298091052990910629A091BA
:10D470000729B0910829281739074A075B0759F788
:10D48000B901CA0108951F920F920FB60F9211248D
:10D4900010921D080F900FBE0F901F9018951F92AD
:10D4A0000F920FB60F920BB60F9211242F933F934A
:10D4B0004F935F936F937F938F939F93AF93BF939C
:10D4C000EF93FF93E0911308F09114088081E091AD
:10D4D0001E08F0911F08309709F00995FF91EF9110
:10D4E000BF91AF919F918F917F916F915F914F917C
:10D4F0003F912F910F900BBE0F900FBE0F901F907A
:10D5000018951F920F920FB60F92112410922A08AD
:10D510000F900FBE0F901F9018951F920F920FB68D
:10D520000F920BB60F9211242F933F934F935F935B
:10D530006F937F938F939F93AF93BF93EF93FF93DB
:10D54000E0912008F09121088081E0912B08F09172
:10D550002C08309709F00995FF91EF91BF91AF9199
:10D560009F918F917F916F915F914F913F912F91FB
:10D570000F900BBE0F900FBE0F901F90189590E06C
:10D580002DE030E0829FF001839FF00D929FF00D1F
:10D590001124ED5EF74FA281B3811C92A481B58165
:10D5A0006C93A681B78188ED8C93A085B1854C934F
:10D5B000128614861386089590E02DE030E0829F55
:10D5C000F001839FF00D929FF00D1124ED5EF74F57
:10D5D00081E08287A081B1816C933A968081882313
:10D5E000E9F708951F93182F8A3031F48091C01302
:10D5F0006DE00E94DC6A02C08D3029F08091C0137A
:10D60000612F0E94DC6A80E090E01F910895EF9204
:10D61000FF921F93CF93DF93182FE62EE7017E0131
:10D62000F72EE7010CC08A3021F4812F6DE00E94B3
:10D63000DC6A69916D3019F0812F0E94DC6A888163
:10D64000882389F7DF91CF911F91FF90EF90089584
:10D650000F931F93DF93CF93CDB7DEB7FE013A96BA
:10D6600001EC13E1C80160E470E0488559859F0131
:10D670000E941FA28F81B8010E94076BCF91DF919A
:10D680001F910F9108951F93CF93DF93182FEB01F4
:10D6900004C0812F0E94DC6A2196FE0164916623FA
:10D6A000C1F7DF91CF911F91089590E02DE030E018
:10D6B000829FF001839FF00D929FF00D1124ED5E8B
:10D6C000F74F748763870895682F80E00E94DC6AB3
:10D6D00008958093C01385E098E090937231809311
:10D6E0007131089584B7877F84BF88E10FB6F894BD
:10D6F00080936000109260000FBE08952FE088E1D3
:10D7000090E00FB6F894A895809360000FBE209328
:10D7100060000895A895089588E10FB6F894809365
:10D720006000109260000FBE0895F89428E088E130
:10D7300090E00FB6F894A895809360000FBE2093F8
:10D740006000FFCF8091182990E0FC01EE0FFF1FD1
:10D750009695982F882797958795E80FF91FE75E8C
:10D76000F64D10820895809110298091102990E043
:10D7700008958091390181FD0CC081E491E06FE151
:10D7800040E00E948C71813039F021E030E081313D
:10D7900029F020E030E002C021E030E0C901089526
:10D7A0008091390181FD12C081E491E06FE140E098
:10D7B0000E948C71982F8151823050F09F3141F03E
:10D7C000913041F081E0923031F402C081E008955F
:10D7D00080E0089580E008950E94D06B8823E1F3F3
:10D7E000089581E491E06FE140E00E948C7108951A
:10D7F000E9E3F1E0808180818D7F80838DE090E09E
:10D800000197F1F782E491E06FE140E023E00E94AC
:10D81000967183E090E00197F1F708950E94EC6B18
:10D820001092A52A0E94F86B809139018260809342
:10D8300039018091282B8823E9F1809194009091FF
:10D8400095002091392B30913A2B82179307A0F441
:10D850008091052B9091062BA091072BB091082B5E
:10D860008C57914EAF4FBF4F8093052B9093062B53
:10D87000A093072BB093082B809194009091950072
:10D88000821B930BA0E0B0E02091052B3091062B7A
:10D890004091072B5091082B820F931FA41FB51F97
:10D8A0008093052B9093062BA093072BB093082B06
:10D8B0001092282B80912A2B8823E9F180919400E3
:10D8C0009091950020913D2B30913E2B821793072C
:10D8D000A0F480910D2B90910E2BA0910F2BB09165
:10D8E000102B8C57914EAF4FBF4F80930D2B9093C1
:10D8F0000E2BA0930F2BB093102B8091940090913E
:10D900009500821B930BA0E0B0E020910D2B30918D
:10D910000E2B40910F2B5091102B820F931FA41FA1
:10D92000B51F80930D2B90930E2BA0930F2BB093CC
:10D93000102B10922A2B08958091A52A882381F01C
:10D9400080910114882321F40E94D06B882331F444
:10D9500081E08093841421E030E004C00E940E6CCA
:10D9600020E030E0C90108950F931F93182F8830ED
:10D9700049F0863039F0893029F0863119F0893143
:10D9800009F041C08091390181FD40C00E94EC6BDB
:10D990000E94F16B082F181709F43BC0183019F4D6
:10D9A0000E94F86B29C0193141F48631A9F482E450
:10D9B00091E06FE140E029E009C0163169F4893156
:10D9C00059F482E491E06FE140E026E00E94967114
:10D9D000E3E0F0E03197F1F782E491E06FE140E0BD
:10D9E000212F0E949671083019F4E9E6F1E002C097
:10D9F000E3E0F0E03197F1F70E94F16B811749F015
:10DA000023E430E008C022E430E005C024E430E044
:10DA100002C020E430E0C9011F910F910895809168
:10DA200094009091950090933E2B80933D2B21E0A4
:10DA300020932A2B8091390181FF15C02093A42ABD
:10DA4000809194009091950090933A2B8093392B7C
:10DA50002093282B809139018D7F8093390180910B
:10DA6000A42A8823E1F786E10E94B46C81E08093C8
:10DA7000A52A08958091A52A882351F48091011444
:10DA8000882321F081E08093831402C00E940F6DEF
:10DA900081E090E008951F93DF93CF930F92CDB76D
:10DAA000DEB78FB7898380910114882331F5F8940C
:10DAB0008091A52A882351F08091390181FD1BC0F6
:10DAC0000E94D06B8823B9F080E003C00E943A6DB9
:10DAD00081E0909147019E3010F010E001C01FEFEF
:10DAE000882311F00E949C6C16FF05C089818FBFAE
:10DAF00021E030E004C089818FBF20E030E0C9011F
:10DB00000F90CF91DF911F91089580918314882306
:10DB100021F00E940F6D1092831480918414882349
:10DB200021F00E940E6C109284141092011408953A
:10DB3000EF92FF92CF93DF93B82FA92FF62FE72F05
:10DB400081E0809301142091E92A3091EA2A4091E2
:10DB5000EB2A5091EC2A2F5F3F4F4F4F5F4F20939E
:10DB6000E92A3093EA2A4093EB2A5093EC2A862F35
:10DB70008E5F87FF0CC08091A22A9091A32A019604
:10DB80009093A32A8093A22ACFEFDFEF0BC022E06D
:10DB900034E1C9016B2F7A2F4F2F5E2F0E94EAA02C
:10DBA000C0E0D0E00E94856DCE01DF91CF91FF9063
:10DBB000EF9008959091390191FD0AC0282F80318E
:10DBC00008F02FE085E491E06FE040E00E9496715C
:10DBD00008958093861408950E94F16B82508131DC
:10DBE00030F4E82FF0E0E85AF74F8081089581E0A3
:10DBF000089508958FEF80934E018CE691E060EFD9
:10DC000044E022E00E9496718CE290E06EE041E0F8
:10DC100025E00E94967180E880936F018091460113
:10DC200080936D0184E491E060E245E021E00E9490
:10DC300096710895CF93DF93CDEFD3E0CE01019796
:10DC4000F1F70E9482711092192910929B2910926B
:10DC50001D2A1092182910921729E9E3F1E080811A
:10DC60008E7F808380818D7F80838DE090E001971F
:10DC7000F1F780818160808382E491E06FE140E090
:10DC800023E00E9496712197F1F780915D018091C8
:10DC90005E010E94FA6D8AE398E060E070E00E9405
:10DCA000BD580E940F6D81E090E0DF91CF91089503
:10DCB000809185140895DF93CF930F92CDB7DEB78F
:10DCC00089830E94EC6B29812093851488E491E07C
:10DCD0006FE140E00E9496710F90CF91DF9108951F
:10DCE0000E945B6E86E00E94B46C0895809362018E
:10DCF0009093630160936001709361014115510538
:10DD000031F1FA01819180936B01DA0111968C91C6
:10DD100080936A01DF011196818180936901FD0181
:10DD2000319611968C9180936801DF011196818163
:10DD300080936701FD01319611968C911197809324
:10DD400066018181809365018281809364010895D9
:10DD50008AE398E00E94E05881E080931029809146
:10DD600011299091122901969093122980931129DB
:10DD700081E090E00895EF92FF92CF93DF9350916E
:10DD80001829252F30E0F901EE0FFF1F3695322FAD
:10DD9000222737952795E20FF31FE75EF64D408166
:10DDA000442309F4CEC02091390121FDCAC020913D
:10DDB000A52A222309F4C5C047FF16C00E94A26B02
:10DDC0008091D92A9091DA2AA091DB2AB091DC2A9D
:10DDD0000196A11DB11D8093D92A9093DA2AA093B0
:10DDE000DB2AB093DC2AADC04330B0F40E94A26BB2
:10DDF0008091D52A9091D62AA091D72AB091D82A7D
:10DE00000196A11DB11D8093D52A9093D62AA09387
:10DE1000D72AB093D82A95C0C42FD0E022976C1788
:10DE20007D07B0F40E94A26B8091D12A9091D22AF2
:10DE3000A091D32AB091D42A0196A11DB11D80933F
:10DE4000D12A9093D22AA093D32AB093D42A79C00E
:10DE5000652F70E09B01220F331F7695762F662782
:10DE600077956795260F371F265E364DB90150E02E
:10DE70000E94EAA020911829822F90E0FC01EE0F69
:10DE8000FF1F9695982F882797958795E80FF91F7C
:10DE9000E756F64D808180930929822F90E0FC019E
:10DEA000EE0FFF1F9695982F882797958795E80F77
:10DEB000F91FE75EF64D10822F5F2093182923305B
:10DEC00010F0109218298091182990E0FC01EE0FB3
:10DED000FF1F9695982F882797958795E80FF91F2C
:10DEE000E75EF64D8081882311F00E94A86E609154
:10DEF000470160930A2980910F29882311F0681740
:10DF000010F460930F2984E070E00E947C606091BF
:10DF1000092983E070E00E947C608091ED2A909155
:10DF2000EE2AA091EF2AB091F02A0196A11DB11D11
:10DF30008093ED2A9093EE2AA093EF2AB093F02AD3
:10DF400002C0C0E0D0E0CE01DF91CF91FF90EF9012
:10DF50000895CF93DF93EC0188819981009729F090
:10DF600024E08B3F920739F505C08BEF94E099834D
:10DF7000888325C0623819F5109210290E94F65F37
:10DF80000E94535F60E870E00E94BB6E181619068D
:10DF900044F40E944E5FE091CB08F091CC080995C3
:10DFA000E4CF80910D2990910E29019690930E292E
:10DFB00080930D29DACF1982188283E001C081E0B5
:10DFC000DF91CF91089591E0909301140E94DA6D52
:10DFD0000E94856D08958091390181FD07C085E417
:10DFE00091E06FE040E00E948C71089580E1089517
:10DFF000CF92DF92EF92FF920F931F93CF93DF9315
:10E00000182F21E0209301140091A52A8091390155
:10E0100081FF16C0809194009091950090933A2BC7
:10E020008093392B2093282B2093A42A80913901A7
:10E030008D7F809339018091A42A8823E1F700E045
:10E040000E94EC6B8091A52A882309F441C080913D
:10E050002A2B8823E9F1209194003091950080913A
:10E060003D2B90913E2B28173907A0F420910D2BC2
:10E0700030910E2B40910F2B5091102B2C57314E7D
:10E080004F4F5F4F20930D2B30930E2B40930F2B50
:10E090005093102B2091940030919500281B390B40
:10E0A00040E050E0C0900D2BD0900E2BE0900F2B55
:10E0B000F090102B2C0D3D1D4E1D5F1D20930D2B40
:10E0C00030930E2B40930F2B5093102B10922A2B32
:10E0D00089E10E94B46C86E00E948760009751F04D
:10E0E0000E94EB6FC82F86E00E94876081500E94DB
:10E0F000DA6D02C0C0E0D0E080919400909195006C
:10E1000090933C2B80933B2B81E08093292BF894B8
:10E1100080913901826080933901809139018D7F2E
:10E1200080933901612F6E5F82E094E10E94C77194
:10E13000789480919F2A9091A02A01969093A02A8A
:10E1400080939F2A0E94EC6B82E491E060EE45E0B0
:10E150000E948C71182F86E00E948760009719F04A
:10E160008C2F0E94DA6D002319F00E940F6D02C0FF
:10E170000E940E6C8091292B8823E9F180919400F4
:10E180009091950040913B2B50913C2B8417950723
:10E19000A0F48091092B90910A2BA0910B2BB091A8
:10E1A0000C2B8C57914EAF4FBF4F8093092B909300
:10E1B0000A2BA0930B2BB0930C2B20919400309141
:10E1C0009500241B350B40E050E08091092B909185
:10E1D0000A2BA0910B2BB0910C2B280F391F4A1F33
:10E1E0005B1F2093092B30930A2B40930B2B5093EA
:10E1F0000C2B1092292B8091A52A882361F0809105
:10E2000094009091950090933E2B80933D2B81E05C
:10E2100080932A2B07C082E491E06FE140E023E085
:10E220000E9496710E94856D1130E1F01330A9F4BF
:10E230008091E12A9091E22AA091E32AB091E42A08
:10E240000196A11DB11D8093E12A9093E22AA0932B
:10E25000E32AB093E42A12E00AC0153029F01730FF
:10E2600031F404C010E003C013E001C011E0812FBD
:10E2700090E0DF91CF911F910F91FF90EF90DF9091
:10E28000CF900895CF93DF93EB010E94986D9C018E
:10E29000009731F4CE010E94F86F9C01009749F07D
:10E2A0008091A22A9091A32A01969093A32A809309
:10E2B000A22AC901DF91CF9108950F931F938091F6
:10E2C000A52A882321F40E943A6D11E001C010E0D4
:10E2D0000E94F16B863111F0813119F400914701F0
:10E2E00009C086E491E06FE140E00E948C71082F44
:10E2F000000F080F112311F00E949C6C802F1F91BA
:10E300000F9108951092881410928714EFE6F0E0B0
:10E310008081806280830895FC018081862390E063
:10E3200002C0959587954A95E2F70895F894FC0107
:10E330009081862F8095892330E002C0220F331F01
:10E340004A95E2F72623282B208378940895DC0150
:10E35000119620917B01FC012083215030E0A9011E
:10E360004F575E4FE0E8F1E061916D93E417F507D8
:10E37000D9F7FC01E058FF4F2F573E4FD9012C91A0
:10E3800020838F579F4F21E0FC0120830895FC01DB
:10E390006093800101966350860F911DA1E8B1E062
:10E3A00021912D93E817F907D9F708951F920F923D
:10E3B0000FB60F920BB60F9211242F933F934F93EA
:10E3C0005F936F937F938F939F93AF93BF93EF93DD
:10E3D000FF938091470180930A292091172930E00B
:10E3E000C901880F991F3695322F22273795279517
:10E3F000820F931F875E964D0E94A7718091172907
:10E400008F5F80931729833010F0109217290E9494
:10E41000A86EFF91EF91BF91AF919F918F917F91E6
:10E420006F915F914F913F912F910F900BBE0F9085
:10E430000FBE0F901F9018951F920F920FB60F925C
:10E4400011240F900FBE0F901F9018951F920F92DE
:10E450000FB60F9211240F900FBE0F901F901895BA
:10E460001F920F920FB60F9211240F900FBE0F90B4
:10E470001F9018951F920F920FB60F9211241092B1
:10E48000A42A0F900FBE0F901F9018951F920F9205
:10E490000FB60F9211241092A42A0F900FBE0F9066
:10E4A0001F9018951F920F920FB60F9211248F9301
:10E4B00081E0809310298F910F900FBE0F901F90D5
:10E4C00018951F920F920FB60F9211241092A42A42
:10E4D0000F900FBE0F901F9018951F920F920FB6BE
:10E4E0000F9211248F939F93809187149091881499
:10E4F000019690938814809387149F918F910F9029
:10E500000FBE0F901F9018950F931F93CF93DF931B
:10E510008091AD2A9091AE2AA091AF2AB091B02AF5
:10E520000196A11DB11D8093AD2A9093AE2AA093B0
:10E53000AF2AB093B02A0E943575EC0189E894E1C6
:10E540000E9482590BC0D8011296ED91FC9113974D
:10E55000309709F00995C8010E94485A082F192FD1
:10E560000115110581F7209719F0CE010E94F2568E
:10E57000DF91CF911F910F9108950E946F7A0E94B1
:10E58000F65F0E943F738CEA98E09093A82A8093EC
:10E59000A72A0E94327582E090E060E074E040E0DB
:10E5A0005EE12FEF31E00E94F3740895CF92DF9285
:10E5B000EF92FF920F931F93CF93DF936C01EB01C8
:10E5C0008A0189E894E10E9482590CC0D70114960F
:10E5D000ED91FC911597309711F0CE010995C70187
:10E5E0000E94485AE82EF92EE114F10479F7C60189
:10E5F000BE01A8010E94FA56DF91CF911F910F91A1
:10E60000FF90EF90DF90CF900895BC0189E894E1EE
:10E610000E94095A0895BC0189E894E10E94D059EA
:10E620000895CF93DF93EC018091A92A9091AA2AB3
:10E63000A091AB2AB091AC2A0196A11DB11D809387
:10E64000A92A9093AA2AA093AB2AB093AC2ACE0110
:10E650000E944C75009769F00E94705FE091B008CD
:10E66000F091B10886ED92E7BE01099521E030E016
:10E6700002C020E030E0C901DF91CF9108958BE81E
:10E6800094E10E947E5908950F93CF93DF93EC019C
:10E690007B836A8318865F834E838BE894E1BE0197
:10E6A0000E94095AE0918D14F0918E14309749F030
:10E6B0004C815D818A819B81688520E030E001E0AA
:10E6C0000995DF91CF910F910895BC018BE894E1FA
:10E6D0000E94D05908950F93DC0118961C92189748
:10E6E000E0918D14F0918E14309759F012968D911F
:10E6F0009C91139760E040E050E020E030E000E0C3
:10E7000009950F9108950F93DC01AB0114962D919B
:10E710003C91159781E018968C93189715967C93E9
:10E720006E931497E0918D14F0918E14309739F018
:10E7300012968D919C91139761E000E009950F91DD
:10E7400008950F93DC01E0918D14F0918E143097B1
:10E7500069F014962D913C91159712968D919C918C
:10E76000139718966C91A90101E009950F910895EE
:10E77000E0918F14F0919014309709F00995089565
:10E780009093901480938F14089590938E14809397
:10E790008D1408958BE894E10E9482590895EF92B8
:10E7A000FF920F931F93CF93DF938C01EB017A01BC
:10E7B0008BE894E10E94825915C0DC0112962D91DC
:10E7C0003C9113972C173D0759F41696ED91FC9147
:10E7D0001797309761F0B801AE019701099507C00E
:10E7E0000E94485A282F392FC901009731F7DF912D
:10E7F000CF911F910F91FF90EF9008950895AF92E0
:10E80000BF92CF92DF92EF92FF920F931F93DF930D
:10E81000CF9300D0CDB7DEB75B010E94535FFC0100
:10E82000008111811A8309830C30110518F4EE243C
:10E83000FF242EC000D000D084E798E0EDB7FEB7EB
:10E8400092838183148303830E9478A10F900F9099
:10E850000F900F9020C00E94535FF701EE0FFF1F33
:10E86000EE0FFF1FE80FF91FC280D3800E94535F95
:10E870000894E11CF11CF701EE0FFF1FEE0FFF1FC4
:10E88000E80FF91F40815181C501B6010E94CF7385
:10E89000E016F10600F30F900F90CF91DF911F91DA
:10E8A0000F91FF90EF90DF90CF90BF90AF900895C1
:10E8B000CF93DF93CCEAD4E16091C2147091C3147A
:10E8C000CE014AE854E720E030E00E94475C0E9415
:10E8D0006C7A6091C2147091C3140E949B9CBC011D
:10E8E000CE0140974FE954E720E030E00E94475CBA
:10E8F000DF91CF9108950F93013051F48091BC14B2
:10E900009091BD149093C3148093C2140E945874C4
:10E910000F9108958091C2149091C3142091C01456
:10E920003091C114880F991F2817390708F4C901BD
:10E930009093C3148093C2140E9458740895EF9268
:10E94000FF92CF93DF930E94F65F0E94535FE82E01
:10E95000E7017E01F92EE701198218820E94CA732D
:10E9600026C028813981F901EE0FFF1FEE0FFF1F2E
:10E97000EC0FFD1FDC0112964D915C9113975383B0
:10E9800042832F5F3F4FF901EE0FFF1FEE0FFF1F76
:10E99000EC0FFD1F14964D915C91159751834083A8
:10E9A000398328830E94485A282F392FC90100979C
:10E9B00021F0FC0120852223A1F688819981880F0E
:10E9C000991F880F991F02960E944E5F8881998136
:10E9D000009721F081E994E10E94C556DF91CF9123
:10E9E000FF90EF900895EF92FF920F931F93CF93B4
:10E9F000DF93FC018B017A01E90181E994E1BF0118
:10EA000041E958E00E94A7561093BD140093BC142E
:10EA1000F092BF14E092BE14D093C114C093C014FE
:10EA20008BE794E70E94C573DF91CF911F910F91FF
:10EA3000FF90EF900895CF93DF93CCEAD4E1CE011D
:10EA40000E94CE5CCE0140970E94CE5CCE014B97D7
:10EA50000E94C256DF91CF9108958091C214909187
:10EA6000C31408950E9406570895EF92FF92CF9322
:10EA7000DF93E0919508F09196080995EC010097D5
:10EA800029F06A817B8181E00E947C60CE01DF9168
:10EA9000CF91FF90EF9008950F931F93CF93DF9343
:10EAA0008C01E0919708F09198080995EC01F80124
:10EAB0006281738181E00E947C6021E030E02097D8
:10EAC00011F420E030E0C901DF91CF911F910F9147
:10EAD0000895E0919908F0919A0809950895FC012C
:10EAE00020E030E004C08181280F311D3296808102
:10EAF0008823C9F7C9010895FC01818190E0308124
:10EB000020E0822B932B02C0880F991F6A95E2F7B1
:10EB1000892F9927FA01E556F74F208130E08223AB
:10EB2000932328E030E0241B350B02C0969587958F
:10EB30002A95E2F708956F927F928F929F92AF92FB
:10EB4000BF92CF92DF92EF92FF920F931F93CF93DA
:10EB5000DF936C017B015A0189012830310544F4AF
:10EB6000CB01BA01A9010E947C75F601808341C0E6
:10EB7000390133E0759467943A95E1F741155105F1
:10EB800021F04C01C0E0D0E016C0DB01FC01C0E088
:10EB9000D0E08D9181932196C615D705D4F3A801B5
:10EBA000477050704115510521F1C7018C0F9D1F11
:10EBB00060E070E019C0C7018C0F9D1FB50148E0EF
:10EBC00050E00E947C75F40181934F012196C61597
:10EBD000D7058CF3A801477050704115510549F0D5
:10EBE000C7018C0F9D1FB5010E947C75CC0DDD1DEA
:10EBF0008883DF91CF911F910F91FF90EF90DF906D
:10EC0000CF90BF90AF909F908F907F906F9008951E
:10EC10004F925F926F927F928F929F92AF92BF922C
:10EC2000CF92DF92EF92FF920F931F93DF93CF93D8
:10EC300000D000D0CDB7DEB70E94535FE82E092F79
:10EC400082E090E00E942F5F009709F464C0EE2DEF
:10EC5000F02F918180E02081820F911D0E941A5730
:10EC60007C01009709F459C00E94535F3C01F701F1
:10EC70004681242F30E02770307081E090E021152C
:10EC8000310511F480E090E0469546954695840F55
:10EC9000911D0E942F5F0097F1F1F701048115810A
:10ECA000CC24DD2453E0452E512C4C0E5D1E4E012C
:10ECB0000894811C911C2AC0F801A180BB24B601D4
:10ECC00043E0759567954A95E1F7660D771DA601B6
:10ECD00047705070883150F0C40195010E949B75B7
:10ECE000F8018081B4010E9490600CC01C821B82DC
:10ECF000C20195010E949B756B817C81F801808126
:10ED00000E947C60CA0CDB1C0E5F1F4FF8018081E3
:10ED1000882391F602C0EE24FF24C7010F900F90C4
:10ED20000F900F90CF91DF911F910F91FF90EF9077
:10ED3000DF90CF90BF90AF909F908F907F906F901B
:10ED40005F904F900895FC0150E080E190E0861BB9
:10ED5000970B821B930B02C0440F551F8A95E2F755
:10ED60008081852B80838181842B818308956F929C
:10ED70007F928F929F92AF92BF92CF92DF92EF924B
:10ED8000FF920F931F93CF93DF938C015B016A0176
:10ED900079012830310524F4C801FA01408156C0B8
:10EDA000390163E0759467946A95E1F7A114B104A1
:10EDB00021F04A01C0E0D0E021C0DA01F80180E092
:10EDC00090E02D912193019686159705D4F3970134
:10EDD0002770307021153105D9F1F601E80FF91FC0
:10EDE000408150E068E070E0621B730B02C05595F3
:10EDF00047956A95E2F7800F911F26C0F401419173
:10EE00004F01C8018C0F9D1FB50128E030E00E9422
:10EE1000A3762196C615D7058CF39701277030701D
:10EE200021153105A9F0F601EC0FFD1F408150E0DE
:10EE3000C5010896821B930B02C0559547958A958C
:10EE4000E2F7C8018C0F9D1F60E070E00E94A3767E
:10EE5000DF91CF911F910F91FF90EF90DF90CF90B6
:10EE6000BF90AF909F908F907F906F9008954F923A
:10EE70005F926F927F928F929F92AF92BF92CF924A
:10EE8000DF92EF92FF920F931F93DF93CF9300D007
:10EE9000CDB7DEB78C01DC0116964C911697842F06
:10EEA00090E08770907021E030E0009711F420E04E
:10EEB00030E04695469546957901E40EF11CC70170
:10EEC00002960E94BB5F009709F453C00E945B5FEB
:10EED000FC01D80112968C911297808313968C9125
:10EEE00081830E945B5FF2E06F2E712C680E791EA9
:10EEF000C30160E070E0A7010E94F3A0F801C480A4
:10EF0000D58000E010E02E010894411C511C2AC05D
:10EF1000D60111968C90119799247801E3E0F5942D
:10EF2000E794EA95E1F7E60CF71C77E0A72EB12C01
:10EF3000A022B122883130F00E949A60AC01C70152
:10EF4000B50107C00E9487609A838983C701B50114
:10EF5000A20194010E94B776080D191DE2E0F0E0CD
:10EF6000CE0EDF1ED6018C91882391F621E030E091
:10EF700002C020E030E0C9010F900F90CF91DF91E7
:10EF80001F910F91FF90EF90DF90CF90BF90AF90C7
:10EF90009F908F907F906F905F904F900895E09139
:10EFA000C908F091CA0809950895E0917208F09196
:10EFB000730809950895E091CD08F091CE08099560
:10EFC0000895E091CF08F091D0080995089580E068
:10EFD00090E008950895E0915408F091550809953E
:10EFE0000895009731F0E0915408F0915508099583
:10EFF0000895E0915608F09157080995089580E02A
:10F0000090E008950F931F93DF93CF93CDB7DEB7B2
:10F01000E0970FB6F894DEBF0FBECDBF0E94A55F8C
:10F020008C010E94535F602FAE014F5F5F4F0E94C3
:10F030003580882309F445C088A99801281B310927
:10F04000C9010E942F5F0097E1F12E81222371F107
:10F050008A859B853BEA8D3C930721F03FEF8F3FEC
:10F06000930779F5223041F088E090E007C00197DE
:10F0700022912F3F41F00BC082E090E0FE01E80FAB
:10F08000F91F3C96F4CF181619068CF30FC089E1CE
:10F09000BE01645F7F4F0E94906089E10E949A6088
:10F0A00066EB78E20E945856009759F088E1BE015D
:10F0B0006A5E7F4F0E949060E091B208F091B308C1
:10F0C0000995E0960FB6F894DEBF0FBECDBFCF9185
:10F0D000DF911F910F910895AF92BF92CF92DF926F
:10F0E000EF92FF920F931F93DF93CF93CDB7DEB7CD
:10F0F000E0970FB6F894DEBF0FBECDBF6C018B0159
:10F10000FE01319680E3DF011D928A95E9F781E0E7
:10F1100089838CE00E9487608C831D821F8280918E
:10F12000C61489878F5F8093C61483E0E82EE88633
:10F130008DEC9BEA9B878A8789E10E949A606CE844
:10F1400077E00E945856009731F082E08E838FEF6F
:10F150008C878D8709C089E10E949A60BC01CE012D
:10F160000C960E944F56EE828DEC9BEA9D8B8C8B09
:10F17000CE01469666EB78E20E944F560E94535F9E
:10F180009FA78EA70E94A55F88AB7E010894E11C13
:10F19000F11CC7010E942C7FA82E90E00E94BB5F4B
:10F1A000009741F10E945B5FBC01C7014A2D0E949C
:10F1B0004A7FA0904A08B0904B080E945B5F7C0198
:10F1C0000E94AF5FBC01C701F5010995C114D104CC
:10F1D00089F0009721F08130910561F404C0C801E5
:10F1E00060E070E003C0C80164E070E041E050E01E
:10F1F000F6010995E0960FB6F894DEBF0FBECDBFBD
:10F20000CF91DF911F910F91FF90EF90DF90CF9002
:10F21000BF90AF9008950E946C7A8093C614E091DD
:10F220005408F091550809950895EF92FF92CF93F5
:10F23000DF93E82EE7017E01F92EE70104C060E0CC
:10F2400070E00E94BD58899199910097C1F7DF91B4
:10F25000CF91FF90EF900895EF92FF92CF93DF93BD
:10F26000E82EE7017E01F92EE70102C00E94025854
:10F27000899199910097D1F7DF91CF91FF90EF900D
:10F280000895CF93DF93EC017B836A830E94FE692C
:10F2900099838883DF91CF910895FC0180819181CA
:10F2A00022813381820F931F918380830895CF93AE
:10F2B000DF93EC010E94FE6999838883DF91CF91EF
:10F2C0000895CF93DF93EC010E94FE692881398174
:10F2D000821B930B019621E030E04A815B81481745
:10F2E000590710F020E030E0C901DF91CF91089577
:10F2F000EF92FF92CF93DF93FC01C281D381808193
:10F300009181C80FD91F0E94FE69C81BD90BCE017D
:10F31000DF91CF91FF90EF900895CF93DF93EFE2CD
:10F32000FBE2C1EFDAE2A3E2BBE211921192199281
:10F330001992199219921D928BE2E734F807A9F7F6
:10F34000DF91CF9108950F931F93CF93DF93FC012B
:10F35000DC01AD5DB44D8C91882339F100919400AE
:10F3600010919500EF01CC0FDD1FCC0FDD1FCF50AA
:10F37000D54DDF01AA0FBB1FA15DB44D8D919C91AE
:10F3800011979801281B390B40E050E06881798182
:10F390008A819B81260F371F481F591F2883398375
:10F3A0004A835B8311961C930E93EE0FFF1FEE0FA3
:10F3B000FF1FEF50F54D6081718182819381DF9154
:10F3C000CF911F910F91089560E070E0CB010895F7
:10F3D000FC01EE0FFF1FEE0FFF1FEF50F54D4083B6
:10F3E0005183628373830895EF92FF920F931F936B
:10F3F000CF93DF9323E23BE2C1EFDAE2EFE2FBE2FD
:10F40000D9018D919D018823C9F0409194005091BC
:10F410009500808191817A01E81AF90A00E010E0F4
:10F4200088819981AA81BB818E0D9F1DA01FB11F6C
:10F4300088839983AA83BB83518340832496329621
:10F44000BBE22F323B07E1F6DF91CF911F910F9185
:10F45000FF90EF9008950E94A97E08950F931F9347
:10F46000FC01CB014091C7145091C814338322830F
:10F470001583048371836083F093C814E093C714E9
:10F480004115510511F40E94C37E80E090E01F9168
:10F490000F9108958091C7149091C8140097C1F0FE
:10F4A0001092C8141092C714DC0114966D917C91CF
:10F4B00015971296ED91FC9113970995E091C71459
:10F4C000F091C814309721F0808191810E94C37E11
:10F4D00008950E94899D08950E94849D089583ED5A
:10F4E00098E00E94F6588BED98E00E94F658089537
:10F4F000EF92FF92CF93DF930E94625F0097C9F073
:10F500008BED98E00E941659E82EE7017E01F92E56
:10F51000E701209731F10E94A55F998388830E94BB
:10F52000A05F9B838A83C70104960E94CE5E8CAB4A
:10F5300018C083ED98E00E941659EC017E01F92E67
:10F54000E701209771F0C70102960E94E55E99835A
:10F550008883B7016E547F4FC7018E579F4F0E941B
:10F560005260CE01DF91CF91FF90EF900895BC01E2
:10F570006E547F4F8E579F4F0E9452600895CF93D5
:10F58000DF93EC0183ED98E0BE010E946159009782
:10F5900019F083ED98E009C08BED98E0BE010E9460
:10F5A0006159009729F08BED98E0BE010E943C590B
:10F5B000DF91CF910895EF92FF92CF93DF93EC010B
:10F5C00083ED98E0BE010E946159009779F068814F
:10F5D0007981CE0102960E941F60BE016E547F4F5A
:10F5E000CE018E579F4F0E9467601BC08BED98E045
:10F5F000BE010E9461590097A1F00E94F65F6881E8
:10F6000079818A819B810E941F608CA990E00E9471
:10F61000BB5F0E945B5F4CA92496BE0150E00E9434
:10F62000EAA0DF91CF91FF90EF900895EF92FF92C3
:10F63000CF93DF93EC0183ED98E0BE010E94615906
:10F64000009711F022960DC08BED98E0BE010E944C
:10F650006159009721F00A80DB81C02D02C0C0E013
:10F66000D0E0CE01DF91CF91FF90EF900895FC01A3
:10F6700080819181089570E06F5B7F4F660F771FE7
:10F68000680F791FCB010895E62FF0E0EF5BFF4F85
:10F69000EE0FFF1FE80FF91F8081918108950895F3
:10F6A0008FE19BE10E946C5B009721F08FE19BE171
:10F6B0000E94575B0895E0912C1BF0912D1B309711
:10F6C00011F00995089580E00895EF92FF920F934D
:10F6D0001F93CF93DF93EC018A0188819981009772
:10F6E00031F023E08C30920709F006C12BC080E096
:10F6F0000BC0E82FF0E0EE0FFF1FEE0FFF1FE35FE0
:10F70000F44E118210828F5F843098F38093271B10
:10F7100080914E1290914F1290931E1B80931D1B4F
:10F720000E94FB578093472B8FE19BE160E470E0E0
:10F730000E94415B0E94C4818CE093E0998388839E
:10F7400081E0DDC0623009F4B9C0633030F4662373
:10F7500009F489C0613081F79CC0673819F06838B6
:10F7600059F741C01092281B4DE0E42E4BE1F42ED6
:10F7700018C0F701828193818017910749F4808135
:10F7800091810E940B83F7011182108213821282F1
:10F7900084E090E0E80EF91E8091281B8F5F809333
:10F7A000281B8091281B843020F3E7E5F0E3848D4B
:10F7B000958D8017910719F4158E148E118EB096C1
:10F7C00090E3E73DF90799F7EDEEF0E38185928547
:10F7D0008017910711F4158214823D9621E3EF36CC
:10F7E000F207A1F7A9CF8BE14F31580709F0A4CF59
:10F7F000CA010E946C5B009709F49ECF1092281BEF
:10F800002DC0F0E035E0EE0FFF1F3A95E1F7E95A21
:10F81000FF4C818D8823E9F08FE19BE10E94575BCB
:10F820008091281B90E025E0880F991F2A95E1F729
:10F83000895A9F4C909356308093553082E00E94B5
:10F840003F838091482B9091492B009711F00E94A3
:10F850005B7B8091281B8F5F8093281BE091281B86
:10F86000E43078F269CF4115510509F465CF509322
:10F8700056304093553083E00E943F838091482B5F
:10F880009091492B009711F00E945B7B0E94507B66
:10F8900053CF4115510509F44FCF50935230409347
:10F8A000513085E00E943F838091482B9091492BF5
:10F8B000009709F441CF0E945B7B3ECF8091482B9B
:10F8C0009091492B009709F437CF8091592B8630BE
:10F8D00031F48091712B81FF02C00E94507B81E046
:10F8E0000E943F838091482B9091492B009709F407
:10F8F00023CF0E948E7D20CF1982188283E0DF9172
:10F90000CF911F910F91FF90EF90089590932D1B31
:10F9100080932C1B089520914E1230914F1260E07D
:10F92000EDE0FBE113C0408151814817590761F4B4
:10F93000428153814217530739F460932B1B118284
:10F9400010820E940B83089534966F5F643058F3E1
:10F9500060932B1B089540E0EDE0FBE116C0542FAF
:10F960005F5F208131812115310569F440932A1BA5
:10F970009183808320914E1230914F1233832283E2
:10F980000E94258308953496452F443040F34093D8
:10F990002A1B0895FC0180914E1290914F12958F71
:10F9A000848F778F668F0895FC0180914E1290911D
:10F9B0004F1292878187748763870895CF93DF936F
:10F9C000EA010E948782FC01009741F080914E126B
:10F9D00090914F1292878187D487C387CF01DF919F
:10F9E000CF9108950F931F93DF93CF9300D000D052
:10F9F000CDB7DEB78C01AB018FEF89838A838B8310
:10FA00008C83CE010196B8010E94DE7CFC01009738
:10FA100011F015830483CF010F900F900F900F907A
:10FA2000CF91DF911F910F91089580EF98E062E0F0
:10FA300040E050E00E94AE581092492B1092482BA3
:10FA40000895AC0180EF98E061E00E948B58089522
:10FA5000AC0180EF98E060E00E948B5808950F930E
:10FA60001F93CF93DF93EA010E94FD818C010097E1
:10FA700061F080914E1290914F12F801958F848F12
:10FA8000D78FC68FC8010E94287DC801DF91CF9112
:10FA90001F910F910895CF93DF93A0915530B091AE
:10FAA0005630109719F0ED016C9605C0C091513099
:10FAB000D091523029968091503086FF22C010920A
:10FAC000291B40E0EDE0FBE116C020813181149656
:10FAD0008D919C9115972817390759F4828193814C
:10FAE000009739F04093291B998388831B821A82DF
:10FAF00006C034964F5F443040F34093291B0E9468
:10FB0000507B88819981009731F04A815B816091B7
:10FB1000472B0E94AE58DF91CF9108950F931F930A
:10FB2000CF93DF938091592B863009F074C0809178
:10FB3000482B9091492B25E08030920709F06BC04B
:10FB4000C4E9D2E0D093492BC093482B02E0009344
:10FB5000522B14E91093532B1092752B1092742B87
:10FB60000E94BC81809590959093752B8093742B07
:10FB700010925B2B10925A2B0E94AB81809590952E
:10FB800090935B2B80935A2B0E945B7BD093492BE5
:10FB9000C093482B0093522B1093532B90915330CA
:10FBA00080915430E92FF82FDF01A459BD4F8CE626
:10FBB00092E00D9001920197E1F788E69BE26CE6F6
:10FBC00072E00E944F8180914C2B8093682B809132
:10FBD0004D2B8093692B80914E2B80936A2B8091C3
:10FBE0004F2B80936B2B1092752B1092742B0E94CD
:10FBF000BC81809590959093752B8093742B109277
:10FC00005B2B10925A2B0E94AB818095909590931C
:10FC10005B2B80935A2B0E945B7BDF91CF911F91CE
:10FC20000F910895282F392FF90120E030E080E06E
:10FC3000A8E112C0419198E0542F5827B52FB17018
:10FC400050FD8A278695B13009F48068915011F0F3
:10FC50004695F2CF2F5F3F4F2617370759F7089584
:10FC60001F920F920FB60F920BB60F9211242F9383
:10FC70003F934F935F936F937F938F939F93AF9334
:10FC8000BF93EF93FF938091940090919500909390
:10FC9000342B8093332B81E08093252B809171004E
:10FCA000807D809371000E944A7A8091252B882361
:10FCB000E9F180919400909195002091332B30913F
:10FCC000342B82179307A0F48091F92A9091FA2A95
:10FCD000A091FB2AB091FC2A8C57914EAF4FBF4F99
:10FCE0008093F92A9093FA2AA093FB2AB093FC2AD6
:10FCF0008091940090919500821B930BA0E0B0E05E
:10FD00002091F92A3091FA2A4091FB2A5091FC2A3D
:10FD1000820F931FA41FB51F8093F92A9093FA2A8C
:10FD2000A093FB2AB093FC2A1092252BFF91EF9110
:10FD3000BF91AF919F918F917F916F915F914F9103
:10FD40003F912F910F900BBE0F900FBE0F901F9001
:10FD500018959FB7F894E1E7F0E08081807D80837B
:10FD600088B38F6288BB10929000E1E9F0E01082C6
:10FD700010929200109295001092940080818560FC
:10FD800080839FBF08952FB7F89490939900809334
:10FD9000980088B38F6288BBE1E7F0E080818260E1
:10FDA00080832FBF0895EF92FF92CF93DF93FC01E2
:10FDB000DB0185E0EB0119928A95E9F7858190E0F6
:10FDC00083709070009711F082E08C93878190E0AF
:10FDD00083709070009721F082E012968C931297B6
:10FDE000858190E083709070009799F0878190E012
:10FDF00083709070009769F023893489818592859A
:10FE00002817390731F481E0848312961C921297E7
:10FE100001C01482858183708250823030F4C82FF3
:10FE2000D0E0C650D74F888101C080E011968C93F6
:10FE30001197E781E370E250E23028F4F0E0E650F9
:10FE4000F74F808101C080E013968C931397DF9168
:10FE5000CF91FF90EF900895DF93CF9300D000D023
:10FE60000F92CDB7DEB7BE016F5F7F4F0E94D37E8A
:10FE700089819A81890F8D5F9B81890F9C81890F70
:10FE80009D81890F0F900F900F900F900F90CF9141
:10FE9000DF910895AF92BF92CF92DF92EF92FF92DF
:10FEA0000F931F93DF93CF9300D000D000D0CDB736
:10FEB000DEB78C017B01BE016F5F7F4F4E830E94D6
:10FEC000D37EC9809A81A92EBB24DB808C81682FC8
:10FED00070E095012C0D311D2D5F3F4F2D0D311D13
:10FEE000260F371F5D81250F311D4E8150E04217CF
:10FEF00053070CF4A8C0D80111964C91119750E00B
:10FF000041705070E3E0440F551FEA95E1F71296F7
:10FF10002C91129730E02170307054E0220F331F83
:10FF20005A95E1F7242B3C913770232B13963C9183
:10FF30001397E32FF0E0E170F07045E0EE0FFF1F44
:10FF40004A95E1F72E2B14963C911497E32FF0E09D
:10FF5000E170F07036E0EE0FFF1F3A95E1F72E2BBF
:10FF6000F701208315964C91159750E0437050701F
:10FF7000440F551F440F551F16962C91169730E0CD
:10FF80002370307054E0220F331F5A95E1F7242B71
:10FF900017963C9117973295330F330F307C322BE5
:10FFA000318318962C9118972283FC2DF23069F436
:10FFB00019962C91D70113962C931397F80122854B
:10FFC00014962C93149745E001C043E0E92FF0E02C
:10FFD0003B96E00FF11F542F0AC09701250F311DEA
:10FFE000C290D901CC925F5F0894A108B108A11416
:10FFF000B10499F7940FBD2DB23089F4F701E90FE0
:020000021000EC
:10000000F11DD80153962C91539720839F5FF701E0
:10001000E90FF11D54962C91549720839F5FE82F90
:10002000F0E07596E00FF11F292F08C0D701A20F4D
:10003000B11D32913C932F5F615070406115710585
:10004000A9F7890F01C080E026960FB6F894DEBFAD
:100050000FBECDBFCF91DF911F910F91FF90EF9019
:10006000DF90CF90BF90AF900895BF92CF92DF9274
:10007000EF92FF920F931F93CF93DF937C01D62EC5
:10008000EA01633008F4ADC0FC018081B82EB2945F
:10009000B694B694B3E0BB22F1E0BF22F7019181A0
:1000A000292F269526952370C92EC294C694C694EE
:1000B000A3E0CA22382F37703883382F369536950B
:1000C000369531703983382F329531703A83829565
:1000D000869581708B83BC822D83892F8295837056
:1000E0008E83CF828281888787010D5F1F4F2223F5
:1000F00061F1F801918180E0F7013381830F911D57
:100100009A87898787010B5F1F4F223081F4CA01CC
:100110000B966CE877E00E944F56F80181818B873F
:10012000F70185818C878701095F1F4F16C0233037
:10013000A1F4F7013D96DA011B9682918D93E017A9
:10014000F107D9F7085F1F4F08C0CA010B966CE88A
:1001500077E00E944F561A861986CC2089F1BB2081
:1001600059F4F801918180E02081820F911D9C8BD0
:100170008B8B0E5F1F4F04C089859A859C8B8B8B60
:10018000FC2DF23071F4CE0145966CE877E00E94C8
:100190004F56F80181818D8B80818E8B0E5F1F4FB2
:1001A00017C0FC2DF330A1F4085F1F4FD801FE01EA
:1001B000759680E09E9191938F5F8830D9F708C043
:1001C000CE0145966CE877E00E944F561C8A1B8A48
:1001D000802F8E199D2D981B9FA71EA70DA7D8169F
:1001E00008F480E0DF91CF911F910F91FF90EF9085
:1001F000DF90CF90BF9008959C0141505040460F32
:10020000571FDB0110C0FC91E0E011968C91119713
:10021000BF01680F711D260F371F2617370710F40F
:100220002F5F3F4F1296A417B50768F3A417B507C1
:1002300049F49C9180E0280F391F2817390710F4E2
:100240002F5F3F4FC9010895CF93DF939091532BB8
:10025000C92FD0E064973091522B20E0C20FD31FFA
:100260009E01280F311DC9016CE57BE248E050E09A
:100270000E94FC8064E67BE2AE010E94FC80009755
:1002800019F0382F292F02C02FEF3FEFC901DF915E
:10029000CF91089590933D1B80933C1B0895FC01E2
:1002A0004381460F40934F2B872F99272281280F98
:1002B00020934E2BA181A0934D2B508150934C2B1A
:1002C00030E02817390748F48A2F8F5F80934D2B31
:1002D000882319F45F5F50934C2B842F90E070704B
:1002E0008617970798F480914E2B8F5F80934E2B43
:1002F000882361F480914D2B8F5F80934D2B882351
:1003000029F480914C2B8F5F80934C2B0895BC0176
:10031000809155309091563008960E944F81E0911F
:100320005530F091563080914C2B808780914D2B29
:10033000818780914E2B828780914F2B83870895F0
:100340009C01AB0180E090E0B9010E94FC80382F55
:10035000292FC901089580E090E060E57BE244E147
:1003600050E00E94FC80009719F0382F292F02C01E
:100370002FEF3FEFC901089586E00E942481089580
:1003800081E10E942481089580E009C0E82FF0E017
:10039000EE0FFF1FE952FF4C118210828F5F8430F5
:1003A000A8F380E00BC0E82FF0E095E0EE0FFF1F10
:1003B0009A95E1F7E95AFF4C118E8F5F843098F3DC
:1003C00080E094E090933F1B80933E1B40E08DE0E3
:1003D00090E00EC0242F30E0289FF001299FF00DFF
:1003E000389FF00D1124E351FF4C158214824F5FAA
:1003F0004A3080F340933A1B089520913E1B309180
:100400003F1B2F5F3F4F4DE72030340710F020E0B7
:1004100030E1522F432FA0E013C0EA2FF0E0B5E007
:10042000EE0FFF1FBA95E1F7E95AFF4CB18DBB23E0
:1004300031F00480F581E02DE417F50711F3AF5F8B
:10044000A43059F730933F1B20933E1B10923A1B68
:1004500020E0E0E0F0E01EC0A22FB0E035E0AA0FFF
:10046000BB1F3A95E1F7A95ABF4C59963C91599751
:10047000332321F420933A1BFD0110C0373049F497
:10048000309731F05A964C915A97328D341708F4C0
:10049000FD012F5F243000F320933A1B3097A9F120
:1004A00022E0218F2091341B24872091351B258742
:1004B0002091361B26872091371B278728ED34E0B3
:1004C000338B228B358B248B21E030E0318B208BDA
:1004D000138E21E0228F23E0208F168A20E1278BC4
:1004E00020913E1B30913F1B322723273227358333
:1004F000248377836683DC012D913D914D915C913E
:1005000013972083318342835383CF0108950F9340
:100510001F93CF93DF9320913E1B30913F1B4DE003
:1005200050E02F5F3F4FADE720303A0710F020E05A
:1005300030E1B22FA32F10E012C0C12FD0E0C49F32
:10054000F001C59FF00DD49FF00D1124E351FF4C35
:100550000480F581E02DEA17FB0719F31F5F1A30BD
:1005600061F730933F1B20933E1B10E02DE030E0FD
:100570001AC0012F0F5FC12FD0E0C29FF001C39FAF
:10058000F00DD29FF00D1124E351FF4CDF011496C2
:10059000448155814115510529F410933A1B309738
:1005A00049F433C0102F1A3020F310933A1BE0E0C7
:1005B000F0E02BC020913E1B30913F1B32272327B8
:1005C000322711963C932E9377836683009729F404
:1005D000108211821282138209C0DC012D913D919B
:1005E0004D915C9120833183428353838DE090E071
:1005F000C89FD001C99FB00DD89FB00D1124A35141
:10060000BF4C80E418968C931897CF01DF91CF915F
:100610001F910F91089540E013C0E42FF0E0542F94
:100620005F5FEE0FFF1FE952FF4C208131812817D9
:10063000390729F440933A1B118210820895452FFF
:10064000443058F340933A1B089540E013C0E42F20
:10065000F0E0542F5F5FEE0FFF1FE952FF4C208147
:1006600031812115310529F440933A1B9183808310
:100670000895452F443058F340933A1B0895EF9264
:10068000FF920F931F93CF93DF93C0915530D0917A
:100690005630843009F4F7C108E71BE21093543058
:1006A0000093533010934B2B00934A2B833071F4FB
:1006B000898D90E08F7090708330910509F074C03F
:1006C00088899989009709F02FC78DC0823009F079
:1006D0008EC08091371B8F5F8093371B882399F4DE
:1006E0008091361B8F5F8093361B882361F4809145
:1006F000351B8F5F8093351B882329F48091341B31
:100700008F5F8093341B1092492B1092482B1092CC
:10071000EC301092EB30898D873011F0853041F448
:100720008A8D8F5F8A8F843109F0FEC6198EFCC6D0
:10073000882309F4F9C6288939892115310509F476
:100740004EC09A8D292F21502A8F992309F0ECC68B
:100750009B8D983031F0282F2150223048F495306D
:1007600039F4198E80E8809350300E944B7D95C5F6
:10077000953048F423E030E0092E02C0220F331FE9
:100780000A94E2F701C020E32A8F9F5F9B8F90E0DD
:100790008F70907083309105E1F0843091054CF4B6
:1007A0008130910509F461C38230910509F0BCC61E
:1007B0000DC08630910509F40CC58830910509F407
:1007C00008C58430910509F0AFC603C51092712B9E
:1007D0004FC384E0809350300E944B7D90C58F7052
:1007E000833009F0A1C688E0809350304BC5853036
:1007F00019F5E0915130F091523084819581009744
:1008000009F492C610925630109255300C50104098
:10081000109354300093533010934B2B00934A2B7A
:100820001092EC301092EB301092492B1092482B22
:1008300088E08093503025C1085210408091502BA1
:10084000853409F071C69091522B80E02091532B92
:100850007C01E20EF11C8091482B9091492B8E1562
:100860009F0508F461C6F092492BE092482B8091D5
:10087000562B90E08F739070009709F055C68091C9
:10088000572B882309F050C68091E7309091E830CB
:10089000C0910009D09101098C179D0759F440912E
:1008A000E9305091EA302091020930910309421752
:1008B0005307A1F02091602B3091612B2817390745
:1008C00009F032C62091622B3091632B8091E93080
:1008D0009091EA302817390709F026C60E94AB81AB
:1008E0002FEF8F3F920709F01FC68091592B86305A
:1008F00009F431C18131E9F1813009F015C68091E7
:10090000642B883009F010C61092642B8091662BFE
:100910009091672B4FEF873F940710F0099601C025
:1009200008969093672B8093662B80915C2B909117
:100930005D2BA0915E2BB0915F2B8093602B9093E9
:10094000612BA093622BB093632B8091E730909141
:10095000E830A091E930B091EA3080935C2B90931D
:100960005D2BA0935E2BB0935F2B80E4F801808712
:10097000B8C5C7014C979093492B8093482B8CE6C0
:100980009BE2909354308093533080916A2B9091E6
:100990006B2B009739F00E94C081FFEF8F3F9F07BC
:1009A00009F0C2C52091662B3091672B21153105C6
:1009B00009F4BAC58DEE90E3909352308093513094
:1009C00060910209709103094091FC085091FD0863
:1009D0000091FE081091FF0839C08481958100972D
:1009E00081F12817390769F586819781009739F0D9
:1009F000A091642BB091652BA817B90711F58081E0
:100A000091818C179D0729F4A281B381A617B7079E
:100A100039F18417950729F4A281B381A017B10792
:100A2000F9F0A0915C2BB0915D2BA817B90749F4A0
:100A3000A0915E2BB0915F2B82819381A817B9079B
:100A400079F03D96F0935230E0935130E09151307F
:100A5000F091523081E3EF36F80708F4BECF64C559
:100A6000109256301092553082E0809350308CE6D0
:100A70009BE290934B2B80934A2B1092EC30109278
:100A8000EB300E944B7D8091EB309091EC300097E1
:100A900009F44AC59C01245E3F4F3093492B2093B3
:100AA000482B3093522B2093532BE0915130F091EF
:100AB000523020852093582B21E12093592B089602
:100AC0009827892798279093692B8093682B1092F9
:100AD0006B2B10926A2B848195819093652B809368
:100AE000642B868197819093672B8093662B8091EE
:100AF000E7309091E830A091E930B091EA308093EE
:100B00005C2B90935D2BA0935E2BB0935F2B808129
:100B10009181A281B3818093602B9093612BA093EC
:100B2000622BB093632B88E79BE2909354308093C1
:100B300053300E94C0818095909590936B2B809349
:100B40006A2B009709F0CDC48FEF9FEF90936B2B2A
:100B500080936A2BC6C40E94BC81EFEF8F3F9E0733
:100B600009F0E2C48091662B9091672B009709F4FD
:100B7000DBC42091642B3091652B2115310509F4DC
:100B8000D3C4C7E5D0E3498D4423E9F06C817D816E
:100B900086179707C1F46E817F812617370799F46E
:100BA000E0915C2BF0915D2B68817981E617F70766
:100BB00051F4E0915E2BF0915F2B6A817B81E61707
:100BC000F70709F46DC1A096F0E3C73DDF07D9F63A
:100BD0002091712B2F732230B9F49093391B80939D
:100BE000381B40E00DC0E42FF0E0EE0FFF1FE9528C
:100BF000FF4C208131814F5F8217930709F46EC04B
:100C0000443088F340933A1B8091712B82FD8CC451
:100C100084E1F80181A388E290E09093492B8093CE
:100C2000482B80E580A380916B2B90916F2B938F45
:100C300030916A2B90916E2B928F368F2091692B79
:100C400090916D2B918F258F9091682B90933A1BEB
:100C500040916C2B408F948F8F5F878F882361F436
:100C6000832F8F5F868F882339F4822F8F5F858F44
:100C7000882311F49F5F948F8091642B9091652B52
:100C80009093391B8093381B2091662B3091672BF2
:100C9000F801358B248B978B868B80915C2B909100
:100CA0005D2BA0915E2BB0915F2B8093602B909376
:100CB000612BA093622BB093632B8091E7309091CE
:100CC000E830A091E930B091EA3080935C2B9093AA
:100CD0005D2BA0935E2BB0935F2BE8C310923A1B61
:100CE00080E0C0E0D0E022C0E82FF0E075E0EE0F39
:100CF000FF1F7A95E1F7E95AFF4C918D992321F472
:100D000080933A1BEF0116C0973079F4209721F0B9
:100D1000228D9A8D921748F4C82FD0E065E0CC0F51
:100D2000DD1F6A95E1F7C95ADF4C8F5F8430E0F22E
:100D300080933A1B209709F4F7C3D0935630C093A1
:100D4000553083E08A8F888F1E8A84E08F8B1B8EBC
:100D50008091662B9091672B9D838C838091642B6F
:100D60009091652B9F838E8380915C2B90915D2B5E
:100D7000A0915E2BB0915F2B88839983AA83BB835C
:100D800081E0898F8091341B8C878091351B8D8702
:100D90008091361B8E878091371B8F8781E090E092
:100DA000998B888B80916B2B8B8780916A2B8A879C
:100DB0008091692B89878091682B888781E090E0FA
:100DC0000E9487818091702B282F30E0207F307027
:100DD000213531050CF449C082958F7090E005975C
:100DE000880F991F880F991F50913B1B40E034C01A
:100DF000F901E05BF44D50A5552329F440933A1BCB
:100E000010923B1B32C0513011F44F5F25C052305D
:100E1000E1F461A56430C9F440933A1B50933B1B45
:100E200032A520E083A590E0822B932B9093391B71
:100E30008093381BF4E0893D9F0710F088ED94E023
:100E40009B8B8A8B9D8B8C8B10C0205B344DF90162
:100E500021A5222331F0420F242F30E02817390733
:100E60003CF240933A1B50933B1B80E18093712BE3
:100E70008091712B82608093712B82E08093782B1C
:100E800084E08093792B80937A2B88ED80937B2B61
:100E90008CE290E09093492B8093482B80E6B3C27C
:100EA000D0935630C0935530109250308091712BB2
:100EB00090E082FF03C0198E80E24EC22091702B19
:100EC00022952F70220F220F20933A1BB701621B2D
:100ED00071099B01245130403093492B2093482BBA
:100EE00050E04F7050704230510539F4AC014F73EF
:100EF00050704231510551F42AC04130510531F44E
:100F0000AC014F7350704230510509F12115310584
:100F100031F49C012370307021153105C1F03091FE
:100F2000682B2885321709F064C23091692B298516
:100F3000321709F05EC230916A2B2A85321709F008
:100F400058C230916B2B2B85321709F052C284FFA7
:100F50004AC0688979896115710509F444C0CE01D8
:100F60000C960E944F8130916C2B80914C2B38173E
:100F7000D1F520916D2B80914D2B2817A1F59091E3
:100F80006E2B80914E2B981771F580916F2B4091AD
:100F90004F2B841741F53C872D879E878F878B8D3C
:100FA0008823D1F42E89888D9A8D891B922F96954E
:100FB00096959695891B280F2E8B87FD81959F8985
:100FC000392F36953695931B980F9F8B822F8695D8
:100FD00086958695890F888F81E080935030888D23
:100FE0008A8F198A188A298D30E0C9018F70907014
:100FF0008430910509F4B5C18530910564F48230DF
:101000009105C9F1833091050CF0B9C0813091058B
:1010100009F08AC211C08630910509F4E2C1863018
:1010200091050CF4BEC18730910509F4E2C1883006
:10103000910509F079C28AC18091503080FF14C0B7
:1010400083E0898F80E480935030198A188A8091D8
:10105000482B9091492B009709F410C122E420936A
:1010600050300E9487810AC18091712B8F7382302A
:1010700009F05AC2FACE8091503080FF75C080913D
:10108000712B8F73823109F06FC08091702B282FE4
:1010900030E0207F3070213531050CF449C0829555
:1010A0008F7090E00597880F991F880F991F5091B6
:1010B0003B1B40E034C0F901E05BF44D50A55523E3
:1010C00029F440933A1B10923B1B32C0513011F46B
:1010D0004F5F25C05230E1F461A56430C9F44093FC
:1010E0003A1B50933B1B32A520E083A590E0822B56
:1010F000932B9093391B8093381B74E0893D97079D
:1011000010F088ED94E09B8B8A8B9D8B8C8B10C0AC
:10111000205B344DF90121A5222331F0420F242F09
:1011200030E0281739073CF240933A1B50933B1BA1
:1011300083E0898F8091682B88878091692B8987CC
:1011400080916A2B8A8780916B2B8B8781E090E05E
:101150000E94878182E480935030198A188A109205
:10116000492B1092482B8AC080E2809350300E9415
:101170004B7DE0915530F0915630118E45CD8091E8
:10118000712B80FF2AC024FD28C088899989009787
:1011900009F0CAC18091482B9091492B01960E9479
:1011A000878120915030822F8061809350308091D0
:1011B000482B9091492B009719F0226120935030D1
:1011C0000E944B7D81E090E0998B888B88E0898F2D
:1011D0001B8E81E18093712B0FC185FF1CC0509144
:1011E000762B40E08091772B90E0842B952B4091DB
:1011F000533050915430480F591F509354304093FE
:1012000053304091482B5091492B481B590B509318
:10121000492B4093482B8091482B9091492B009764
:1012200049F024FD07C020915030226020935030B7
:101230000E9487819091722B80E02091732B820F06
:10124000911D9093391B8093381B2C893D89281759
:10125000390710F0009721F43093391B2093381B85
:101260008091381B9091391B9B8B8A8B80915030D9
:1012700090E083709070009709F456C11092EC30A2
:101280001092EB300E944B7D8091503085FF07C05B
:101290001092EC301092EB30198E84E19BCF84FFDA
:1012A0000AC01092EC301092EB3081E090E0998B04
:1012B000888B84E08CCF2091EB303091EC3021157D
:1012C0003105E1F080FF02C0198A188A888999895E
:1012D000009781F48A899B898217930720F4909361
:1012E000EC308093EB308091EB309091EC30998B27
:1012F000888B04C09093EC308093EB301B8E8091F0
:101300004A2B90914B2B9093543080935330809183
:10131000EB309091EC30009759F0888999890097CB
:1013200039F088969093492B8093482B88E10BC025
:101330008091503081FFF8C088E290E09093492B73
:101340008093482B80E18093712B5CC0809150305A
:1013500080FFEAC0198E80E1809350300E944B7D5F
:10136000E3C08091482B9091492B009711F00E9487
:1013700087819091712B8091503090FF0BC080FF3E
:1013800006C087E0898F1A8E198A188A19C086E0EC
:10139000898F16C080FF1EC085E0898F198A188A40
:1013A000C3C08091482B9091492B009711F00E9467
:1013B00087818091712B80FF0DC087E0898F1A8E05
:1013C00081E090E00E94878180E1809350300E940C
:1013D0004B7D0FC08091482B9091492B009749F489
:1013E000A3C08091503080FF9FC087E0898F1A8E04
:1013F0009BC080E1F80181A388E290E09093492BA3
:101400008093482B80E58093702B888580936C2B8C
:10141000898580936D2B8A8580936E2B8B85809335
:101420006F2B8C858093682B8D858093692B8E859F
:1014300080936A2B8F8580936B2B86E08093592B4A
:101440008C819D819093652B8093642B8E819F81ED
:101450009093672B8093662B8091E7309091E830D2
:10146000A091E930B091EA3080935C2B90935D2B92
:10147000A0935E2BB0935F2B88819981AA81BB8159
:101480008093602B9093612BA093622BB093632B7E
:10149000898D84FF05C01092732B1092722B06C0A9
:1014A00084E08093722B88ED8093732B80E480938B
:1014B000582B8091482B9091492B9093522B8093DD
:1014C000532B1092772B1092762B1092752B109233
:1014D000742B0E94BC81809590959093752B80937E
:1014E000742B85E48093502B1092512B1092572B24
:1014F0001092562B80913C1B90913D1B019690932E
:101500003D1B80933C1B9093542B8093552B109242
:101510005B2B10925A2B0E94AB81809590959093F3
:101520005B2B80935A2B04C01092492B1092482BAE
:1015300010925030DF91CF911F910F91FF90EF905B
:101540000895382F292FC9010895382F292F40E0F9
:1015500050E076276727762780E090E0CB01772759
:101560006627262B372B482B592BB901CA01089522
:10157000AC01E0914A2BF0914B2B222733272E1BF5
:101580003F0B205B3F4C621773070CF49B01121654
:10159000130664F42093EB303093EC304E175F0762
:1015A00029F0CF01BA01A9010E94EAA00895ACE296
:1015B000B0E0EDEDFAE80C94FF9C29833A834B836D
:1015C0005C836D837E838F839887A986BA86CB865A
:1015D000DC86ED86FE860F87188B69807A808B808B
:1015E0009C8069A27AA28BA29CA2840173018FEFD6
:1015F0009FEFA0E0B0E0E822F9220A231B231401A8
:101600004424552469847A848B849C846DA27EA2B0
:101610008FA298A664015301A822B922CA22DB2214
:10162000340188249924C601B501A80197010E94BC
:101630007C9C69A77AA78BA79CA7C401B3010E94D1
:101640007C9C7B018C01C601B501A20191010E9425
:101650007C9C5B016C01C401B3010E947C9C9B01DA
:10166000AC01EA0CFB1C0C1D1D1D69A47AA48BA403
:101670009CA4C401AA27BB27E80EF91E0A1F1B1F42
:10168000EA14FB040C051D0520F4205030404F4F98
:101690005F4FC801AA27BB27820F931FA41FB51F46
:1016A0008D8F9E8FAF8FB8A38701FF24EE2429A5CD
:1016B0003AA54BA55CA540705070E20EF31E041FC6
:1016C000151FE98EFA8E0B8F1C8FDE2CAA8CCB8C0B
:1016D0006C8C8D8B8E8D8E8B8F8D8F8B88A1888F50
:1016E0002D853E854F85588969A17AA18BA19CA142
:1016F0000E947C9C7B018C012D813E814F8158850D
:101700006DA17EA18FA198A50E947C9CE60EF71E7C
:10171000081F191F6D897E898F89988D6E0D7F1D19
:10172000801F911F6D8B7E8B8F8B988F7E892D2DC7
:101730003A2D4C2D562D8F89988DAC96E2E10C9464
:101740001B9D0F93DF93CF93CDB7DEB760970FB696
:10175000F894DEBF0FBECDBF002309F459C0298322
:101760003A834B835C836D837E838F839887E0E22B
:10177000E01B29813A814B815C811E16BCF01986E1
:101780001A861B861C868E2F992787FD909590952B
:1017900081959F4F04C0220F331F441F551F8A9508
:1017A000D2F72D873E874F87588B2AC0CA01B901CF
:1017B000002E04C0660F771F881F991F0A94D2F766
:1017C00069877A878B879C87DA01C90104C0B6953F
:1017D000A79597958795EA95D2F72D813E814F8100
:1017E000588504C0220F331F441F551F0A95D2F796
:1017F000822B932BA42BB52B8D879E87AF87B88B1D
:1018000029853A854B855C856D857E858F85988990
:1018100060960FB6F894DEBF0FBECDBFCF91DF91BB
:101820000F9108950F93DF93CF93CDB7DEB76097F5
:101830000FB6F894DEBF0FBECDBF002309F459C028
:1018400029833A834B835C836D837E838F83988760
:1018500060E2601B8D819E81AF81B8851616CCF049
:101860009C01AD01550F220B322FA9012D873E8718
:101870004F87588B262F332727FD3095309521959C
:101880003F4F04C0B595A795979587952A95D2F7B0
:1018900024C09C01AD01002E04C055954795379595
:1018A00027950A94D2F72D873E874F87588B04C01F
:1018B000880F991FAA1FBB1F6A95D2F729813A8109
:1018C0004B815C8104C056954795379527950A95BD
:1018D000D2F7822B932BA42BB52B89879A87AB87C2
:1018E000BC8729853A854B855C856D857E858F858E
:1018F000988960960FB6F894DEBF0FBECDBFCF912A
:10190000DF910F910895A0E1B0E0E9E8FCE80C94C4
:10191000079D29833A834B835C836D837E838F830A
:101920009887A986BA86CB86DC86ED86FE860F87E9
:10193000188B2D813E814F8158858D859E85AF8581
:10194000B889281739074A075B07C8F08217930739
:10195000A407B50790F029813A814B815C81898584
:101960009A85AB85BC85281739074A075B0738F08D
:1019700082179307A407B50720F482E003C080E034
:1019800001C081E06096EAE00C94239DACE4B0E0F5
:10199000ECECFCE80C94FF9CF50129833A834B8323
:1019A0005C836D837E838F839887A986FA87CB8635
:1019B000DC86ED86FE860F87188B8D809E80AF803B
:1019C000B884B7FE66C02195B1E0121608F0B0E009
:1019D0003195A1E0131608F0A0E0232E2B1AB22DAA
:1019E000BB24B394321508F0BB24AB29419531E0F8
:1019F000141608F030E0342E3A1AA32DBB24B39409
:101A0000431508F0BB243B29519541E0151608F019
:101A100040E0A52EA31A31E05A1508F030E0432B20
:101A2000619531E0161608F030E0B62EB41A41E0A8
:101A30006B1508F040E0342B719541E0171608F063
:101A400040E0572F531B31E0751708F030E0432B6F
:101A5000819531E0181608F030E0482E441A442DE4
:101A600061E0841508F060E0362B9195931B298383
:101A7000BA83AB83AC82BD825E834F8398872FEF9E
:101A80003FEFA90121962CAF3DAF4EAF5FAF21973D
:101A900006C021961CAE1DAE1EAE1FAE21978D85D1
:101AA0009E85AF85B889B7FF68C021964CAD5DAD06
:101AB0006EAD7FAD219740955095609570952196BC
:101AC0004CAF5DAF6EAF7FAF2197E19581E01E1601
:101AD00008F080E0F19591E01F1608F090E04F2F9C
:101AE000481B81E0F41708F080E0982BC19481E056
:101AF0001C1408F080E06C2D691B91E0C61608F0FC
:101B000090E0892BD19491E01D1408F090E05D2DB8
:101B1000581B81E0D51608F080E0982BE19481E015
:101B20001E1408F080E03E2D391B91E0E31608F00A
:101B300090E0892BF19491E01F1408F090E02F2D94
:101B4000281B81E0F21608F080E0982B019581E0D7
:101B5000101608F080E0702F791B972F71E009179D
:101B600008F070E0872B1195181BE9874A876B876F
:101B70005C873D872E879F87188B79856A855B8573
:101B80004C853D852E859F858889E981E98BEA8191
:101B9000EA8BEB81EB8BEC81EC8BED81ED8BEE81B5
:101BA000EE8BEF81EF8BE885E88F798F6A8F5B8F03
:101BB0004C8F3D8F2E8F9F8F88A3E98CFA8C0B8DD5
:101BC0001C8D2D8D3E8D4F8D58A189899A89AB89A9
:101BD000BC898DAB9EABAFABB8AFAD88BE88CF88AC
:101BE000D88C211531054105510509F0BEC3AE144D
:101BF000BF04C006D10608F04FC190E0E91690E09E
:101C0000F90691E0090790E0190758F4AFEFEA16DA
